:020000040800F2
:10000000E81E002095020008A5300008D52E000843
:10001000A13000084B1F00088D4C000800000000B4
:100020000000000000000000000000000738000889
:100030005D29000800000000DD3200087942000858
:10004000AF020008AF020008AF020008AF020008CC
:10005000AF020008AF020008AF020008AF020008BC
:10006000AF020008AF020008AF020008AF020008AC
:10007000AF020008AF020008AF020008AF0200089C
:10008000AF020008AF020008AF020008AF0200088C
:10009000D14A0008AF020008AF020008AF02000812
:1000A000AF020008AF020008AF020008AF0200086C
:1000B000AF020008AF020008AF020008AF0200085C
:1000C000AF020008AF020008AF020008AF0200084C
:1000D000AF02000825450008AF020008AF02000883
:1000E000AF020008AF0200081B48000800F002F849
:1000F00000F0B0F80AA090E8000C82448344AAF112
:100100000107DA4501D100F0A5F8AFF2090EBAE80F
:100110000F0013F0010F18BFFB1A43F0010318473B
:100120004C5800006C5800000A444FF0000C10F8C6
:10013000013B13F0070408BF10F8014B1D1108BF65
:1001400010F8015B641E05D010F8016B641E01F805
:10015000016BF9D113F0080F1EBF10F8014BAD1C55
:100160000C1B09D16D1E58BF01F801CBFAD505E073
:1001700014F8016B01F8016B6D1EF9D59142D6D3CD
:10018000704700000023002400250026103A28BFF5
:1001900078C1FBD8520728BF30C148BF0B607047F9
:1001A0006E2900F01A83702900F06F84662905F02B
:1001B0000183652905F0FE82672905F0FB8261292C
:1001C00005F0FA8203681B0A28BF41F08001692903
:1001D00000F0A080642900F09D80752900F09A80CD
:1001E0006F2900F0FC83782900F03B84E92900F0B6
:1001F0009783E42900F09483F52900F09183EF2997
:1002000000F0F983F82900F03A840368DB0928BF7D
:1002100041F08001632901F05180732901F056807B
:10022000E32901F06180F32901F066800020704726
:100230001FB501F0B7F804000020002105F0A4FA72
:10024000401C60600020002105F088FAE0601FBDBE
:1002500010B510BD01F078F81146FFF7E9FF05F081
:1002600067F801F055F903B4FFF7F2FF03BC04F09F
:10027000D2FF0000EFF30980704780F309887047D0
:10028000EFF30880704780F30888704740BA7047E2
:10029000C0BA70470948804709480047FEE7FEE7B3
:1002A000FEE7FEE7FEE7FEE7FEE7FEE7FEE7FEE726
:1002B00004480549054A064B704700007D42000886
:1002C000ED000008E8180020E81E0020E81A0020D1
:1002D000E81A0020704700001CB50C46064B7B4412
:1002E00069460090204600F092FA044600206946D4
:1002F00000F0A0FA20461CBD530500000FB40449CD
:1003000010B503AA029800F09BFA10BC5DF814FB2C
:10031000480000202DE9F0410646002410687529A8
:10032000314616A510D000F0C4F9002802DA404288
:1003300013A507E031688A0701D512A502E0490735
:1003400004D511A5012401E000F0BCF900210A2226
:1003500006F1240709E0B0FBF2FCB0FBF2F302FB6C
:100360001C00303078541846491C0028F3D123462D
:100370002A463046BDE8F04100F0D6B90000000042
:100380002D0000002B000000200000002DE9F05F90
:10039000894604464FF0000ADFF874B1FB44C0F808
:1003A00020A02046E1688847002874D0252806D080
:1003B000D4E901219047206A401C2062F1E7002621
:1003C0005F462046E16888472028054607DB312D37
:1003D00005D2781910F8200C08B10643F1E7B007F0
:1003E00001D526F00406C4F81CA00027C4F818A004
:1003F0002A2D09D0284604F007FF38B304EB8708FC
:10040000303DC8F8185019E059F8041B204604EB99
:1004100087029161E1688847012F054618D1E0699C
:10042000002820DA26F020061DE0D8F8180000EB9E
:10043000800005EB40003038C8F818002046E1681D
:100440008847054604F0E0FE0028EED1012F0AD0CF
:100450002E2D08D12046E16888477F1C0546022FD3
:1004600046F02006C4DBA069002803DA404246F0CB
:100470000106A061F00701D026F010066C2D0BD00C
:10048000682D09D04C2D39D06A2D35D0742D35D03A
:100490007A2D33D016E038E0E1682F4620468847B1
:1004A000B842054609D16C2F26D04FF48060E16830
:1004B000064320468847054604E06C2F1AD04FF4C7
:1004C000807006430DB3A5F14100192802D82035EC
:1004D00046F400664A462946204626604E46FFF707
:1004E0005FFE80B101280BD0F61D26F0070000F159
:1004F000080956E74020E4E78020D8E70020D6E747
:1005000006F104094DE7284652E7206ABDE8F09F4E
:10051000CD54000010B5431C02E010F8011B71B16E
:100520008107FAD14FF0013202C88C1A8C4314EAC9
:10053000C211F9D0C01A0A0603D0C01E10BDC01ADD
:1005400010BD0A0401D0801E10BD0902FCD0401E5F
:1005500010BD032A40F2308010F0030C00F015802B
:1005600011F8013BBCF1020F624498BF11F801CBB6
:1005700000F8013B38BF11F8013BA2F1040298BF1B
:1005800000F801CB38BF00F8013B11F0030300F085
:100590008782083AC0F0088051F8043B083A51F8C5
:1005A00004CBA0E80810F5E7121D5CBF51F8043B2E
:1005B00040F8043BAFF30080D20724BF11F8013BA1
:1005C00011F801CB48BF11F8012B24BF00F8013B03
:1005D00000F801CB48BF00F8012B70474FF0013CF9
:1005E00050F8042B51F8043B9A4221D1A2EB0C03A2
:1005F000934313EACC1317D150F8042B51F8043B62
:100600009A4215D1A2EB0C03934313EACC130BD1FE
:1006100050F8042B51F8043B9A4209D1A2EB0C0389
:10062000934313EACC13DBD04FF00000704700BFB8
:10063000D01A01BAB1FA81F101F0180122FA01F0E1
:10064000CB40C1F12001DBB2C0B2C01A2CFA01F3D9
:10065000D11A914311EAC311E6D170477047704730
:100660007047704770B5044685690068C10601D5BA
:10067000302600E02026C00707D070BDD4E9012154
:1006800030469047206A401C20626D1EF6D570BD32
:1006900070B5044685690078C00707D170BDD4E9FC
:1006A000012120209047206A401C20626D1EF6D553
:1006B00070BD09684A0501D540B27047C905FCD52F
:1006C00000B2704709684A0501D5C0B27047C90534
:1006D000FCD580B2704770B50C460546012A05D09E
:1006E0002878800600D5EA69002302E0012305E0AE
:1006F0005B1C934202D2E05C0028F9D1A869E6189D
:10070000C01AA861286A184428622846FFF7AAFF81
:1007100004E0D5E9012114F8010B9047B442F8D365
:100720002846FFF7B5FF70BD2DE9F0470D46994605
:100730009246044600F124080168880604D5E06961
:1007400021F01001216000E00120A84201DD471BDB
:1007500000E00027A1697A1902EB0900081AA061DC
:100760002078C00602D42046FFF77CFF002608E070
:10077000D4E901211AF806009047206A401C761C33
:1007800020624E45F4DB2078C0060AD52046FFF7EC
:1007900069FF06E0D4E9012130209047206A401C1F
:1007A0002062381EA7F10107F4DC07E0D4E901213B
:1007B00018F805009047206A401C2062281EA5F109
:1007C0000105F3DC2046FFF763FF2078000602D521
:1007D0000220BDE8F0870120FBE711680268006A8B
:1007E000530501D508700AE0D30501D5088006E05D
:1007F000130603D5C217C1E9000200E0086001201A
:100800007047000001694A1C02610878704700B512
:100810008FB0CDE901310021059105497944CDE939
:10082000031011466846FFF7B1FD0FB000BD000090
:10083000E5FFFFFF0A6802F8010B0A60704700003D
:10084000074B70B50D467B44FFF7E1FF0446284691
:1008500000F056FD10B14FF0FF3070BD204670BD66
:10086000634A00002DE9FF5F15468A460446DFF81B
:10087000AC80F8440027D8E900103E46CDE90010CE
:1008800010E03AF816106A4602A800F03DFD411C3F
:1008900007D02178890603D5E269391891420DD82D
:1008A0000744761C2078800602D5E069B84205DD51
:1008B000AE42E6DB3AF816000028E2D1A069C01B80
:1008C000A0612046FFF7CEFED8E90010CDE9001068
:1008D000002017E03AF818106A4602A800F014FD4C
:1008E000B0F1FF3F81460BD000250DF1080B05E06C
:1008F000D4E901211BF8050090476D1C4D45F7D345
:1009000008F10100B0428046E4DB206A38442062EE
:100910002046FFF7BDFEBDE8FF9F00000A50000023
:100920002DE9F0418046D21D22F007020025D2E9D0
:100930000002F52915A614D0011E72F1000106DA95
:100940000023D0EB030063EB020211A608E0D8F805
:1009500000108B0701D50FA602E0490701D50EA6AE
:1009600001251146002408F1240704E000F0CAF82C
:1009700030323A55641C50EA0102F7D12B46324618
:1009800021464046BDE8F041FFF7CEBE0000000022
:100990002D0000002B0000002000000030B40021DA
:1009A00000F1240408E002F00705D208303542EADD
:1009B0004372DB086554491C52EA0305F3D104680D
:1009C000002310A2250707D5A40600D421B1C469CD
:1009D00001230DA2641EC46130BCFFF7A5BE10B593
:1009E000044621461068FFF76DFE02462046BDE82A
:1009F00010400023D2E7D21D22F00701D1E90023E5
:100A0000CCE700000000000030000000F0B40D460C
:100A10000188090502D5214C7C4402E01F4C7C442E
:100A20000E34002100F1240608E002F00F0712093D
:100A3000E75D42EA03721B097754491C52EA030737
:100A4000F3D102780023120704D5702D06D009B126
:100A5000022311342246F0BCFFF766BE0123103496
:100A6000F8E770B504460D4621461068FFF72AFEE8
:100A7000024629462046BDE870400023C6E7D21D45
:100A800022F00703D3E90023C0E70368126843F0AC
:100A9000200303600823C3610023B7E76C4E000006
:100AA00010B5203AC0F00B80B1E81850203AA0E809
:100AB0001850B1E81850A0E81850BFF4F5AF5FEA3D
:100AC000027C24BFB1E81850A0E8185044BF18C9F0
:100AD00018C0BDE810405FEA827C24BF51F8043B97
:100AE00040F8043B08BF7047D20728BF31F8023BEB
:100AF00048BF11F8012B28BF20F8023B48BF00F87F
:100B0000012B704730B5B0F10A024FEA900E71F137
:100B100000034EEA817EB0EB0E0061EB91014FEADB
:100B2000101E4EEA017E10EB0E0041EB11114FEA50
:100B3000102E4EEA016E10EB0E0041EB11214FEA30
:100B4000104E4EEA014E10EB0E0041EB11414018E1
:100B500041F100014FEAD00040EA41704FEAD10173
:100B600010EB80054FEA810444EA907444EB0104E1
:100B70006D1944EB0404521BA3414FF0000348BF1E
:100B80000A3200D530BD401C41F1000130BD704734
:100B90002DE9FF4F0C461E464FF0FF378BB0D2E9D0
:100BA0000001DDF860800A908A46C1F30A5505B954
:100BB0003D46002108464FF00000BAF1000F00F456
:100BC000400005DA00EB80004FF4400101EA5000DC
:100BD0004FEA9059B9F1010F00DDB9460A9850EA81
:100BE0004A000ED044F61050A5F2FF3545432F14AD
:100BF000B8F1000F1ED07542291E1EDDC9F100029A
:100C00001CE0B8F1010F4FF0000001D0302103E0EB
:100C1000F24305E02154401CB042FBDB3046002289
:100C2000002121540B99C1F80880C1E900200FB0C0
:100C3000BDE8F08FBD1B6D1CDEE74A4600DA694255
:100C400006A800F0F3FB06AB93E8070003AB83E8CC
:100C5000070050460A9900F069FC8DE80700A0F5EE
:100C600000501F3800900398002D0ADD42F21F014A
:100C70004A460844002303A90390684600F0D2FEC8
:100C800009E0A0F500504A461F38002303A903904D
:100C9000684600F0DCFE8DE807000004000C03D07D
:100CA0004FF0FF30410800E01046B8F1000F03D0CC
:100CB0000022009215461EE0751E05D4FFF722FFA4
:100CC000303262556D1EF9D5B3460122084302D079
:100CD00000227F1C04E02078302801D100227F1EF2
:100CE000002A099784D01DE0112D07DAFFF70AFFCB
:100CF000303262556D1C50EA0102F5D1084302D032
:100D00000098C8B10EE00021681E05E0235C625C1B
:100D100063542254401E491C8142F7DBAB46A81B9A
:100D2000401E0990002004F80B000B98099AC0F8A7
:100D30000880C0E9002B7AE711264FF0000857E73A
:100D40002DE9F04F88460446D21D22F0070191B0EC
:100D5000D1E90001CDE90A0104F042FA02460B98FC
:100D6000C00F01D02D2007E02068810701D52B207E
:100D700002E0202101EAC000032A099001D0072ADD
:100D800005DB03464146204600F010FB0BE12078CE
:100D9000800601D5E06900E00620B8F1650F8146C4
:100DA00006D0B8F1660F18D0B8F1670F70D131E0F6
:100DB0000020B9F1110F009001DB112301E009F1CE
:100DC00001030AAA01A90CA8FFF7E2FEDDE90C70F5
:100DD000002609F10105834647E001204B460090BB
:100DE0004FF000470AAA01A90CA8FFF7D1FEDDE9E0
:100DF0000DB00C995D46002610B909F101000D18DF
:100E0000B9EB050003D4C0F1FF3609F10105A5EBEC
:100E100009002BE0B9F1010F01DA4FF001090020C0
:100E2000B9F1110F0090484601DD112300E003469F
:100E30000AAA01A90CA8FFF7ABFEDDE90C704D462C
:100E400000268346207800070AD4AB4500DA5D46C9
:100E500001A8012D04DD411911F8011C302907D02A
:100E60004F4502DA17F1040F04DA012082460FE041
:100E70006D1EEEE7002F02DCED1B3E4403E0781C04
:100E8000A84200DD7D1CB81B00F1010A4FF00047AD
:100E90002078000703D4AA4501DB4FF0FF3A002178
:100EA000B7F1004F0DF143088DF8431024D0022014
:100EB0002B23002F01DA7F422D230A21021EA0F1ED
:100EC000010000DC5FB197FBF1FC97FBF1F201FB45
:100ED0001C7C17460CF1300C08F801CDEEE7A8F1A8
:100EE000010003702188090501D5452100E0652135
:100EF000A0F1010800F8011C09980FA9A1EB08074F
:100F0000FF1D00B10120411901EBEA70A1693844CD
:100F1000081A401EA0612078C00602D42046FFF7C0
:100F2000A1FB099828B1D4E901219047206A401C0F
:100F300020622078C00622D52046FFF793FB1EE0F2
:100F4000002E04DBB34502DD01A8805D00E0302007
:100F5000D4E901219047206A401C2062761CAAF146
:100F600001005FEA000A0AD100F01CFAC0680168BB
:100F7000405CD4E901219047206A401C2062281E71
:100F8000A5F10105DCDC07E0D4E9012118F8010B2B
:100F90009047206A401C2062381EA7F10107F3DC4D
:100FA0002046FFF775FB032011B041E62DE9F04F15
:100FB00004460D46D21D22F0070089B0D0E9009703
:100FC0004846394604F00CF90246F80F01D02D23AB
:100FD00007E02068810701D52B2302E0202101EAE8
:100FE000C0038DF820300BB1012000E00020032A5F
:100FF000824601D0072A04DB2946204600F0D6F9B4
:101000003FE12078800601D40D2500E0E569C7F3B3
:101010000A560D2D49DA00214FEA175B08464FF0BA
:101020000000002F00F4400007DA00EB80004FF4CE
:10103000400100EBD07001EA60008115012901DD5B
:101040004FF0FF3100224FEA850CBCF1180F06D398
:101050001346ACF118004FF08052C24003E04FF449
:10106000801323FA0CF30CF10C0CBCF1200F04D309
:10107000ACF1200C09FA0CF001E007FA0CF00029A1
:101080004FF0004801DD18B90FE00ED140450CD3F8
:1010900019EB02095F4121B9404502D19F4329EA7A
:1010A0000209BBEB175F00D0761C2088000502D533
:1010B0007B48784402E07A487844193808AA3023FB
:1010C00002F80A30037C0AF10101002E0AF1020A3B
:1010D00053546A4602DC4FF0300101E04FF0310119
:1010E0004FF001088DF8001002D0A6F2FF3603E0A1
:1010F00059EA470100D06B4E002D02DC2178090728
:1011000004D54FF002082E218DF80110C4460021AD
:101110000BE0C7F303433F01C35C491C6D1E02F89B
:101120000830052908F1010801DA002DF1DC002161
:101130000CE000EB1973491C1B786D1E082902F89E
:1011400008304FEA091908F1010801DA002DF0DC36
:1011500021688B0602D516E0A8F10108E04505DDFF
:1011600002EB080313F8013C302BF5D0B8F1000F67
:1011700009DD02EB080313F8013C2E2B03D109070C
:1011800001D4A8F10108002D05DD3E2102F8081068
:101190006D1E08F10108407C002E02F8080008F1DD
:1011A000010804DA2D20764202F8080002E02B2024
:1011B00002F808000A214FF47A70864208F101080B
:1011C0000BDB96FBF0F3303302F8083096FBF0F3BC
:1011D00008F1010800FB136601E0642E0CDB6420BB
:1011E00096FBF0F3303302F8083096FBF0F308F189
:1011F000010800FB136601E00A2E06DB96FBF1F006
:10120000303002F8080008F1010896FBF1F001FB0C
:101210001060303002F80800A16908F1010808EBFD
:10122000050202EB0A00081AA0612078C00602D469
:101230002046FFF717FA216A08AE01EB0A00206288
:1012400004E0D4E9012116F8010B9047BAF1010A34
:10125000F7D22078C00602D52046FFF703FA6E4683
:1012600009E016F8010B3E280FD0D4E90121904780
:10127000206A401C2062B8F10108F2D22046FFF734
:1012800007FA09B00320BDE8F08F206A28442062E5
:1012900003E0D4E90121302090476D1EEBD3F8E73D
:1012A0000D48000002FCFFFF10B5436913B1AFF316
:1012B000008001E0FFF70FFA012010BD127800F165
:1012C00024010A7000224A700122EDE711684FF0F4
:1012D000FF32E9E710B5436913B1AFF3008001E0D5
:1012E000FFF7C0FA012010BD128800F124018284AA
:1012F0000022C2840122EDE711684FF0FF32E9E7D6
:10130000007B00F08000704770B516460C4605461D
:1013100000F040F8036893F80101012806D0FF2C83
:101320000FD8185D68B101202C7070BDD3F807018B
:101330003246214603F2071303442846BDE87040B5
:1013400018474FF0FF3070BD754600F0EBF8AE4621
:1013500005006946534620F00700854618B020B5C1
:10136000FEF7A6FFBDE820404FF000064FF0000753
:101370004FF000084FF0000B21F00701AC46ACE83D
:10138000C009ACE8C009ACE8C009ACE8C0098D46AA
:101390007047000010B500F005F8001D10BD00BF3B
:1013A000E943000000487047A41800202DE9F041EF
:1013B0001F46044603260168072A01F4006004DB87
:1013C00008B116A505E016A503E008B115A500E0D3
:1013D00015A521F010002060A069C01EA0610FB10A
:1013E000401EA0612046FFF73DF94FB1D4E901212D
:1013F00038469047206A401C2062C01C206206E0EC
:10140000206AFAE7D4E9012115F8010B9047761E0E
:10141000F8D22046FFF73CF9BDE8F0814E414E007E
:101420006E616E00494E4600696E66002DE9F04718
:10143000814616468AB0354878440DC88DE80D00BF
:1014400032487844801C03AC0DC884E80D0041F696
:101450009B300844372190FBF1F290FBF1F5A5F1A8
:10146000800501FB12041B3C02D56442012000E010
:101470000020DFF898A080460027FA44AAF1BE0AAF
:101480000EE0E0070AD03246684607EB4701012329
:101490000AEB810100F0DBFA8DE8070064107F1C85
:1014A000002CEED1194F7F44AE3F19E0E80715D06C
:1014B00007EB04100DF1180A90E80E008AE80E0000
:1014C000C068F04201D1981908903246012306A95C
:1014D00003A800F0BCFA03AB83E807006D10641C9E
:1014E000002DE3D14FF0010332466946B8F1000FF9
:1014F00003A802D000F096FA01E000F0A8FAC9E9CA
:101500000001C9F808200AB0BDE8F08718450000BE
:1015100010B50446AFF300802046BDE81040FEF74A
:10152000A2BE000000487047841800205FEA400C0B
:1015300008BF91F0000F4FEA8C234FEAC12243EA23
:1015400051514FEA1C5018BF00F5F0404FEA3000EF
:1015500018BF41F000415FEA6C5C00F02980BCF1EB
:10156000FF3F08BF40F080407047130C06BF1204D5
:101570004FF0100C4FF0000C130E04BF12020CF1D0
:10158000080C130F04BF12010CF1040C930F04BFDD
:1015900092000CF1020CD30F04BF52000CF1010CAD
:1015A00011464FF00002A0F11F00A0EB0C007047A5
:1015B00011F0004F08BF704731F000413FF4D5AF44
:1015C0000B0C06BF09044FF0100C4FF0000C0B0E73
:1015D00004BF09020CF1080C0B0F04BF09010CF148
:1015E000040C8B0F04BF89000CF1020CCB0F04BF5D
:1015F00049000CF1010CCCF12003A0EB0C0022FA05
:1016000003F302FA0CF241EA030100F10100704712
:1016100020F07F4C80EA030023F07F47ACEB070308
:1016200003F57C5300F0004003F1FF032DE98049EE
:101630004FEA154B09B44FEA144325EA0B4E24EA4E
:1016400003480FF2042606EB132749083E785FEAA9
:10165000320203FB0667C7F5000707FB06F64FEAF1
:1016600054374FEAD64606F1020607FB066CCCF16A
:10167000005C4FEA1C472CEA074C07FB06F40CFB06
:1016800006F504EB15464FEA961634BF00204FF0DE
:1016900000404FEAD13706FB07FC4FEA1C4C0CFB1D
:1016A0000BF7D21B03FB0CF761EB07010CFB0EF7EA
:1016B000B0EB074072EB17420CFB08F734BFA2EB0C
:1016C0000742B2EB074261EB17414FEA0C444FEA85
:1016D000910706FB07FC4FEA1C4C0CFB0BF7B0EB29
:1016E000C74072EB573203FB0CF734BFA2EBC74283
:1016F000B2EBC74261EB57310CFB0EF7B0EBC70002
:1017000072EB57720CFB08F734BFA2EBC702B2EBC7
:10171000C70261EB5771039F4FEA816141EA921161
:1017200004EBCC044FEAD1374FEA826206FB07FC98
:1017300042EA90124FEA80604FEA1C4C0CFB0BF718
:10174000D21B03FB0CF761EB07010CFB0EF7B0EBB0
:10175000074072EB17420CFB08F734BFA2EB0742BD
:10176000B2EB074261EB17414FEA8C554FEA910704
:1017700004EB9C2406FB07FC4FEA1C4C0CFB0BF70C
:10178000B0EBC74072EB573203FB0CF734BFA2EB50
:10179000C742B2EBC74261EB57310CFB0EF7B0EB1F
:1017A000C70072EB57720CFB08F734BFA2EBC702FD
:1017B000B2EBC70261EB577115EB4C254FEA816123
:1017C00041EA92114FEA82624FEAD13742EA90121F
:1017D00006FB07FC44F100044FEA80604FEA1C4C12
:1017E0000CFB0BF7D21B03FB0CF761EB07010CFBA7
:1017F0000EF7B0EB074072EB17420CFB08F734BF53
:10180000A2EB0742B2EB074261EB174115EB1C1547
:101810004FEA813141EA92414FEA823242EA9042F4
:101820004FEA80304FEA0C7644F1000448EA034363
:101830004EEA0B484FF0000EB2EB080C71EB0307B9
:1018400024BF624639464EEB0E0E4FF0000B0018D7
:10185000524149414BEB0B0BB2EB080C71EB030708
:101860007BF1000B24BF624639464EEB0E0E4FF063
:10187000000B0018524149414BEB0B0BB2EB080C2B
:1018800071EB03077BF1000B24BF624639464EEB38
:101890000E0E51EA020718BF46F0010616EB0E764F
:1018A00055F1000254F1000103D5BDE88901BDE8FE
:1018B0000088BDE88901BDE80048B619524141EBF6
:1018C0000101A3F10103704780807F7E7D7C7B7ADC
:1018D0007978777676757473727171706F6E6E6DDC
:1018E0006C6C6B6A6A696868676666656464636382
:1018F00062616160605F5F5E5E5D5D5C5C5B5B5A08
:101900005A59595858575756565555555454535374
:1019100052525251515050504F4F4F4E4E4D4D4DCF
:101920004C4C4C4B4B4B4A4A4A494949484848471A
:101930004747474646464545454444444443434358
:101940004342424242414141002B9C4630D4770001
:101950002BD01CB54FEA370703B44FF010004FF0FF
:101960001001BAF1000F06D0BCF1000FDCBF40F04F
:10197000080040F008014FF000000FBCBDE8104027
:101980000BF1010BBBF1010F08BF5FEA170722BF84
:1019900012F1010211F101014FF0004143F1000386
:1019A00000F0004043EA00007047F9D35708D0E741
:1019B00046EA064613F1400F4FEA16461FDD13F1C3
:1019C000200FDFBF16430A46002120335B42BED002
:1019D000C3F1200746EA064602FA07F74FEA164621
:1019E00046EA0706C3F1200722FA03F201FA07F7D5
:1019F00021FA03F14FF0000342EA0702A7E746EAA3
:101A0000020646EA06464FEA164646EA0106BCBF0B
:101A100046EA0646360C4FF000034FF000024FF046
:101A2000000194E72DE9804C9A46934670B491E802
:101A3000380007C831EA400C48BF34EA430C03D5EC
:101A4000FFF7E6FDFFF780FFF0BCBDE8008C2DE955
:101A5000804C9A46934670B491E8380007C810F05D
:101A6000804F08BF13F0804F03D100F005F8FFF757
:101A70006BFFF0BCBDE8008C20F07F4780EA0300DC
:101A800023F07F4C07EB0C03A3F57C5300F00040E0
:101A9000A3F1FE0392F0000F00F0B38095F0000F69
:101AA00000F077802DE901494FEA11404FEA1446D2
:101AB00021EA004800FB06FC24EA064708FB06F67C
:101AC00007FB08F800FB07F718EB06484CEB164C31
:101AD0004FEA124B18EB07484FEA15464CEB1740FC
:101AE00022EA0B4E0BFB06FC25EA06470EFB06F628
:101AF00007FB0EFE0BFB07F71EEB064E4CEB164CDE
:101B00004FF000061EEB074E4CEB174B18EB0B0883
:101B100040F1000018EB0E0B58EB000840F10000FC
:101B20008F1A4FF000013CBFC943661B14BFB5EBD1
:101B3000040C00213CBFC943F61B4FEA17444EEA90
:101B40008E0E27EA04454FEA1C4704FB07622CEA85
:101B5000074C05FB07F70CFB05F604FB0CFC16EB2A
:101B6000074642EB174216EB0C4642EB1C421BEBBE
:101B7000060658EB0202414146EA9E0601D5BDE841
:101B80000189B619524141EB0101A3F10103BDE8FE
:101B900001894FEA14454FEA114724EA054621EA34
:101BA000074C05FB07F406FB07F70CFB06F105FBEA
:101BB0000CFC11EB074144EB17444FEA124711EBC1
:101BC0000C4144EB1C4422EA074C05FB07F206FBE0
:101BD00007F70CFB06F605FB0CFC16EB074642EB81
:101BE000174216EB0C4642EB1C456A1854F10001F3
:101BF00048BF7047B619524141EB0101A3F10103FF
:101C0000704795F0000F37D04FEA11424FEA144762
:101C100021EA024624EA074C02FB07F106FB07F71C
:101C20000CFB06F402FB0CFC14EB074441EB1741E0
:101C30004FEA154714EB0C4441EB1C4125EA074CD5
:101C400002FB07F506FB07F70CFB06F602FB0CFC94
:101C500016EB074645EB174516EB0C4645EB1C42C9
:101C6000121951F1000148BF7047B619524141EBBA
:101C70000101A3F1010370474FEA14454FEA1147F0
:101C800024EA054621EA074C05FB07F106FB07F7A6
:101C90000CFB06F24FF0000605FB0CFC12EB0742B2
:101CA00041EB174112EB0C4251EB1C4148BF70470E
:101CB000921841EB0101A3F10103704721B1826841
:101CC00042F00102826003E0826822F00102826039
:101CD0007047000000B587B000F032FB01214802D8
:101CE00001F090FB0121042001F06CFB7F20ADF896
:101CF000040004208DF8070001A9294801F005F827
:101D00004FF4804001F052FB0020029001208DF83A
:101D10000C008DF80D004FF4602004900020059019
:101D200005208DF8180002A91E4800F075F805235B
:101D3000012200211B4800F097F80523022201210F
:101D4000184800F091F8052303220221154800F0FD
:101D50008BF8052304220321124800F085F805239F
:101D60001A4604210F4800F07FF801210D4800F0C9
:101D70001BF801210B48FFF7A1FF0A4800F0D0F83B
:101D8000084800F0DDF800BF064800F03BF80028E6
:101D9000FAD10121034800F0C8F807B000BD0000E7
:101DA000000801400024014021B1826842F48072A1
:101DB000826003E0826822F480728260704730B5EE
:101DC00002461161022008E0C0F1050552F82550D5
:101DD00014692C441461441CE0B20528F4DD052488
:101DE0001069B0FBF4F01061108A83B2002005E0A6
:101DF00052F82050441E42F82450401C0528F7DBBE
:101E0000184630BD014600208A6802F004020AB17B
:101E1000012000E00020704730B50246002000237A
:101E200050680F4C20400D790C6844EA052420438B
:101E3000506090680B4C2040D1E902542C434D79FE
:101E400044EA450420439060D06A20F470000C7C82
:101E5000641EE4B2234340EA0350D06230BD000068
:101E6000FFFEF0FFFDF7F1FFF0B504460D46002040
:101E70000021092D11DDE068A5F10A0606EB4607F1
:101E8000072606FA07F18843A5F10A0606EB46067F
:101E900003FA06F10843E0600CE0206905EB450712
:101EA000072606FA07F1884305EB450603FA06F113
:101EB00008432061072A0FDA606B561E06EB86077F
:101EC0001F2606FA07F18843561E06EB860605FA1A
:101ED00006F10843606322E00D2A0FDA206BD61F5B
:101EE00006EB86071F2606FA07F18843D61F06EB86
:101EF000860605FA06F10843206310E0E06AA2F1C5
:101F00000D0606EB86071F2606FA07F18843A2F1A5
:101F10000D0606EB860605FA06F10843E062F0BD01
:101F2000816841F008018160704721B1826842F404
:101F3000A002826003E0826822F4A00282607047FF
:101F4000816841F004018160704700BFFEE7000036
:101F500010B50446082C51D2DFE804F050040F1AE3
:101F600025303B4663214FF4657002F0B7F94FF41A
:101F7000E571234802F07FFA40E063214FF44C7092
:101F800002F0ACF94FF4CC711D4802F074FA35E060
:101F9000632140F2D72002F0A1F940F26B111848FA
:101FA00002F069FA2AE0632140F2BA2002F096F9C1
:101FB00040F25D11124802F05EFA1FE0632140F228
:101FC000632002F08BF94FF4E5710D4802F055FAE9
:101FD00014E063214FF4087002F080F94FF4887127
:101FE000074802F048FA09E0632140F2E51002F0E8
:101FF00075F9F221024802F03EFA00BF00BF10BDA1
:10200000000400400146CAB20B1243EA02207047A6
:1020100008B50020009022E19748008800F00F00EA
:10202000964908700846007800287CD194480068DA
:10203000944908800846008800F0300092490880E2
:102040009048008800F440508E4908808C49096807
:102050004BF6BF7201EA020080F4005080F02000CD
:1020600040F4004141F08001854A116082480088B7
:1020700000F0100090BB1046006848F60F71084051
:102080001146086000F068FF7D4909684BF6BF7291
:1020900001EA02007B49098801F4805109B180F40A
:1020A00080507849098801F4005109B180F400504A
:1020B0007549098801F0100109B180F010007249DA
:1020C000098801F0200109B180F0200081B241F4BB
:1020D000004141F080016A4A116008BDFFE768488D
:1020E000006880B20090BDF8000000F40060B0B35A
:1020F00063480068C0F30E0048F68F7108406049DD
:10210000086001F02FFD5E4909684BF6BF7201EAD5
:1021100002005C49098801F4805109B180F48050C3
:102120005849098800E056E001F4005109B180F4F3
:1021300000505549098801F0100109B180F01000E4
:102140005149098801F0200109B180F0200081B2D5
:1021500041F4004141F08001494A1160BDE7FFE7C9
:10216000BDF8000000F40040002878D04448006822
:10217000C0F30E0048F68F7108404149086001F035
:1021800071F83F4909684BF6BF7201EA02003D4908
:10219000098801F4805109B180F4805039490988D7
:1021A00001F4005109B180F400503749098801F069
:1021B000100109B180F010003349098801F02001B5
:1021C00009B180F0200081B241F4004141F080016A
:1021D0002B4A116081E7294800782C4901EB8000E7
:1021E000D0F8000C80B20090BDF8000000F4004070
:1021F000C0B12248007801EB8000D0F8000CC0F399
:102200000E0048F68F7108401C4909781F4A02EBFE
:102210008101C1F8000C19490978491E1C4A52F87D
:1022200021008047BDF8000000F08000B8B11348DD
:102230000078164901EB8000D0F8000C48F60F71C9
:1022400008400E490978114A02EB8101C1F8000CDF
:102250000A490978491E0F4A52F821008047084868
:102260004430006880B20449088000F4004000282F
:102270007FF4D2AE00BF30E794000020540000206D
:10228000005C0040680000206A0000200050004010
:10229000BC000020A00000200B4A02EB8001D1F816
:1022A000001C01F4804171B102EB8001D1F8001CE7
:1022B00048F68F7211404CF280021143024B03EB3F
:1022C0008002C2F8001C7047005000400B4A02EB2D
:1022D0008001D1F8001C01F0400171B102EB8001D6
:1022E000D1F8001C48F68F72114048F2C002114329
:1022F000024B03EB8002C2F8001C70470050004004
:10230000084A02EB8001D1F8001C48F68F621140A8
:1023100048F280021143034B03EB8002C2F8001C19
:10232000704700000050004021B1026842F00102F5
:10233000026004E002684FF6FE731A4002607047C4
:1023400000B58BB00121084601F03CF8144800F0BC
:102350002DF81448009014480190002002900A9033
:1023600005200390002004908020059040000690F6
:1023700080000790202008900002099000200A9019
:102380006946074800F0C1F801220221044800F024
:10239000B3F801210248FFF7C7FF0BB000BD0000F2
:1023A000080002404C2401400A06002001684FF654
:1023B000FE72114001600021016041608160C160D6
:1023C0004B49884208D14A490839496841F00F0110
:1023D000474A083A51608AE045491431884208D199
:1023E00043490839496841F0F001414A083A5160CF
:1023F0007DE03F492831884208D13D490839496884
:1024000041F470613A4A083A516070E038493C3111
:10241000884208D136490839496841F47041344A44
:10242000083A516063E032495031884208D130495E
:102430000839496841F470212D4A083A516056E044
:102440002B496431884208D129490839496841F447
:102450007001274A083A516049E02549783188429D
:1024600008D123490839496841F07061204A083A87
:1024700051603CE01F49884206D1011F096841F0C4
:102480000F01021F116032E01A491431884208D14D
:102490001849091F096841F0F001164A121F11601E
:1024A00025E014492831884208D11249091F0968DA
:1024B00041F470610F4A121F116018E00D493C3160
:1024C000884208D10B49091F096841F47041094A43
:1024D000121F11600BE007495031884207D10549AE
:1024E000091F096841F47021024A121F11607047E8
:1024F00008000240080402401AB103680B4303605D
:1025000002E003688B430360704710B50022026845
:1025100047F6F0739A430C6A8B6823430C69234394
:102520004C6923438C692343CC6923434C6A23437E
:102530008C6A23431A430260CB6843600B68836054
:102540004B68C36010BD00002DE9F04728480068C3
:1025500000F110052E8826480068077AD6B9042FA6
:1025600018D12448007801280FD1002122480068A2
:1025700080B2801C214A42F8101030202049088087
:1025800000BF00201B49087003E0072710201C49EA
:10259000088027E0AC88A64201D8042000E0022091
:1025A0000746B44200D93446A0B2A968884780469D
:1025B000002000F065FC8146A2B24946404602F088
:1025C00067FBA1B2002001F0F5F92888001B2880E4
:1025D0006888204468803020094908800002094941
:1025E000088000BF024909680F72BDE8F08700004B
:1025F0005800002050000020505C00400060004067
:102600006A000020680000202DE9F0412848006899
:1026100000F110042688A068C0B1BEB1A588B542FB
:1026200000D93546A8B2A168884707462088401BD4
:102630002080608828446080002000F0FFFB8046F6
:10264000AAB24146384600F035FE00BF208850B19E
:102650004FF44050174908800021084601F0AAF9BC
:102660003020154908802088A188884204DB032097
:102670000F490968087218E02088002804DD052049
:102680000B490968087210E0208870B906200849D3
:102690000968087200210948006880B2801C084A55
:1026A00042F81010302004490880BDE8F081000095
:1026B00058000020680000206A000020505C0040A4
:1026C000006000402DE9F84F9B48006845780027DE
:1026D000BA46062D1BD198480068007800F07F00AC
:1026E000002813D1944909688878012803D19349B7
:1026F0000968CF690AE0022803D1904909680F6A86
:1027000004E0032802D18D4909684F6A94E0002D46
:1027100064D189480068408800285FD186480068F5
:10272000C08802285AD1844800680079002855D111
:1027300081480068007800F07F0028B97E48006872
:10274000808808B97E4F77E07B480068007800F009
:102750007F00012810D178490968487977490968CC
:102760008A6900219047002866D173480068807A02
:10277000002861D0724F5FE06F480068007800F079
:102780007F00022858D16C480068407900F00F069D
:1027900069480068407900F070096748006840792E
:1027A00000F0800038B1674901EB8600D0F8000CDA
:1027B00000F0300806E0634901EB8600D0F8000C19
:1027C00000F4405860480078B04235D9B9F1000FA4
:1027D00032D1B8F1000F2FD0594F2DE0082D07D17D
:1027E00055480068007800F07F0028BB574F23E071
:1027F0000A2D21D150480068007800F07F000128A0
:102800001AD14D480068807AB0B14B4800684088C2
:1028100090B949480068007970B947480068C08895
:10282000012809D1444909684879444909688A69F5
:102830000021904700B9464F57B13F480068A0F8C3
:1028400012A03D48006887610020B84700240FE0CF
:10285000394A12685078394A126811698847044623
:10286000032C05D10920344909680872BDE8F88FA6
:1028700031480068008A4FF6FF71884204D1092070
:102880002D4909680872F1E7022C03D02A48006834
:10289000008A20B90820284909680872E6E7264816
:1028A0000068007800F08000E0B323480068C0882A
:1028B000009021480068008A0099884204D91E4986
:1028C00000980968088223E01B480068008A1A49BA
:1028D0000968C98888421BDA17480068008A1749C6
:1028E000096891F82C10884203DA00201949087011
:1028F0000EE011480068008A1049096891F82C1010
:1029000090FBF1F201FB120010B90120114908708F
:102910000A48006890F82C10074800688182FFF789
:1029200013FE07E0FFE7032003490968087200036C
:102930000949088000BF99E7580000205C0000208A
:10294000053E000800500040E4000020893D0008DA
:10295000D93D000850000020680000207047002189
:1029600009E0002201E0531C9AB241F2B0239A42DE
:10297000F9DB4B1C99B28142F3DB704770B52248FA
:10298000B0F802042049B1F80014884200D170BDAB
:102990001D48B0F802041C49B1F80014884208DA56
:1029A0001948B0F800041849B1F80214401A84B26A
:1029B00005E01548B0F80204C0F5806084B2402CF0
:1029C00000DD40241048B0F80254B0F8020420445E
:1029D0000D49A1F802040846B0F80204B0F5806F72
:1029E00002DB0020A1F80204074948192246C02151
:1029F00002F04EF92146012000F0DCFF012001F039
:102A000007F800BFC3E700000007002010B5074922
:102A1000032002F09FF884B2E1B2054B054A034857
:102A200002F0B0F8032000F09BFF10BD221300203D
:102A30008F0000208C0000200149086070470000D2
:102A400014040140002123498279002A3AD00A4621
:102A5000126803689A430B461A600A1D12680368DD
:102A60009A430B1D1A60027911440A6803681A43DD
:102A70000A60184A0832126803689A43154B0833F3
:102A80001A601A1D126803689A43124B0C331A60BD
:102A90004279102A0ED11A1F126803681A430D4B8F
:102AA00008331A601A1D126803681A43094B0C3365
:102AB0001A600DE00749427911440A6803681A4315
:102AC0000A6005E0027911440A6803689A430A60C3
:102AD000704700000004014010B503A0FDF70EFC94
:102AE00003200849086010BD75736220656E746527
:102AF00072206C6F7720706F776572206D6F6465E0
:102B00000D0A00006C010020F3B581B00D460024D1
:102B10000026002000900427019800F075F8064672
:102B200000F0D4F800BF13E010494A1402FB04106F
:102B300000F020F80746012D09D1611C684600F01D
:102B400043FA684600F078FE09A000F075FE641CA8
:102B5000B44201D2042FE7D000F04CF8B44201D1C6
:102B6000042F01D00020FEBD0120FCE700800008FA
:102B70004000000030B5044604254FF4302000F03A
:102B8000B1F80546042D17D10C48006940F0020049
:102B90000A49086108464461006940F04000086144
:102BA0004FF4302000F09EF805460448006941F6D5
:102BB000FD71084001490861284630BD00200240EF
:102BC00004200B49C96801F0010109B101200EE0A0
:102BD0000749C96801F0040109B1022007E004496E
:102BE000C96801F0100109B1032000E0042070471A
:102BF000002002400348006940F08000014908615C
:102C0000704700000020024001B500200099C1F388
:102C100009021AB1012202EB912000E0880A08BDE6
:102C200070B504460D460426F00200F05BF8064637
:102C3000042E11D10948006940F0010007490861DC
:102C40002580F00200F04EF806460448006941F67F
:102C5000FE71084001490861304670BD0020024005
:102C600078B506460C46042500200090E80200F0E6
:102C700039F80546042D24D11348006940F00100BD
:102C8000114908613480E80200F02CF80546042D53
:102C900010D1B01C0090200C00990880E80200F0D0
:102CA00021F805460848006941F6FE7108400649CA
:102CB000086106E00448006941F6FE7108400249D7
:102CC0000861284678BD0000002002400248034900
:102CD0004860034848607047230167450020024070
:102CE000AB89EFCD00B502460423FFF769FF034629
:102CF00003E0FFF765FF0346521E012B01D1002AB6
:102D0000F7D102B90523184600BD2DE9F04102466E
:102D100000250026002000230024002791F803C08E
:102D20000CF00F0591F803C00CF0100CBCF1000F73
:102D300003D091F802C04CEA050591F800C0BCF13F
:102D4000000F31D0146800202BE04FF0010C0CFA7A
:102D500000F3B1F800C00CEA03069E4220D18300C4
:102D60004FF00F0C0CFA03F7BC4305FA03FC4CEAD6
:102D7000040491F803C0BCF1280F06D14FF0010CF8
:102D80000CFA00FCC2F814C00AE091F803C0BCF1D0
:102D9000480F05D14FF0010C0CFA00FCC2F810C02E
:102DA000401C0828D1D31460B1F800C0BCF1FF0F5B
:102DB00034DD546800202EE000F1080C4FF00108CB
:102DC00008FA0CF3B1F800C00CEA03069E4221D1C8
:102DD00083004FF00F0C0CFA03F7BC4305FA03FC19
:102DE0004CEA040491F803C0BCF1280F05D100F1AE
:102DF000080C08FA0CF8C2F8148091F803C0BCF172
:102E0000480F07D100F1080C4FF0010808FA0CF840
:102E1000C2F81080401C0828CED35460BDE8F08171
:102E20000246002093680B400BB1012000E0002017
:102E300070474161704701617047000001460548D5
:102E4000006880B200EBC100001D034A32F8100098
:102E500080B27047505C0040006000400146064868
:102E6000006880B200EBC100801D044A32F81000F7
:102E7000C0F3090070470000505C00400060004053
:102E800001460548006880B200EBC100034A32F8F1
:102E9000100080B270470000505C004000600040AD
:102EA00070B50A480468001D0568001D06683444B2
:102EB00054B108220649204600F0B2F80422044921
:102EC0001031284600F0ACF870BD0000E8F7FF1F95
:102ED0007200002000BFFEE710B5154800681549D4
:102EE0000840B0F1005F1CD1002001F0F5FD4FF467
:102EF0002F7002F0B5F900204FF0E021086172B6A2
:102F00000B4840680C490860084600680B49086097
:102F100007490868FDF7B7F90848006880470020AE
:102F200010BD07A002F0FCFB4FF0FF30F8E70000F7
:102F3000008000080000FE2F8C0100208801002086
:102F40000D0A2052756E20746F20617070206572BA
:102F5000726F722E0D0A000010B518480068047ACE
:102F6000022C01D0042C05D1FFF7EEFA13480068BB
:102F7000047A1CE0062C19D1104800684078052816
:102F80000ED10E480068007800F07F0040B90B4970
:102F90000968C87800F064FC09490968086A804734
:102FA0000849096888688047082400E00824034924
:102FB00009680C7200F094F910BD00005800002060
:102FC000640000205C000020F0B5144A00250024B5
:102FD000002320E0B1FBF2F6303606F0FF0C2E465F
:102FE0006D1C00F806C0B1FBF2F602FB16110A26B2
:102FF000B2FBF6F26E1E865D302E01D1012600E096
:1030000000260CB9012700E000273E400EB1002544
:1030100000E0641C5B1C0A2BDCD3F0BD00CA9A3BA9
:1030200030B50B46002100BF16E00A24B4EB107F38
:1030300005D9302404EB107403F8114005E0412455
:1030400004EB10740A3C03F81140000100254C0009
:10305000641C1D554C1CE1B29142E6DB30BD000002
:1030600010B5074C07A0FDF749F9A07A18B1052063
:103070000A49086002E001200849086010BD00000C
:10308000E40600206C65617665206C6F7720706FB8
:10309000776572206D6F64650D0A00006C01002079
:1030A00000BFFEE77047704770B5002100230F2274
:1030B000C47804B3154C246804F4E064C4F5E064F7
:1030C000210AC1F10403CA40447804FA03F1847868
:1030D0001440214309010E4C0678A155047804F0F0
:1030E0001F050124AC4005786D11AD0005F1E02508
:1030F000C5F8004109E0047804F01F050124AC4044
:10310000044D0678761145F8264070BD0CED00E0C0
:1031100000E400E080E100E002490143024A11605E
:10312000704700000000FA050CED00E070B50226C3
:1031300047480068447846480068007800F07F00FF
:10314000002844D1092C03D100F0DCFE06465FE0E4
:10315000052C14D13E480068C0787F280BDC3C4821
:103160000068807838B93A480068808818B93848CB
:103170000068807A08B1082565E0002648E0032C45
:103180000ED133480068C078012807D13048006864
:10319000808818B900F0DAFE064639E0022637E0EA
:1031A000012C35D12A480068C07801280DD1284863
:1031B0000068808848B926480068407A00F02000FE
:1031C00018B100F02BFD064622E0022620E0204840
:1031D0000068007800F07F00012805D10B2C17D182
:1031E00000F030FF064613E019480068007800F050
:1031F0007F0002280BD1012C03D100F00FFD064601
:1032000006E0032C04D100F0B5FE064600E00226DD
:103210004EB1E0B20F4A1268516988470646032E44
:1032200001D109250FE00EB108250CE0062500218B
:103230000948006880B2801C084A42F8101030200B
:103240000749088000BF024909680D7270BD00007F
:10325000580000205C000020505C004000600040EE
:103260006A00002010B511480068047A022C01D0D1
:10327000042C01D1082412E0032C01D0052C05D127
:10328000FFF7C2F909480068047A08E0072C05D165
:1032900007490968C8688047082400E008240349F2
:1032A00009680C7200F01CF810BD000058000020E6
:1032B0005C000020F0B5561C7510074E06EB41046B
:1032C0002B4605E034F8047B20F8017B401C5B1E94
:1032D000002BF7D1F0BD00000060004070470000F7
:1032E00010B50D4890F82C10002000F0F3FA0B48B0
:1032F0000068007A082805D140020949088010209A
:103300000849088005480068007A092801D1012091
:1033100010BD0020FCE70000E8000020580000205D
:10332000680000206A00002008B50121102000F08C
:1033300069F84FF40040ADF8000003208DF802005A
:1033400010208DF8030069460748FFF7DEFC4FF4B4
:103350008040ADF8000048208DF80300694602481F
:10336000FFF7D3FC08BD00000010014010B501209C
:1033700001F05AFA01240B48046000200A49088031
:1033800008460088074908600020091D08604FF4BE
:10339000E05005490880084600880249086000207E
:1033A00010BD0000405C004062000020014600208B
:1033B000034A506820F440400843506070470000C2
:1033C0000010024029B1064A52690243044B5A6177
:1033D00004E0034A52698243014B5A61704700007E
:1033E0000010024029B1064AD2690243044BDA6157
:1033F00004E0034AD2698243014BDA61704700005E
:103400000010024029B1064A92690243044B9A61B6
:1034100004E0034A92698243014B9A6170470000BD
:103420000010024030B500210022002400232D4D61
:103430006D6805F00C0121B1042905D0082923D1BC
:1034400005E0294D056022E0274D05601FE0254D70
:103450006D6805F47012234D6D6805F48034022503
:1034600005EB92421CB9214D554305600BE01D4D03
:103470006D6805F400351DB11C4D5543056002E033
:10348000194D5543056002E0174D056000BF00BFB0
:10349000144D6D6805F0F0010909154D6B5C056868
:1034A000DD4045600F4D6D6805F4E061090A104D7F
:1034B0006B5C4568DD4085600A4D6D6805F46051C0
:1034C000C90A0B4D6B5C4568DD40C560054D6D68F4
:1034D00005F44041890B074D6B5CC568B5FBF3F5FE
:1034E000056130BD0010024000127A0000093D0065
:1034F0002D0000203D0000200149086070470000B9
:10350000D800424270B505460C46164601F0DCFE76
:10351000002842D1206022480078182817D006DC05
:10352000012809D002280AD004281FD10BE0412825
:1035300019D061281AD117E08020206019E04FF4DB
:103540008060206015E000202060022070BD1448DB
:103550000078182804D14FF0FF3020600020F5E7F4
:103560004FF0FF30F2E700BF0120EFE74FF0FF30F0
:10357000ECE700BF2068421D09492846FCF7E9FF37
:103580006978A87880F0FF00814202D04FF0FF30C8
:10359000DCE700F007F80020D8E74FF0FF30D5E770
:1035A000090F0020FF200149087070478F0000209C
:1035B00070B50546072D01D02E4805702D480078BE
:1035C00008284ED2DFE800F004111A202B384E4FA5
:1035D0002948006828B900F053F8062025490870EA
:1035E00002E005202349087041E000F049F804207A
:1035F0002049087001202049086038E002201D4958
:1036000048700320087032E01A484078401E19497B
:1036100048700846407808B90420087027E0174829
:10362000006884B244F01004144804600520114975
:1036300008700A2048701AE00E484078401E0D4974
:1036400048700846407858B90C48006884B224F0A5
:1036500010040A480460062008700020064908602B
:1036600005E000BF00BF06200249087000BF00BF90
:1036700070BD00007101002074010020405C00401A
:1036800010B50748006884B224F0040404480460BC
:10369000FFF7E6FC4FF43F400149086010BD000011
:1036A000405C004010B50948006805280CD1084866
:1036B00001680068401C064A1060052904D10020FA
:1036C00011460860FFF75AF910BD00006C01002098
:1036D0009000002030B503460C461546002207E056
:1036E000184600F008F824F812009B1C501C82B207
:1036F000AA42F5DB30BD0146088870472DE9F05F2E
:1037000080468A461746B8F1006F02D3B8F1805F51
:1037100001D3BDE8F09FFFF7D9FAA8F1006B4FEA9B
:103720009B25CBF34809C9F50074A74200DC3C4651
:103730004DE04FF0006101EB85208A142749FFF727
:10374000C9FF00260BE009EB0600244931F8100000
:103750004FF6FF71884200D003E0701C86B2A6428B
:10376000F1DB00BFA6421BDA4FF0006101EB8520C0
:10377000FFF700FA002608E03AF8160006EB090108
:10378000164A22F81100701C86B2A642F4DB4FF0F4
:10379000006101EB85208A14104900F021F804E053
:1037A00022465146404600F01BF8A74200D10FE0E8
:1037B0006D1C4FF000090AEB440AA044381B87B285
:1037C000B7F5007F02DD4FF4007400E03C46B0E73F
:1037D00000BFFFF70FFA00BF9BE700008413002033
:1037E0002DE9F04105460E461746002407E036F85D
:1037F00014102846FFF714FAAD1C601C84B2BC42BA
:10380000F5DBBDE8F081704710B50446204601F0B5
:1038100025FA002010BD000010B5044621460548D9
:1038200000F0F7FF00BF8021024800F025FF0028CC
:10383000F9D010BD0038014010B5044603E02078EF
:10384000FFF7EAFF641C20780028F8D110BD0000C3
:103850004FF6F8710140014A11607047505C00401A
:1038600030B501460F4B1A78002014E003060E4CC9
:1038700004EB9353D3F8003C48F68F74234048F28E
:1038800080042343C4B223430406074D05EB94543C
:10389000C4F8003C401C9042E8D341F08003034C44
:1038A000236030BDE4000020005000404C5C00402C
:1038B00010B54A105300054A126892B202EBC002DA
:1038C000121D034C44F8123010BD0000505C004043
:1038D0000060004010B502460F48006880B200EB5F
:1038E000C200801D0D4C04EB40033E290BDD481146
:1038F00001F01F040CB9441EA0B24FF4004444EA86
:1039000080241C6007E0481001F001040CB1441C45
:10391000A0B284021C6010BD505C004000600040FA
:1039200030B50E4C04EB8003D3F8003C4BF68F749B
:1039300003EA040201F480530BB182F4805201F4D3
:1039400000530BB182F4005242F4004343F0800371
:10395000024D05EB8004C4F8003C30BD005000402F
:1039600010B50B4B03EB8002D2F8002C4BF68F7393
:1039700002EA030181F4805181F4005141F40042D4
:1039800042F08002024C04EB8003C3F8002C10BD0F
:103990000050004010B54A105200044B1B689BB207
:1039A00003EBC003024C44F8132010BD505C0040F0
:1039B00000600040044A126892B202EBC002921CFE
:1039C000024B43F812107047505C0040006000400A
:1039D00030B50E4C04EB8003D3F8003C48F6BF74BE
:1039E00003EA040201F010030BB182F0100201F0AF
:1039F00020030BB182F0200242F4004343F0800325
:103A0000024D05EB8004C4F8003C30BD005000407E
:103A100010B50B4B03EB8002D2F8002C48F6BF73B5
:103A200002EA030181F0100181F0200141F400421B
:103A300042F08002024C04EB8003C3F8002C10BD5E
:103A40000050004010B5074B03EB8002D2F8002C69
:103A500048F68F131A400A43024C04EB8003C3F864
:103A6000002C10BD0050004010B500F001F810BD52
:103A70000CB50020019000903348006840F480307D
:103A80003149086000BF3048006800F40030009001
:103A90000198401C0190009818B90198B0F5A06FEA
:103AA000F1D12948006800F4003010B101200090E5
:103AB00001E0002000900098012843D123480068CD
:103AC00040F01000214908600846006820F003001B
:103AD00008600846006840F0020008601A48406824
:103AE000194948600846406848600846406840F404
:103AF000806048600846406820F47C1048600846B2
:103B0000406840F4E81048600846006840F0807063
:103B1000086000BF0C48006800F000700028F9D071
:103B20000948406820F0030007494860084640689B
:103B300040F00200486000BF0348406800F00C00FD
:103B40000828F9D10CBD00000010024000200240FE
:103B500010B50020FFF7D0FC0121C805FFF742FC9B
:103B600010BD000038B501242948006880B2001D4E
:103B7000284931F8100080B201EB4000009026483F
:103B80000068007A092832D0009800782249096834
:103B900008700098401C0090009800781E49096841
:103BA00048700098401C0090009800EB4400009082
:103BB000009931F8020B0091FEF724FA16490968C2
:103BC0004880009800EB44000090009931F8020B07
:103BD0000091FEF717FA104909688880009800EBF9
:103BE00044000090009800880B490968C8800120B3
:103BF00009490968087208480068C08810B9FFF7C9
:103C000095FA01E0FEF75EFDFFF76AFB38BD0000A4
:103C1000505C004000600040580000202DE9F04753
:103C200054480068007800F07F08B8F1000F0AD10E
:103C300050480068407A00F0DF004E490968487239
:103C40000020BDE8F087B8F1020F7CD14948006838
:103C5000408818B947480068007908B10220F0E7A9
:103C6000DFF8149143480068477927F080052C4617
:103C700040480068407900F0800038B13F4901EBCE
:103C80008400D0F8000C00F0300606E03B4901EB60
:103C90008400D0F8000C00F4405699F80000A842C7
:103CA00004D91EB133480068807A08B90220C8E7F9
:103CB00007F0800080B1314901EB8400D0F8000C9E
:103CC00000F0300010284BD1E0B2FEF7FFFAE0B26E
:103CD0003021FFF77DFE43E0284901EB8400D0F856
:103CE000000C00F44050B0F5805F39D1E4B9244AAB
:103CF00092F82C10E0B2FFF7EDFD204A02EB8401B0
:103D0000D1F8001C4BF68F7201EA020080F480505B
:103D100080F4005040F4004141F08001174B03EB68
:103D20008402C2F8001C1BE0E0B2FEF7B5FA134AA9
:103D300002EB8401D1F8001C4BF68F7201EA0200FD
:103D400080F4805000E011E080F4005040F4004125
:103D500041F08001094B03EB8402C2F8001C00BF54
:103D6000084909684869804700206AE700BF0220C7
:103D700067E7000058000020E400002000500040E9
:103D8000E80000206400002010B504462CB9012092
:103D9000064909680882002010BD054909680868BD
:103DA0008047024800680A30F6E70000580000200B
:103DB0006400002010B5024606480068438A32B904
:103DC0008888C01A034C24682082002010BD08682F
:103DD0001844FBE75800002010B504462CB9012018
:103DE000064909680882002010BD054909688868ED
:103DF0008047024800680C30F6E7000058000020B9
:103E00006400002010B504462CB902203949096825
:103E10000882002010BD002037490880354800681E
:103E2000007800F07F0018BB32490968487A00F03A
:103E3000200131B13049097841F002012E4A117058
:103E400005E02D49097801F0FD012B4A117000F0C1
:103E5000400131B12849097841F00101264A117029
:103E600005E02549097801F0FE01234A11703AE086
:103E700020480068007800F07F00012801D11E482A
:103E8000C8E71C480068007800F07F00022828D1AD
:103E9000184A1268517901F00F0001F080027AB1DE
:103EA000164B03EB8002D2F8002C02F03002102AED
:103EB00016D1114A127842F001020F4B1A700FE02E
:103EC0000E4B03EB8002D2F8002C02F44052B2F504
:103ED000805F05D1084A127842F00102064B1A7041
:103EE00001E0002096E70649096808698047024812
:103EF00090E70000580000204E00002000500040D5
:103F00006400002010B50E480068C0780D4949785B
:103F1000884213DC0A480068807878B9084800684D
:103F2000808858B906480068C078054909688872D1
:103F30000549096848688047002010BD0220FCE759
:103F400058000020E40000206400002010B507485D
:103F50000068407A40F0200004490968487204492A
:103F60000968C8698047002010BD00005800002083
:103F7000640000202DE9F0412E480068467926F0C3
:103F800080073C462B480068407900F0800038B13B
:103F9000294901EB8400D0F8000C00F0300506E060
:103FA000254901EB8400D0F8000C00F4405523486B
:103FB0000078A04208D91F480068408820B91DB188
:103FC0001C480068807A10B90220BDE8F08106F034
:103FD0008000A0B1184A02EB8401D1F8001C48F619
:103FE000BF7201EA020080F0100040F4004141F08D
:103FF0008001114B03EB8402C2F8001C14E00E4A4E
:1040000002EB8401D1F8001C4BF68F7201EA02002A
:1040100080F4805040F4004141F08001064B03EBF6
:104020008402C2F8001C00BF0549096888698047FE
:104030000020CAE75800002000500040E4000020A3
:104040006400002010B5174B1B68D978154B1B680E
:104050005879154B1B689A699047044611480068C7
:10406000807AE8B13CB90F480068007918B90D486A
:104070000068807808B1022010BD8CB90B4909682E
:10408000C868804707480068407906490968C872CF
:1040900004480068C0780349096808730020EBE70A
:1040A0000220E9E7580000205C00002064000020A6
:1040B00070B502460C4600210025002310783028F8
:1040C00043D15078782802D0507858283DD1907844
:1040D00008B9002070BD022130E0505C10B92360A7
:1040E00001252DE0505C412802DB505C46280BDDA9
:1040F000505C612802DB505C662805DD505C30288E
:1041000019DB505C392816DC505C302805DB505C2C
:10411000392802DC505C30380AE0505C412805DB6D
:10412000505C462802DC505C373801E0505C573860
:1041300000EB031301E0002502E0491C0B29CCD35E
:1041400000BF0B2934D3002532E000212AE0505C67
:1041500010B92360012527E0505C6B2802D0505C29
:104160004B2804D119B19B02236001251CE0505C4F
:104170006D2802D0505C4D2804D119B11B05236075
:10418000012511E0505C302809DB505C392806DC41
:10419000505C303803EB830600EB460301E000255A
:1041A00002E0491C0B29D2D300BF0B2900D3002504
:1041B00028468FE738B50025002000902148006888
:1041C00084B200BF09E0204901EB8500D0F8000C63
:1041D00080B21E4941F825006D1C082DF3D344F42C
:1041E00080641848046044F00104046024F0010471
:1041F000046000BF1348001D006800F480600028C0
:10420000F8D04FF6FF300F49091D0860002509E07E
:104210000E4850F8250080B20B4A02EB8501C1F828
:10422000000C6D1C082DF3D344F00804054804600D
:10423000006884B244F0040402480460FEF74CFCB9
:1042400038BD0000405C0040005000406413002076
:10425000042808D14FF0E021096941F004014FF032
:10426000E022116107E04FF0E021096921F004012B
:104270004FF0E022116170477047000010B51348FD
:10428000006840F001001149086008464068104984
:1042900008400E494860084600680E4908400B492E
:1042A00008600846006820F48020086008464068DE
:1042B00020F4FE0048604FF41F008860FFF7D4FB35
:1042C0004FF000600449086010BD0000001002407B
:1042D0000000FFF8FFFFF6FE08ED00E030B589B002
:1042E00004460D4601210220FFF77CF8012104203D
:1042F000FFF788F84020ADF8200018208DF8230043
:1043000003208DF8220008A91A48FEF7FEFCADF83C
:104310001840ADF814500020ADF81A00ADF81600A2
:1043200005A9154800F0ACF86020ADF804000120A4
:10433000ADF80600204604EBD071C1F34F01ADF893
:104340000A100220ADF80C0001A90B4800F03EF85D
:104350000121094800F02AF80821074800F082F8F6
:104360000121054800F00AF80121034800F012F885
:1043700009B030BD000801400004004021B10288AE
:1043800042F08002028004E002884FF67F731A40F8
:104390000280704721B1028842F00102028004E0ED
:1043A00002884FF6FE731A400280704731B1B0F8B0
:1043B000442042F40042A0F8442005E0B0F8442034
:1043C000C2F30E02A0F844207047000070B500242C
:1043D00000220023058C4FF6FE7635400584028CC2
:1043E0008388048B4FF68F752C40B51E2C400D88AA
:1043F0002C43751E2A400D892A434D882A43144DAB
:10440000A8420BD0134DA84208D0134DA84205D0A6
:10441000124DA84202D0124DA84213D14FF6F775A3
:104420002A404D892A434FF6FB752A408D882A433E
:104430004FF6FF652B404FF6FF552B408D892B43E0
:10444000CD892B4383800483CD888586028470BD0B
:10445000002C014000340140004001400044014074
:10446000004801400A460021018B4FF6F7731940BE
:104470001143018370478186704781877047000030
:10448000002202881D4B98420ED01D4B98420BD043
:10449000B0F1804F08D01B4B984205D01A4B984280
:1044A00002D01A4B984204D14FF68F731A404B88B2
:1044B0001A43174B984207D0164B984204D04FF638
:1044C000FF431A40CB881A4302808B8883850B8870
:1044D00003850A4B98420BD0094B984208D00E4BEB
:1044E000984205D00D4B984202D00D4B984201D115
:1044F0000B7A03860123838270470000002C014061
:10450000003401400004004000080040000C00405E
:1045100000100040001400400040014000440140F1
:104520000048014010B540F225511D4800F0B1F897
:1045300010B31B4800F068F9C4B21A48008800F4B0
:104540000040C8B91748008800F4804060B10A2CC8
:1045500003D000201349088020E01248008840F46E
:1045600000401049088019E00D2C06D10D48008844
:1045700040F480400B49088010E00A480088C0F3EE
:104580000D0009490C5407480088401C0549088063
:1045900008460088C72801DD0020088010BD000003
:1045A000003801404C0000201C06002021B1828907
:1045B00042F40052828104E082894DF6FF731A4072
:1045C0008281704710B500200E49A1F80204A1F8BD
:1045D00000040D4908800D4801790DA0FBF78EFEFF
:1045E0000A48417910A0FBF789FE0848817915A097
:1045F000FBF784FE0548016819A0FBF77FFE012048
:1046000010BD0000000700206C000020DC0000202E
:104610006C696E65636F64696E672E666F726D613B
:10462000743A25640D0A00006C696E65636F6469F5
:104630006E672E706172697479747970653A256459
:104640000D0A00006C696E65636F64696E672E64A5
:10465000617461747970653A25640D0A0000000088
:104660006C696E65636F64696E672E6269747261EE
:1046700074653A25640D0A0002460020B1F5007FFA
:1046800000D100BF13880B400BB1012000E00020D7
:10469000704770B50246002400230025002040F634
:1046A0006A16B14200D100BFC1F3421501F01F03E9
:1046B000012606FA03F3012D02D19689334006E064
:1046C000022D02D1168A334001E0968A33400C1243
:1046D000012606FA04F41688344013B10CB1012007
:1046E00000E0002070BDF0B5034600240026002540
:1046F000002040F66A17B94200D100BF1846C1F346
:10470000421401F01F06012707FA06F5012C01D11A
:104710000C3004E0022C01D1103000E014301AB14A
:1047200007682F43076002E00768AF430760F0BDEA
:104730002DE9F04786B005460E460024A24600BF8C
:10474000A1460027B08900B100BF2F462C8A4CF645
:10475000FF700440F08804432C82AC894EF6F310BD
:104760000440B08831890843718908430443AC810F
:10477000AC8A4FF6FF400440B0890443AC8201A8E4
:10478000FEF750FE1F48874202D1DDF810A001E07D
:10479000DDF80CA0A88900F4004040B10AEBCA0083
:1047A00000EB0A1031684900B0FBF1F807E00AEBB2
:1047B000CA0000EB0A1031688900B0FBF1F86420F0
:1047C000B8FBF0F004012009642101FB1089A889DD
:1047D00000F4004040B1322000EBC900B0FBF1F022
:1047E00000F00700044308E0322000EB09106421C8
:1047F000B0FBF1F000F00F0004432C8106B0BDE8DF
:10480000F08700000038014001468888C0F30800A6
:104810007047C1F308028280704710B54FF48020C2
:10482000FEF70AF910BD000010B504461CB104A043
:10483000FBF764FD02E008A0FBF760FD10BD00007F
:104840007573622070756C6C20757020656E616286
:104850006C650D0A000000007573622070756C6C49
:104860002075702064697361626C650D0A00000038
:1048700010B508480849086002200968087207480E
:104880000749086007480849086005490968086839
:10489000804710BDE406002058000020E8000020FA
:1048A0005C00002018010020640000200EB54FF4C9
:1048B0008020FEF7C1F84FF48020009008208DF88A
:1048C000050001208DF806006846FEF7BBF81420AD
:1048D0008DF8080001208DF8090000208DF80A00ED
:1048E00001208DF80B0002A8FEF7DEFB2A208DF8D0
:1048F000080000208DF8090002A8FEF7D5FB0EBDC8
:1049000010B588B0002469480068694908800846E5
:10491000008800F4007067490988084050B14FF6DC
:10492000FF506249086064480078401C6249087082
:10493000FEF7B8FE5E48008800F400405D49098833
:10494000084008B1FDF764FB5948008800F4806016
:1049500058490988084030B14FF6FF305349086084
:104960005649486880475248008800F40050514931
:104970000988084018B14DF6FF704C4908604C4852
:10498000008800F480504B490988084030B14EF649
:10499000FF70464908600020FEF70AFE4448008880
:1049A00000F4006043490988084060B14448007839
:1049B00010B1FFF7FFFB02E00220FEF7F9FD4FF216
:1049C000FF703A4908603A48008800F4807039491D
:1049D00009880840002866D04FF6FF603349086018
:1049E000081D006800F40040002856D035480068D3
:1049F000401C3449086008460068032850D92B48F9
:104A0000001F006800F00800002849D12748001F57
:104A1000006880B22C490860002408E02B4901EBB3
:104A20008400D0F8000C80B24DF82400641C082CDF
:104A3000F4D32548006840F0010023490860084687
:104A4000006880B21949091F08601F48006820F0FB
:104A500001001D4908600846006880B21349091F1B
:104A6000086000BF1148006800F480600028F9D099
:104A70004FF6FF300D490860002408E05DF824007F
:104A800080B2124A02EB8401C1F8000C641C082CAD
:104A9000F4D300200B49086002E0002009490860B7
:104AA0000720FEF785FD08B010BD0000445C004003
:104AB000940000206200002096000020E800002002
:104AC00070010020980000209C0000200050004051
:104AD00010B5FFF715FF10BD10B5044601210420E5
:104AE000FEF790FC3CB11048006880B220F0020054
:104AF0000D49086016E00C48006880B240F00200E2
:104B0000094908600948006820F47F2007490860C7
:104B10000846006840F44C30086089140348001FC0
:104B2000FEF787F910BD0000405C0040040801401A
:104B30000020064908604FF43F40054908800846B8
:104B400000880249091F086000207047445C00404B
:104B5000620000202DE9F04104460E46002504F0D5
:104B60007F00FEF77BF9054604F07F00FEF766F94B
:104B700007462A4639463046FEF79CFB2846BDE8E4
:104B8000F0810000F0B505460E4600245BE0295D8B
:104B900001290DD12E48008800F4004040B985203D
:104BA0002C4F38802A48008840F40040284F388035
:104BB00002290ED12648008800F4004048B940F28E
:104BC0000540244F38802248008840F40040204FA0
:104BD000388004290DD11E48008800F4004040B9F7
:104BE00001201C4F38801A48008840F40040184FBC
:104BF00038801748008800F4004010B3144800883B
:104C0000C0F30D00144F395411480088401C104F58
:104C1000388038460088C0F30D000E4F3F88B842F8
:104C20000BD10B480088C0F30D0010800020084F06
:104C30003880084F3880187003E000201080FF2073
:104C40001870601CC4B2B442A1DB0020F0BD0000AB
:104C50006C0000206E000020090F00200A49B1F806
:104C60000014094A50541146B1F80014491CA2F826
:104C700000141146B1F80014B1F5806F02D1002183
:104C8000A2F80014704700000007002000BFFEE7F4
:104C9000F0B5144604F1010C4FEA6C07DFF824C0AC
:104CA0000CEB41033D460AE00678401C90F800C03A
:104CB00046EA0C2223F8022B9B1C401C6D1E002D83
:104CC000F2D1F0BD0060004070B504460025212CF3
:104CD00008D112480068007800F07F0021280ED12A
:104CE0000F4D0CE0202C0AD10C480068007800F031
:104CF0007F00212800D10B4D20200B4908700DB9F1
:104D0000022070BD054800688561002103480068E5
:104D100041820020A8470020F3E70000580000204F
:104D2000554D0008E54E0008D800002010B5044697
:104D300002492046FFF73EF810BD00004401002064
:104D400010B5044602492046FFF734F810BD0000B4
:104D50003C010020014629B90820034A126810824C
:104D6000002070470148FCE758000020DC000020CC
:104D700070B5054606480068C478042C01DD0020A3
:104D800070BD044800EBC4012846FFF713F8F7E7AD
:104D9000580000204C0100200246002901DD0220BD
:104DA0007047012A01DD0220FAE70020F8E7000041
:104DB000014608480068007800F07F00212807D1EC
:104DC000022901D100207047222901D10020FAE7F1
:104DD0000220F8E75800002010B500203449096887
:104DE00088723448C07932490968487200203049D5
:104DF0000968C872FEF72CFD4FF400710020FEF721
:104E000021FE10210020FEF7E3FD40210020FEF7E7
:104E10004FFD80210020FEF7BDFD0020FDF770FA58
:104E2000254890F82C100020FEF754FD0020FEF7D6
:104E300097FD00210120FEF705FEC0210120FEF7AD
:104E4000A9FD20210120FEF7C3FD00210120FEF76E
:104E500067FD4FF4C0610220FEF7F4FD4FF480714E
:104E60000220FEF797FD00210220FEF759FD2021C8
:104E70000220FEF7ADFD00210320FEF7E3FD4FF415
:104E800088710320FEF714FD40210320FEF722FD68
:104E90004FF440510320FEF743FD00210320FEF7AD
:104EA00097FD0020FEF7DCFC01200449086010BDDE
:104EB00058000020CE570008E80000206C010020B8
:104EC0000348817A11B10521024A11607047000040
:104ED000E40600206C0100200420014908607047AE
:104EE0006C010020014629B90820034A126810828B
:104EF000002070470148FCE758000020DC0000203B
:104F000010B505480078202804D1FFF75BFB00208E
:104F10000149087010BD0000D80000207047000053
:104F200010B5FDF7BDFF0020054909688872FEF73E
:104F30001DFAFFF7FDFD00200249086010BD0000CA
:104F4000580000206C0100202DE9F04FADF22C4DEF
:104F50000646002001909D489D4908604FF480411D
:104F60009C48FDF75DFF38B9022000F079F94FF455
:104F700000419848FDF75DFF4320FEF745FC4FF0E8
:104F8000000BD8460020029000BF642000F068F9B2
:104F9000002700200390B14600BF642000F060F9B4
:104FA0004FF4801204A909A8FEF7ACFA20B1012839
:104FB00073D0022872D1C8E04FF000080498B0F115
:104FC000FF3F01D070B907E00620FEF71DFC00206E
:104FD0000DF22C4DBDE8F08F0620FEF715FC0120E8
:104FE0000390A7E09DF82500F9B2884203D0152070
:104FF000FEF70AFC9DE0002F58D19DF827000028FD
:105000004DD000250DF1270405E014F8012B2846AA
:105010006D1C71490A54207808B1FF2DF5DD00227E
:1050200028466D1C6C490A540025641C05E014F8E0
:10503000012B28466D1C05A90A542078202801D090
:10504000102DF4DB002228466D1C05A90A5401A985
:1050500005A8FFF72DF80198B0F5003F08DB1820F0
:10506000FEF7D2FB1820FEF7CFFB4FF0FF30AFE783
:1050700000210198FDF748FD40B91820FEF7C4FB58
:105080001820FEF7C1FB4FF0FF30A1E70620FEF726
:10509000BBFB4320FEF7B8FB48E04DE05CE0062098
:1050A000FEF7B2FB01200390834643E00DF1270198
:1050B0004846049AFBF74DFA484806604FF0000A4C
:1050C00027E0FDF703FE4548006801684048006896
:1050D000FDF7C6FDFDF78EFD3D48006800683F49BD
:1050E00009680968884208D01820FEF78DFB18204F
:1050F000FEF78AFB6FF001006AE735480068001D83
:105100003349086035480068001D344908600AF1D9
:10511000040A0498824506DA2C49019808442C496F
:1051200009688842CDD80620FEF76EFB7F1C01205F
:10513000029000BF00BF31E01820FEF765FB182089
:10514000FEF762FB6FF0020042E71520FEF75CFB02
:1051500001200390834621E00298002801DD08F138
:105160000108B8F1050F07DD1820FEF74DFB1820E8
:10517000FEF74AFB00202BE74320FEF745FB4FF4E8
:1051800080411448FDF74CFE38B9022000F068F861
:105190004FF400410F48FDF74CFE00BF00BF0398DD
:1051A00000283FF4FAAE00BF00BFBBF1000F3FF490
:1051B000ECAE0620FEF728FB4320FEF725FB062079
:1051C000FEF722FB00BF00BF019801E70080000846
:1051D0007801002000100140841700208001002089
:1051E000490050EAC12018BF04204A0D18BF40F002
:1051F000010040F2FF72B2EB515F08BF40F00200C5
:10520000012808BF0520704730380A2801D2012044
:1052100070470020704700BF7047000010B56FF066
:105220000400FFF715F80A4800680A49B0FBF1F0DE
:10523000094908700846007800EB4001C1EBC01036
:105240004FF6FF7101EAC0000449088010BD00005C
:105250000000002000127A004200002044000020DC
:105260000146114A12884A434FF0E0235A61002256
:105270009A611A46126942F001021A6100BF4FF0AA
:10528000E022106900F001021AB100F48032002A15
:10529000F5D04FF0E022126922F001024FF0E02336
:1052A0001A6100229A6170474400002000BF054A3D
:1052B000128802F04002002AF9D0C2B2014B1B1D35
:1052C0001A8070470038014001480078704700009C
:1052D0008F00002010B586B00024074801680191B6
:1052E0008088ADF8080005A101A8FBF777F900B99F
:1052F0000124204606B010BD2213002075706461A1
:105300007465000008B501210820FEF77BF8022033
:10531000ADF8000003208DF8020048208DF803004E
:1053200069460248FDF7F1FC08BD0000000C014091
:1053300008B50024FFF772FF00F064F9FFF7E2FF01
:10534000FDF7F2FF00200090012269467A48FEF73F
:10535000C1F9BDF800004AF25A5188423CD00846D3
:105360007649088001227448FEF7C8F9744800782D
:105370007249088001227048801CFEF7BFF971480D
:1053800000786E49088001226B48001DFEF7B6F9CF
:105390006D4800786949088001226748801DFEF742
:1053A000ADF96A48008865490880012262480830E2
:1053B000FEF7A4F9664800886049088001225E482B
:1053C0001030FEF79BF9634800885C490880012291
:1053D00059481230FEF792F902215F48FDF720FD8F
:1053E00020BB4FF480415D48FDF71AFDF0B9012064
:1053F0005B490870C1035948FDF71DFD00F0BEF878
:105400000120FCF7A5FD4FF49670FDF7A8FA0220E5
:10541000FCF79EFD4FF49670FDF7A1FA0320FCF710
:1054200097FD4FF49670FDF79AFA01E0FDF754FDF1
:105430004FF4A060FDF770FEFFF7F0FE4FF4E1308F
:1054400000F01EF9FCF746FC4FF4E160FFF708FF9F
:105450000020FFF741FB4FF42F70FFF701FF012001
:10546000FFF73AFBFEF774FBFFF720FAFFF700FAAD
:1054700061E04FF480413948FDF7D2FCE0B90220E9
:10548000FFF7EEFE0320FCF763FD4FF49670FDF787
:1054900066FA0220FCF75CFD4FF49670FDF75FFAA8
:1054A0000120FCF755FD4FF49670FDF758FA4FF4C4
:1054B00000412A48FDF7BDFC2A48006884420FD00D
:1054C00028480068C4B2052C05D14FF48051224809
:1054D000FDF7AFFC04E04FF480511F48FDF7ABFC33
:1054E000214801882148FCF76AFC214908801E48B0
:1054F00041881E481430FCF762FC1D4948801A4858
:1055000081881A482830FCF75AFC194988801648C7
:10551000C18816483C30FCF752FC1549C880FFF79B
:10552000D9FE012805D11348FFF70EFD1249086086
:1055300000E000BF00BF9CE7007A000822000020C6
:105540001400002015000020160000201800002084
:105550001A0000201C000020000C01400010014037
:105560002C0000206C0100200A0600209C05002071
:10557000000600209C0100202800002010B5002417
:1055800002E000F055F8641C082CFADB002402E06D
:1055900000F04EF8641C082CFADB002402E000F056
:1055A00005F8641C082CFADB10BD000010B54FF4A0
:1055B00000611348FDF73FFC00BF00BF00BF00BF04
:1055C00000BF00BF00BF00BF00BF00BF00BF00BFE3
:1055D00000BF00BF00BF00BF00BF00BF00BF00BFD3
:1055E00000BF00BF00BF00BF00BF4FF40061044810
:1055F000FDF71FFC00BF00BF00BF00BF10BD0000D3
:10560000000C014008B501210820FDF7FBFE4FF416
:105610000060ADF8000003208DF8020010208DF826
:10562000030069460148FDF770FB08BD000C01400E
:1056300010B54FF400611148FDF7FDFB00BF00BF3E
:1056400000BF00BF00BF00BF00BF00BF00BF00BF62
:105650004FF400610948FDF7ECFB00BF00BF00BF3D
:1056600000BF00BF00BF00BF00BF00BF00BF00BF42
:1056700000BF00BF00BF00BF10BD0000000C014014
:1056800010B586B00446012144F20400FDF7BAFECD
:105690004FF40070ADF8140003208DF816001820A8
:1056A0008DF8170005A91C48FDF72FFB4FF480600B
:1056B000ADF8140004208DF8170005A91648FDF771
:1056C00024FB25208DF8000003208DF801008DF8C3
:1056D000020001208DF803006846FDF7E5FC019407
:1056E0000020ADF80800ADF80A00ADF80C00ADF8E8
:1056F00010000C20ADF80E0001A90848FFF718F8BB
:10570000012240F225510548FEF7EDFF0121034833
:10571000FEF74CFF06B010BD000801400038014004
:105720000FB438B505A800900B48009A0499FAF711
:10573000D3FD002000900848FAF7ECFE85B2002463
:1057400005E00549085DFFF789FA601C84B2AC42A8
:10575000F7DB38BC5DF814FB040B002010B5002902
:105760000AD00878002807D005487844FAF736FFB1
:10577000002801D0002010BD0248784410BD000070
:10578000220200001A02000010B500290AD0087891
:10579000002807D005487844FAF720FF002801D0F8
:1057A000002010BD0248784410BD00001202000025
:1057B0000A020000FBF7C4BAFBF7F8BB12010002B3
:1057C0000200004083044057000201020301090265
:1057D0004300020100C0320904000001020201007E
:1057E00005240010010524010001042402020524FF
:1057F000060001070582030800FF09040100020AF0
:105800000000000705030240000007058102400078
:1058100000040309042603530054004D006900638B
:105820000072006F0065006C006500630074007218
:10583000006F006E00690063007300320353005470
:10584000004D0033003200200056006900720074E1
:1058500000750061006C00200043004F004D0020E7
:105860000050006F0072007400200020000400004F
:10587000080000000000000002000100001000000D
:10588000000000000000000030313233343536377C
:105890003839414243444546403058003031323374
:1058A0003435363738396162636465664030780074
:1058B0003031323334353637383961626364656686
:1058C000787000303132333435363738394142431D
:1058D000444546585000000002400000000000A06F
:1058E0000000000005400000000000C800000000AB
:1058F0000C4000000000409C000000001940000027
:105900000020BCBE0000000034400000BFC91B8E58
:1059100000000004B5400000504BCFD06607E2CF36
:10592000010000006C4100003E8251AADFEEA73466
:1059300001000000D9420000DCB5A0E23A301F9718
:10594000FFFFFFFFB4450000FD25A0C8E9A3C14F3C
:10595000FFFFFFFFFF3F000000000080000000008D
:10596000FF3F00000000008000000000B85A00085F
:10597000000000209C01000028010008585B00087E
:105980009C0100204C1D0000840100081C00000048
:1059900043000000F8FFFFFF0C0000000E000000B5
:1059A0000F0000002E000000100100004300000066
:1059B000F8FFFFFF00404040404040404040414130
:1059C00041414140404040404040404040404040D4
:1059D000404040404005020202020202020202026E
:1059E000020202020220202020202020202020026B
:1059F00002020202020290909090909010101010FB
:105A00001010101010101010101010101010101096
:105A1000020202020202888888888888080808082A
:105A200008080808080808080808080808080808F6
:105A3000020202024000000000000000000000001E
:105A40000000000000000000000000000000000056
:105A50000000000000000000000000000000000046
:105A60000000000000000000000000000000000036
:105A70000000000000000000000000000000000026
:105A80000000000000000000000000000000000016
:105A90000000000000000000000000000000000006
:105AA00000000000000000000000000000000000F6
:105AB00000000000000000001184A24A04200B0135
:105AC0000203040607080903012A0210011429250C
:105AD0006929052F02040608141A03531254124DA3
:105AE00012330214320210FF137D290C1C08A73058
:105AF000040B100D2A14512AC2C212081A040713EB
:105B0000214F1408D94D1B0801081A1D0413C94C54
:105B10001B08B1101A99041A41041A2D041A7104B1
:105B200041324029440B18C14E741AD91C13BC577A
:105B30003308121ACE0832431311583308041A15C9
:105B40000832261A3B0829E6227073201A2992513E
:085B50002A8099011E000000EB
:04000005080000ED02
:020000040800F2
:10800000C84700209981000823D60008FFCE000849
:1080100051D40008AD8A00082F03010800000000B9
:1080200000000000000000000000000001810008C6
:10803000F79200080000000045810008A9E600084A
:10804000B3810008B3810008B3810008B381000840
:10805000B3810008B3810008B3810008B381000830
:10806000B3810008B3810008B38100089D92000825
:10807000B3810008B3810008A9920008B5920008F6
:10808000B3810008C1920008B3810008B3810008E1
:108090006D020108B3810008B3810008B3810008B4
:1080A000B38100083DE70008B3810008B3810008F0
:1080B00065E70008B381000871E70008B381000894
:1080C000B3810008B3810008B3810008B3810008C0
:1080D000B3810008F1EC0008B3810008B381000807
:1080E0001D930008B3810008B3810008DFF80CD0AD
:1080F00000F0F8FB00480047450C0108C847002085
:10810000224B19680868B0E8F00F80F30988BFF3C4
:108110006F8F4FF0000080F311884EF00D0E704706
:108120000000000006480068006880F3088862B616
:1081300061B6BFF34F8FBFF36F8F00DF00BF00BF8B
:1081400008ED00E0EFF30980BFF36F8F0F4B1A6863
:1081500020E9F00F106008B54FF0500080F311884F
:10816000BFF34F8FBFF36F8F0AF002F84FF000009C
:1081700080F31188BDE8084019680868B0E8F00F7E
:1081800080F30988BFF36F8F704700BFE4000020C1
:10819000EFF3058070470000064880470648004717
:1081A000FEE7FEE7FEE7FEE7FEE7FEE7FEE7FEE7A7
:1081B000FEE7FEE73BE70008ED800008202A04DB2D
:1081C000203A21FA02F00021704721FA02F3D04050
:1081D000C2F1200291400843194670470649074AF8
:1081E0000868504343F23902104408604008704761
:1081F00001490860704700000C0500206D4EC64123
:1082000040EA01039B0703D009E008C9121F08C018
:10821000042AFAD203E011F8013B00F8013B521E98
:10822000F9D27047D2B201E000F8012B491EFBD20F
:1082300070470022F6E710B513460A460446194671
:10824000FFF7F0FF204610BDF0B480EA0102D40F22
:108250004200B2EB410F02D20246084611464A00E4
:1082600042D0C30DDDB2C1F3C752AD1A202D35DAAD
:10827000C1F3160141F4000204B15242C5F12006D7
:1082800002FA06F12A411044B3EBD05F23D0C4B107
:10829000012DA0EBC35009DCF0BC4FF0004202EA14
:1082A000C352DBB200F5000000F090BA400000F1CC
:1082B000807000EBC350A0F1807040EAD17049009B
:1082C00009E0490841EAC071A0EBC35000F5000085
:1082D000400800EBC350F0BC00F06FBA61420122CD
:1082E00002EB4101001BF6E7F0BC704781F0004152
:1082F000AAE780F00040A7E780EA010210B502F08B
:108300000043400022D04A001FD0010E01EB126151
:10831000C0F35600C2F3560240F4000042F40002DB
:10832000A0FB022000047F39140400D0401C50EA56
:10833000124001D44000491EC2B20C0604EBD0101A
:10834000401C4008802A02D003E0002010BD20F02D
:108350000100002900DA0020184310BD30B480EA83
:10836000010202F0004530F0004221F0004013D03D
:1083700090B1C30DD40DC2F31601C0F31600E41A78
:1083800041F4000140F400027D34914201D3641CA9
:1083900000E04900002C02DA30BC002070474FF4A6
:1083A00000000023914201D3891A034340084FEA99
:1083B0004101F7D151B1914202D14FF0004105E0A6
:1083C00002D24FF0010101E06FF0010103EBC45054
:1083D000284430BC00F0F1B92DE9FE4F804681EA17
:1083E0000300C00F0C46009021F0004123F000452F
:1083F000B8EB0200A94105D24046214690461C46F2
:108400000B46024623F00040104347D0270DC7F328
:108410000A00C3F30A510290401A019040286BDA17
:10842000C3F3130040F4801B0098924620B1002350
:10843000D2EB030A63EB0B0B01985946C0F14002E3
:10844000504600F099F906460D4650465946019AA5
:1084500000F0A1F910EB08006141002487EA1152F5
:1084600084EAE7731A4340D0009A62B3019A012A62
:108470004FEA075215DC001B61EB02014FF000428E
:1084800002EA0752CDE90042001C41F58011324654
:108490002B4600F0D8F903B0BDE8F08F40462146E6
:1084A000F9E7001B61EB0201001C41F58013001885
:1084B0005B412018A2F5001747EB030140EAD57095
:1084C000B6196D4111E06D084FEA360645EAC075F0
:1084D0004FEA0752001B61EB0201001C41F58011BD
:1084E00049084FEA30000019514132462B4603B08B
:1084F000BDE8F04F00F098B9009801224000002339
:10850000D0EB020263EBE073009821464FEAE0747F
:10851000B8EB000061EB0401E9E783F000435BE79F
:1085200081F0004158E72DE9FE4F81EA030404F091
:10853000004421F0004100944FF0000B23F0004371
:1085400050EA01045ED052EA03045BD0C3F30A543C
:10855000C1F30A552C44A4F2F3340194A0FB025455
:10856000C1F3130141F48011C3F3130343F48013E7
:1085700001FB024400FB034E840A970A44EA81543B
:1085800047EA8357A4FB076802958D0A05FB078518
:108590004FEA932C04FB0C542705029D4FEA065822
:1085A00047EA1637B5EB08056EEB070C870E920EFF
:1085B00047EA811742EA8312A7FB0201B6EB0B01DF
:1085C00064EB00042B0D43EA0C335E1844EB1C50A3
:1085D000DA465146E7FB0201C5F313044FEA0B33B9
:1085E00043EA14534FEA0432019C43EA0603A4F120
:1085F0000C040294009CCDE900B400F024F903B00F
:10860000BDE8F08F00200146F9E72DE9F04D81EA41
:10861000030404F0004B21F0004514464FF0000A1B
:1086200023F0004150EA050220D054EA01021DD097
:10863000C5F30A570246C5F31303C1F31300C1F390
:108640000A5640F4801543F48013A7EB0608101B6C
:10865000D64608F2FD3873EB050002D308F1010895
:1086600001E092185B41B8F1000F03DA00200146E7
:10867000BDE8F08D00204FF48011064684460EE0E0
:10868000171B73EB050705D3121B63EB05030643AA
:108690004CEA010C49084FEA300092185B4150EA5D
:1086A0000107EDD152EA030012D082EA040083EA06
:1086B0000501084305D0101BAB4106D2012200235F
:1086C00006E000224FF0004302E06FF00102531079
:1086D0001AEB06004CEB085110EB0A0041EB0B01C2
:1086E000BDE8F04D00F0A0B8C10F80EAE07008448A
:1086F000CA079623002100F069B89623002211468C
:1087000000F064B80EB540F2334102910021CDE98A
:1087100000110A460B4600F096F803B000BD20F0A9
:108720000040C10DC0F3160040F400007F2901DABB
:1087300000207047962903DCC1F19601C8407047BC
:10874000963988407047C1F30A5210B5C1F313013E
:1087500040F2FF3341F480119A4201DA002010BD4B
:1087600040F233439A42A2F2334203DC5242FFF713
:1087700025FD10BD904010BD202A04DB203A00FAF0
:1087800002F1002070479140C2F1200320FA03F368
:10879000194390407047202A06DBCB17203A41FA54
:1087A00002F043EAE07306E041FA02F3D040C2F17E
:1087B000200291400843194670470029A8BF70471E
:1087C000401C490008BF20F00100704710B4B0FA07
:1087D00080FC00FA0CF050EA010404BF10BC7047A2
:1087E00049B1CCF1200421FA04F411FA0CF118BFBC
:1087F000012121430843A3EB0C01CB1D4FEA00618B
:108800004FEA102042BF002010BC704700EBC3505D
:1088100010440029A4BF10BC7047401C490008BF89
:1088200020F0010010BC704710B5141E73F1000455
:1088300008DA401C41F1000192185B411A4301D152
:1088400020F0010010BD2DE9F04D92469B4611B17C
:10885000B1FA81F202E0B0FA80F220329046FFF7DE
:108860008BFF04460F4640EA0A0041EA0B015346DB
:108870005A46084313D0114653EA010019D0C8F1F3
:1088800040025046FFF79AFC05460E4650465946B0
:108890004246FFF771FF084305D0012004E020465F
:1088A0003946BDE8F08D0020054346EAE0762C43CA
:1088B00037430A986305E40AA0EB08000022FD0A8A
:1088C00044EA47540A3002D500200146E9E7010591
:1088D00010196941DDE9084500196941BDE8F04D0D
:1088E000A2E70000064C074D06E0E06840F00103F7
:1088F00094E8070098471034AC42F6D3FFF7FAFB30
:10890000143101083431010870B58C1810F8015B7E
:1089100015F0070301D110F8013B2A1106D110F818
:10892000012B03E010F8016B01F8016B5B1EF9D11C
:108930002B0705D40023521E0DD401F8013BFAE7A2
:1089400010F8013BCB1A921C03E013F8015B01F80D
:10895000015B521EF9D5A142D8D3002070BD70B57D
:10896000044600688168C943C9071BD1816821F0AA
:108970000101816002F02AF805460EE002F026F8B7
:10898000401B022809D9A06A40F01000A062E06AEA
:1089900040F00100E062012070BD20688068C043A3
:1089A000C007EBD0002070BD10B50146406A826A56
:1089B00012F0500F05D0006A026BBDE81040084667
:1089C0001047816A41F40071816201688968C1F3CE
:1089D000424107290CD1017B51B9816A21F4807190
:1089E0008162816AC90403D4816A41F00101816214
:1089F00001F04EFB10BD10B5406A816A41F04001A4
:108A00008162C16A41F00401C16201F043FB10BD03
:108A100010B5406A01F03DFB10BD0000F8B500261E
:108A20000446009600688168C943C90727D0816859
:108A300041F001018160134813490068B0FBF1F077
:108A400000E0401E00900028FBD101F0BFFF05466A
:108A500010E001F0BBFF401B02280BD9A06A40F0D8
:108A60001000A062E06A40F00100E06284F8246037
:108A70000120F8BD20688068C043C007E9D100200C
:108A8000F8BD0000E000002040420F00064910B58C
:108A9000322201F5967001F0D5FB002803D0BDE825
:108AA000104000F03FBC10BDB8090020FEE710B533
:108AB00000F032F9032000F0D5F84FF4C8742046D6
:108AC00001F0A4FD022000F0CDF8204601F09EFD4B
:108AD000012000F0C7F8204601F098FDBDE81040E5
:108AE00000F020B92DE9F0410F46804601F06EFFFD
:108AF000374E00244FF00105C6E904047178B278BE
:108B0000F3780A431A4357D089B1D6E90623821A6B
:108B100064EB0301962300209A1A884107D27470EF
:108B2000B57000F0FFF801F051FFC6E90804B07815
:108B300028B3D6E90401D6E90823821A61EB0301C0
:108B40000023D2F196008B4119D2B47030787F1E89
:108B5000B8420DDA757000F0DFF8404600F082F898
:108B600001F034FFC6E906043078401C307006E09E
:108B700034702746F57001F029FFC6E90A07F0783E
:108B8000002817D0D6E90421D6E90A30D31A61EBC0
:108B900000014FF4FA700022C01A8A410AD2F47020
:108BA000757000F0B9F8404600F05CF801F00EFF77
:108BB000C6E90604BDE8F081757001F007FFC6E95B
:108BC000060400F0A9F8404600F04CF83470F1E7D4
:108BD000E002002070B50D46044600F09DF82046E6
:108BE00000F040F8284608F0DBF9BDE8704000F0DE
:108BF00099B810B500F090F8012000F033F84FF468
:108C0000C874204601F002FD022000F02BF8204637
:108C100001F0FCFC032000F025F8204601F0F6FCF2
:108C2000BDE8104000F07EB810B500F075F80720E0
:108C300000F018F8C82008F0B3F900F073F8C82065
:108C400008F0AEF900F068F8072000F00BF8C82033
:108C500008F0A6F900F066F8BDE81040C82008F05A
:108C60009FB9000010B51C4B4FF4E574082823D2BF
:108C7000DFE800F02204070E151C232A4FF465706C
:108C800016E04FF44C7003F099FE4FF4CC7020E0E6
:108C900040F2D72003F092FE40F26B1019E040F250
:108CA000BA2003F08BFE40F25D1012E040F2632028
:108CB00003F084FE1868446310BD4FF4087003F09D
:108CC0007DFE4FF4887004E040F2E51003F076FE7C
:108CD000F2201968486310BD4C0C002010B500F05C
:108CE0001BF80120FFF7BEFFC82008F059F900F07B
:108CF00019F8C82008F054F900F00EF80120FFF729
:108D0000B1FFC82008F04CF900F00CF8BDE81040A5
:108D1000C82008F045B900000021014803F0F4BC68
:108D20004C0C00200021014803F006BE4C0C002032
:108D300010B50A4C2021204601F0DAFC80212046A3
:108D400001F0D6FC064C0421204601F0D1FC21158F
:108D50002046BDE8104001F0CBBC000000080140F7
:108D6000000C014070B5044600F03CF81C49FF209F
:108D700000264870642001F049FC00F077F800B943
:108D80000126012001F042FC24B1012C05D0022C67
:108D900008D105E0124D923504E0114D4A3501E04D
:108DA0000F4DAD1CD6B9002405EB4400417815F8F1
:108DB000140000F0C1F8142000F09EFA641CE4B224
:108DC000242CF1D30A2000F097FA012000F06EF86D
:108DD000362000F087F80A2000F08EFA304670BD89
:108DE0002803002001222021014801F0EABD0000F3
:108DF00000080140094902880A8042884A80828826
:108E00008A80C288CA8002890A8142894A8182890D
:108E10008A81C089C881002070470000C2430020B9
:108E20007CB540F080000F4D8DF800004FF4805469
:108E300000222146284601F0C4FD01231A46694656
:108E4000094802F053FF01231A4601A9064802F01F
:108E5000A3FE01222146284601F0B3FD9DF804003F
:108E60007CBD0000000C0140640B002010B53020D8
:108E700000F038F8012001F0C9FB002000F016F8DE
:108E80000E20FFF7CDFFC42801D0002010BD012027
:108E900010BD000004490A78824204D008700146DF
:108EA0003E2000F049B870472803002010B5012883
:108EB0000DD002284FF02F014FF002000ED000F02D
:108EC0003BF82F210020BDE8104000F035B82F21DD
:108ED000002000F031F86F210220F4E700F02CF8B8
:108EE0006F21EFE731B50A4D4FF48054002221463F
:108EF000284601F066FD01231A466946054802F03E
:108F0000F5FE01222146284601F05BFD38BD000038
:108F1000000C0140640B002070B505460C463B2058
:108F2000FFF7E0FF224629463F2000F023F8BDE886
:108F300070403520FFF7D6BF38B50C4D8DF80000D6
:108F40008DF801104FF4805400222146284601F08C
:108F500038FD012302226946054802F0C7FE0122BE
:108F60002146284601F02DFD38BD0000000C0140CF
:108F7000640B00202DE9F843104E1746884604463E
:108F80004FF4805500222946304601F01AFD44F086
:108F900040008DF8000001231A466946084802F097
:108FA000A5FE01233A464146054802F09FFE0122F4
:108FB0002946304601F005FDBDE8F883000C01406C
:108FC000640B0020012001F021BB00002DE9F041DD
:108FD0004E4C0746607938B3617B207C814204D0D7
:108FE000012005F08BFA607B2074A17B607C8142BC
:108FF00004D0022005F082FAA07B6074217BE07B24
:10900000814204D0062005F079FA207BE073207AB3
:10901000002520B10121FF2005F070FA2572607A49
:1090200000B1657265716DE0E07A394D58B901F0B3
:10903000CDFCA968401A322805D901F0C7FCA86008
:1090400000F094FC5EE0324EB61C3078FF2813D15D
:1090500001F0BCFCA968401A32280DD901F0B6FC19
:10906000A8606878402802D0202802D04AE0002179
:1090700000E0012106202CE07078FF2813D101F0D8
:10908000A5FCA968401A32280DD901F09FFCA86000
:109090006878402802D0202802D033E0012100E087
:1090A0000221012015E0B078FF2815D101F08EFCD7
:1090B000A968401A32280FD901F088FCA8606878A6
:1090C000402802D0202802D01CE0002100E002212C
:1090D000022000F02DFC15E0E07A98B13078FF28EE
:1090E00010D07078FF280DD0B078FF280AD008483B
:1090F0003946283000F09AFC05491A2228310548E3
:1091000003F006FE0020BDE8F0810000B24500201B
:10911000A8040020D80C0020012001F077BA00201C
:10912000704700207047000010B50121094806F083
:109130003DF8C2B20748084BD0F8B812002003E04F
:109140000C5C1C54401CC0B29042F9D305F014F9D9
:10915000002010BDA00D0020A81500200F2800D968
:109160000F200949402231F81010A1F5577101EB89
:109170004101C90302EB114189B2072801D941F429
:1091800000610846704700004C04002011B1904275
:1091900004D801E0984201D20020704701207047B6
:1091A00030B51748807AC1B200F00703022901D216
:1091B000891CC9B2E92901D9E739C9B22F20B1FB0D
:1091C000F0F200FB121008B9491CC9B200220D4D83
:1091D000EB245818B0FBF4F304FB1303180003D07E
:1091E0005A2801D0DC2801D1581CC0B22E2A00D93F
:1091F0000020A854521CD2B2322AEAD330BD00005B
:109200006C040020B04400200B4810B5008860B109
:10921000022000F0F5FCA0F6B830404280B240F2E7
:109220001A41884205D2002010BD002000F0E8FC61
:10923000F5E7012010BD00002A02002010B5002330
:109240000E4A072810D2DFE800F00406090F0C10C0
:109250001400517006E05370117004E053701370E5
:1092600005E053701370937010BD517011709170C0
:1092700010BD802050701370907010BD1404002039
:109280000448002101818171034890F82F0000F00B
:10929000D3B900006C040020B0440020014801F064
:1092A000A3B80000140B0020014801F09DB8000095
:1092B000180D0020014801F097B800005C0D002057
:1092C000014801F091B80000940C002030B590F8EE
:1092D00040500124AC40C56B6C6004686360436817
:1092E000102B036803D099600068C26030BD9A609B
:1092F0000068C16030BD70472DE9F041064600F0BE
:109300008DFD04460D46002700F088FD001B61EB33
:109310000501801BB941F7D3BDE8F0814FF48060AF
:1093200001F058BA70470000064A0021D161064991
:109330000A6942F002020A614861086940F040008F
:10934000086170477016002000200240044B002284
:10935000DA61044A136943F0010313610180704725
:10936000701600200020024014490020CA68D3066D
:10937000134A04D5D06940F00200D0611020CB68B8
:109380005B0705D5D36943F00103D36140F00400C6
:10939000CB69DB0707D0D36943F00403D361CA6903
:1093A00022F00102CA61A0F58072013A01D0C860C2
:1093B0007047C86920F00100C86170470020024072
:1093C0007016002070B5044601F000FB0546114EF2
:1093D00009E0601C07D024B101F0F8FA401BA0425C
:1093E00001D9032070BDF068C007F2D1F068800693
:1093F00001D52020F060F068C00605D4F069C007F0
:1094000002D1F068400703D5FFF7AEFF012070BD21
:10941000002070BD002002402DE9F041274D044698
:10942000E87100F0C3FA688100F04EFA4FF0E020D6
:109430008069FEF7DDFEFEF7D1FE2E2190FBF1F2F2
:1094400001FB1200401CC2B26A7003E0491C01F02B
:109450000300A870A978501A8007F7D1C8B2101A73
:109460008008E8702046FFF77DFC012824D0144EC8
:10947000002406F132073620FFF734FD315D0A2063
:10948000FFF75AFD3320FFF72DFD012001F0BEF854
:109490002520FFF7C5FC3855641CE4B2302CEAD314
:1094A00008480078FFF7F6FC022068712879305CE4
:1094B000BDE8F04100F008B8BDE8F08140040020AC
:1094C000244400202903002010B504463620FFF76D
:1094D00009FD0848015D2520FFF72EFD05483238BB
:1094E000015D0A20FFF728FDBDE810401420FFF7BA
:1094F00003BF0000564400202DE9F047404A0026F3
:10950000404DD179012913D01D21297051890B0AB1
:109510006B70A9700221E9701179937801EB8313C4
:109520002B71D3786B710123AB71212902D003E039
:109530002021EAE7212111714FF0000885F807800A
:1095400085F8088091799146C9074FF0080A00D044
:1095500008262B4902880C3100240A8042884A8060
:1095600082888A80C288CA8002890A8142894A81A7
:1095700082898A81C089C8813046FFF7EFFD761C59
:109580000746F6B23046FFF7E9FD2919C7F3032273
:1095900042EA0012761C4F720009E41C8A72E4B29F
:1095A000F6B2C8720C2CE7D385F815A099F806100E
:1095B000491C89F8061099F807004FF01601012898
:1095C0000ED040466854491CC9B21C29FAD319214F
:1095D000E81C06F051FF010A29776877BDE8F0879B
:1095E00042466A54491CC9B21F29FAD31C21E81CFF
:1095F00006F042FF010AE97785F82000EEE7000057
:10960000400400208844002010B50446082118209A
:10961000FFF792FC0CB1032102E006484089010AE1
:109620000920FFF789FC0521BDE810400720FFF75E
:1096300083BC00006C04002010B504463620FFF700
:1096400051FC0848015D2520FFF776FC05483238BB
:10965000015D0A20FFF770FCBDE810403320FFF7E2
:1096600041BC0000E244002030B5244B244A1121C3
:10967000197051890C0A5C7099705178D970002169
:10968000197101225A719972D972197459741C494D
:1096900002880C310A8042884A8082888A80C28887
:1096A000CA8002890A8142894A8182898A81C08965
:1096B000C8810022104606F0BFFE042A03EB020117
:1096C0000BD2887103EB5201D5078C7A6D0FC0F372
:1096D0000320A84004438C720BE00872111F03EBB7
:1096E0006101D5070C7C6D0FC0F30320A840044333
:1096F0000C74521CD2B2082ADCD330BD14450020B1
:109700006C04002070B53620FFF7ECFB5C210D20C7
:10971000FFF712FC76210E20FFF70EFC27210F2009
:10972000FFF70AFC0220FFF7E7FD3620FFF7DAFB20
:109730005C210D20FFF700FC76210E20FFF7FCFBDB
:1097400027210F20FFF7F8FB0C4D2F246878B0FB82
:10975000F4F104FB11000A49095C2520FFF7ECFB3A
:109760006878B0FBF4F104FB110005493239095C5B
:10977000BDE870400A20FFF7DFBB00006C0400204A
:10978000E244002070B5334A0021334CD0790128DF
:1097900052D04FF01D0020704FF0030060704FF06A
:1097A0000105A57050894FEA1023E37020711089DC
:1097B0004FF00A02B0FBF2F302FB1300264B00EB62
:1097C0008002A3F164036271985CA07102F101024E
:1097D000D0B21A5C00F10100C0B2E2711A5C00F173
:1097E0000100C0B222721A5C00F10100C0B26272C4
:1097F000185CA0724FF00200E07225736173A173D0
:10980000E17321746174A174E17421756175A175AE
:10981000E17521766176A176E17610D121776177C5
:10982000A1774FF01C0104F1030006F025FE010AA8
:10983000E17784F8200070BD4FF02000ABE74FF0D7
:10984000190104F1030006F017FE010A2177607781
:1098500070BD0000400400208844002018481121F9
:10986000184A0170032141700121817051890B0A4E
:10987000C370017111890A22B1FBF2F302FB1311CB
:1098800001EB8101A0F164024171535C491CC9B232
:109890008371535C491CC9B2C371535C491CC9B282
:1098A0000372535C491CC9B24372515C817200213E
:1098B000C172017341738173C17301744174704744
:1098C000144500206C04002030B51748807AC1B2DE
:1098D00000F00703022901D2891CC9B2E92901D984
:1098E000E739C9B22F20B1FBF0F200FB121008B922
:1098F000491CC9B200220D4DEB245818B0FBF4F3FB
:1099000004FB1303180003D05A2801D0DC2801D12E
:10991000581CC0B22E2A00D90020A854521CD2B222
:10992000322AEAD330BD0000400400202444002045
:1099300010B50C4CEE220623227063702C23A3700A
:10994000E270EA2222716071A1710521A01C06F06B
:1099500083FDE0712146BDE810400822024803F073
:10996000D7B90000B4040020D80C002010B50D4C6D
:10997000EE2005212070042060702820A0700020B7
:10998000E070EA202071542060719320A071A01C27
:1099900006F062FDE0712146BDE810400822024851
:1099A00003F0B6B9B4040020D80C00200EB5684608
:1099B00000F018F99DF800009DF802109DF80620AF
:1099C00008449DF80410114408449DF808109DF8BF
:1099D000032008449DF80A1008449DF80110114422
:1099E0009DF8052002EB002008449DF8071008446C
:1099F0009DF8091008449DF80B10084480B20EBD74
:109A000010B50022084B114601EB81040444491CA7
:109A100033F81440C9B222440529F5D30520B2FB1E
:109A2000F0F080B210BD0000B80900202DE9F0432D
:109A3000814697B00C464888FEF764FE644B0022CE
:109A4000CDE90423634BDFF89481CDE90223624B17
:109A5000CDE90023434607F029F9614D688020884D
:109A6000FEF750FE5A4B0022CDE90423594BCDE9B5
:109A70000223594BCDE90023434607F017F928800C
:109A8000A088FEF73FFE524B0022CDE90423514B44
:109A9000CDE90223504BCDE90023434607F006F9F8
:109AA000A880E088FEF72EFE494B0022CDE9042372
:109AB000484BCDE90223484BCDE90023434607F04C
:109AC000F5F8E8802089288161896981A189A981C7
:109AD000E189E981FEF716FE3D4B0022CDE9042322
:109AE0003C4BCDE902233C4BCDE90023434607F034
:109AF000DDF807466889FEF705FE354B0022CDE903
:109B00000423344BCDE90223334BCDE900234346F4
:109B100007F0CCF80646A889FEF7F4FD2C4B00228E
:109B2000CDE904232B4BCDE902232B4BCDE90023B8
:109B3000434607F0BBF80446E889FEF7E3FD244BF3
:109B40000022CDE90423234BCDE90223224BCDE9AA
:109B50000023434607F0AAF82988069169880791EF
:109B6000A9880891E988CDE90C404FF478700B96EC
:109B70000E900F90109011901290139014901590D9
:109B8000CDE90917EE2189F8001009F1010018212B
:109B900000F8011B1621441C0022017011461346D7
:109BA00006AD55F823608E4032430B3103E004F8D4
:109BB000012B120A0839C9B20829F8D25B1C102BF4
:109BC000EFDB172106F048FC207017B0BDE8F083EA
:109BD00000009C400000684000409F4000408F40D3
:109BE000EA0400200549096801600449091D096863
:109BF000416002490831096881607047E8F7FF1F3A
:109C00002DE9F04780460024424800F00DFFB8F1EE
:109C1000010F08D0B8F1020F05D0B8F1030F02D040
:109C2000B8F1000F73D13C483B4F08EB4806007871
:109C3000183707EB460478B937F81600A0F57F41CE
:109C4000FF3909D140F6C41027F816004FF4FA6026
:109C5000608040F2DC50A0804046FFF7D1FE37F82C
:109C60001650A84209D84046FFF7CAFEA588A84268
:109C700003D34046FFF7C4FE0546B4F80280DFF880
:109C80009CA04FF08849A8451BD837F81600A0EBD8
:109C90000800FEF729FD01464846FEF75FFB044633
:109CA0004046FEF72AFD06462846FEF726FD3146C9
:109CB000FEF71CFB2146FEF71FFB5146FEF7C4FAD8
:109CC00019E0A088A8EB0000FEF70EFD014648460B
:109CD000FEF744FB04462846FEF70FFD05464046C6
:109CE000FEF70BFD2946FEF701FB2146FEF704FBBC
:109CF0005146FEF7FEFAFEF712FD84B240F2DC7028
:109D0000844203D84FF47770844200D20446204640
:109D1000BDE8F087580B0020A40200200080BB445F
:109D20000148006970470000680200200148807AFD
:109D3000704700006802002001480078704700006A
:109D4000400200202DE9F047334A4FF4777540F286
:109D5000DC7640B140F2DC57012806D0022826D03C
:109D6000032856D14BE040214BE01021904610468D
:109D700000F022FE012805D12021404600F01CFE03
:109D800000B92C4610214546404600F015FE30B97A
:109D90002021284600F010FE012800D13446102171
:109DA000284600F009FE012833D1202120E080213F
:109DB0009046104600F000FE4FF40079012804D1CF
:109DC0004946404600F0F8FD00B380214546404634
:109DD00000F0F2FD28B94946284600F0EDFD0128C3
:109DE00016D08021284600F0E7FD012811D1494610
:109DF000284600F0E1FD01280BD13C4609E04FF474
:109E00008071104600F0D8FD012801D02C4600E0FA
:109E100034462046BDE8F087000C014070B508F0DC
:109E200059FD4FF0E02200215369946952691B1BD0
:109E30004FF47A746343B3FBF2F32246A0FB02466D
:109E400001FB026200FB01221819514170BD0000A4
:109E500070B54A4D4A4801226978006805F1180436
:109E6000012907D002291AD0002403297BD0AC7025
:109E70002C7070BD2A70022108F0B6F90220FFF79D
:109E8000BFFDE0810320FFF7BBFDA0820120FFF7AB
:109E9000B7FD20810020FFF7B3FD608070BDA97879
:109EA00061B961882180A1802189E1806181E18996
:109EB000A1812182A18A6182E182AA70042108F035
:109EC00093F90020FFF79CFD2188884203D90020E8
:109ED000FFF796FD20800020FFF792FDA1888842C1
:109EE00003D20020FFF78CFDA0800120FFF788FD42
:109EF000E188884203D90120FFF782FDE08001203C
:109F0000FFF77EFD6189884203D20120FFF778FDCB
:109F100060810220FFF774FDA189884203D90220E5
:109F2000FFF76EFDA0810220FFF76AFD218A8842BB
:109F300003D20220FFF764FD20820320FFF760FDBB
:109F4000618A884203D90320FFF75AFD608203200B
:109F5000FFF756FDE18A8842A0D20320FFF750FDAB
:109F6000E08270BDFFE7082108F03EF90221A868F1
:109F700008F03AF904F090F96C70F2E7A4020020BE
:109F8000E802002010B5FEF781FDBDE8104003F0A7
:109F900031BE0000F8B50023009390F824201C4641
:109FA000012A12D0012280F824204A681F26072A9D
:109FB0000DD205686F6B521E02EB82029640B743CA
:109FC0000E68964037436F6319E00220F8BD0568BC
:109FD0000D2A0AD22F6BD21F02EB82029640B743A2
:109FE0000E68964037432F6309E0EF6A0D3A02EBA3
:109FF00082029640B7430E6896403743EF620A6884
:10A00000072605680A2A0AD3EF680A3A02EB4202D9
:10A010009640B7438E6896403743EF6008E02F695B
:10A0200002EB42029640B7438E68964037432F6159
:10A030000A68102A01D0112A20D1124D0268AA42C2
:10A0400017D195682D0219D4956845F400059560DF
:10A050000968102912D10C490C4A0968B1FBF2F1C8
:10A0600001EB8101490000E0491E00910029FBD16C
:10A0700004E0816A41F020018162012380F82440DC
:10A080001846F8BD00240140E000002040420F00C7
:10A0900070477047704700002DE9F0414FF000060F
:10A0A000040035467DD0A06A002728B9E76284F80D
:10A0B0002470204600F07EF82046FEF750FCA16A8E
:10A0C000C90600D420B1A06A40F01000A06268E088
:10A0D000A16A21F4885141F00201A1626268E1693C
:10A0E000237B0A4346EA43010A43A1684FF4807682
:10A0F000B14208D0012906D0002194F814C0BCF167
:10A10000010F02D00AE03146F7E7F3B1A36A43F04A
:10A110002003A362E36A43F00103E3622368D3F8F8
:10A1200004C02CF4694C4CEA010CC3F804C021684B
:10A130008B68DFF874C003EA0C0313438B60A168DB
:10A14000B1420BD0012909D00CE0DFF860C0A3694F
:10A150000CEB43330B4343F40061DFE7218A0D0529
:10A16000A5F580152168CB6A23F470032B43CB62DD
:10A17000216889680E4B1940914208D1E762A16AB3
:10A1800021F0020141F00101A162BDE8F081A06A65
:10A1900020F0020040F01000A062E06A40F00100F0
:10A1A000E0620120F1E70000FDF7E1FF00E0FFFFC2
:10A1B000FE0E1FFF70B586B0002406460094019481
:10A1C0000294039400681A4988422FD1194988697A
:10A1D00040F400708861886900F400700490886918
:10A1E00040F0040088618869694600F0040004902A
:10A1F0001F200090032001900F4800F0F7FA104D47
:10A200000E48C5E900048020C5E9024040002861ED
:10A21000800068612020A861C001E861284600F044
:10A220008FF908B1FFF77EF835626E6206B070BD37
:10A2300000240140001002400008014008000240D4
:10A24000140B00202DE9F047894604463B4900687D
:10A250003B4F0E1D9046884201D0B84207D130686E
:10A2600010F4702F03D001252846BDE8F08794F83C
:10A27000240001280CD0012084F824002046FEF799
:10A28000CDFB05004FF0000104D084F82410EBE76B
:10A290000220EAE7A06A40F60162904340F4807031
:10A2A000A0622068B84218D1326812F4702F14D01E
:10A2B000A06A40F48010A0623068400505D5A06A0D
:10A2C00020F4005040F48050A062A06AC0040AD577
:10A2D000E06A20F00600E06206E0A26A22F4801242
:10A2E000A2624068E9E7E16284F82410216A154817
:10A2F0008862216A1448C862216A14480863216888
:10A300006FF0020008602068816841F4807181600C
:10A31000216843464A464C31206A00F03FF92068E4
:10A320008168C1F342410729816803D041F480115B
:10A33000816099E741F4A001FAE7000000240140A0
:10A3400000280140A9890008118A0008F78900083F
:10A3500010B590F821100024022903D00421816354
:10A3600001243DE001680A6822F00E020A600168DB
:10A370000A6822F001020A601A4A0168914201D17A
:10A38000012121E0174A1432914201D110211BE032
:10A39000144A2832914201D1891515E0114A3C3204
:10A3A000914201D189140FE00E4A5032914202D1FC
:10A3B0004FF4803108E00B4A6432914202D14FF4ED
:10A3C000801101E04FF08071064A083A5160012186
:10A3D00080F82110002180F82010416B01B18847DE
:10A3E000204610BD080002402DE9F05FC16B0B68EC
:10A3F00001680A68046C4FF0040C0CFA04FC4A4D26
:10A40000DFF828A14A4E4B4FDFF82CB1DFF82CE1E2
:10A410001CEA030F2DD05FEA427C2AD50A68920617
:10A4200003D40A6822F004020A600168A94201D13B
:10A43000042119E0514501D1402115E0B14202D17A
:10A440004FF4806110E0B94202D14FF480410BE03B
:10A45000594502D14FF4802106E0714502D14FF4F5
:10A46000800101E04FF080612F4A083A5160C16AD3
:10A470003BE04FF0020808FA04F818EA030F4FF027
:10A4800000094FF0010C35D05FEA827832D50A68B6
:10A49000920605D40A6822F00A020A6080F821C0F8
:10A4A0000168A94201D1022119E0514501D12021C1
:10A4B00015E0B14202D14FF4007110E0B94202D16F
:10A4C0004FF400510BE0594502D14FF4003106E042
:10A4D000714502D14FF4001101E04FF00071124AB2
:10A4E000083A516080F82090816A00291AD0BDE8AE
:10A4F000F05F08470825A5401D4213D0120711D56B
:10A500000A6822F00E020A6090F84010C26B0CFA42
:10A5100001F15160C0F838C080F821C080F8209067
:10A52000016BE2E7BDE8F09F080002401C0002401A
:10A530003000024044000240580002406C000240DB
:10A5400030B528B302C8134A14230A44B2FBF3F20D
:10A550009200C263104A8263022242770B6843F67C
:10A56000F0729343D0E900242243D0E902452C4302
:10A5700022430469224344692243846922431A43E3
:10A580000A6000214163012242770177084630BD0D
:10A59000012030BDF8FFFDBF0000024070B5044649
:10A5A00090F82000002501280CD0012084F820001C
:10A5B00094F821600020012E06D084F820000225A6
:10A5C000284670BD022070BD022684F82160A06379
:10A5D0002068066826F0010606602046FEF776FE33
:10A5E000E06A00282068016802D041F00E0106E010
:10A5F00021F0040101602068016841F00A01016056
:10A600002068016841F001010160D9E770B5044696
:10A6100000F0DCF90546601C02D0044800780444D0
:10A6200000F0D4F9401BA042FAD370BDD400002042
:10A630000348016941F0800101610020704700007A
:10A64000002002402DE9F05F05461D4888460024A1
:10A65000017E16461F46012909D001218146017657
:10A660004CF2503A5046FEF7ADFE18B123E00220FE
:10A67000BDE8F09F012D02D0022D00D00425D34665
:10A68000DFF840A015E0220130463946FDF796FD7F
:10A6900081B208EB4400FEF759FE5846FEF792FEE1
:10A6A000DAF8102022F00102CAF8102018B9641C50
:10A6B000E4B2AC42E7D3002289F81820D8E70000C2
:10A6C0007016002000200240064900200A69120688
:10A6D00007D5054A4A60054A4A600969090600D556
:10A6E000012070470020024023016745AB89EFCD70
:10A6F0002DE9F0430022DFF8C0904FF00F0C55E039
:10A70000012393400B404FD022F003054D44AC6829
:10A710009607370F0CFA07F606EA0408274CA04202
:10A7200001D100240FE0264CA04201D101240AE00F
:10A73000244CA04201D1022405E0234CA04201D1C7
:10A74000032400E00424BC40444512D1AC68B44367
:10A75000AC601E4C25689D432560241D25689D43E3
:10A760002560241D25689D432560241D25689D4383
:10A770002560FF2B01D8044601E000F104044FEAF4
:10A78000820501D9A5F1200526680CFA05F726EA0D
:10A7900007064FF0040707FA05F746EA07062660A2
:10A7A000C46824EA0304C46002F1010231FA02F32E
:10A7B000A6D1BDE8F0830000000001400008014080
:10A7C000000C014000100140001401400004014051
:10A7D00070470000044910B50A68024202D00860C0
:10A7E000FFF7F6FF10BD0000140401402DE9F84FFB
:10A7F000DFF8A491002409F1040A0AF1040B2346AE
:10A800004FF00F080BF1040EBEE00127A7403A40BD
:10A81000BA4272D1DFF884C14D68A5EB0C066545DC
:10A820002BD00DDC032D34D005DC35B3012D19D030
:10A83000022D2FD11BE0112D16D0122D2AD119E097
:10A84000B6F5881F19D006DCB6F5803F15D0B6F5F1
:10A85000801F1FD111E0B6F5001F0ED0B6F5041F02
:10A8600018D10AE0CB6815E0CB681B1D12E0CB685D
:10A8700008330FE0CB680C330CE08B682BB1012B55
:10A880004FF0080303D0476104E0042302E00761AE
:10A8900000E00023FF2A01D8064601E000F104068B
:10A8A0004FEA840501D9A5F12005376808FA05FCAF
:10A8B00027EA0C0703FA05F547EA050737604D68F4
:10A8C000ED0060D5364DAE6946F00106AE61AD696A
:10A8D00024F0030605F001050095324D7719BE6896
:10A8E000A5072D0F08FA05FC26EA0C06DFF8B8C00C
:10A8F000604503D14FF0000C17E044E0DFF8ACC036
:10A90000604502D14FF0010C0FE0DFF8A4C06045B4
:10A9100002D14FF0020C08E0DFF898C0604502D188
:10A920004FF0030C01E04FF0040C0CFA05FC4CEA6C
:10A93000060CC7F808C04D68D9F80060ED034D4615
:10A9400001D5164300E096432E604D68DAF80060AA
:10A95000AD03554601D5164300E096432E604D6881
:10A96000DBF80060ED025D4601D5164300E096433A
:10A970002E604D68DEF80060AD02754601D51643C5
:10A9800000E096432E60641C0A6832FA04F57FF4F6
:10A990003CAFBDE8F88F000000040140000011103A
:10A9A000001002400000014000080140000C01407E
:10A9B00000100140001401408068084000D00120D0
:10A9C00070470AB1016170470904FBE701488068DC
:10A9D00070470000D400002070B5040011D0216839
:10A9E0004CF6CC400860216845F255500860D4E927
:10A9F000000141602168A0688860FFF7E7FF054615
:10AA000008E0012070BDFFF7E1FF401B262801D9B7
:10AA1000032070BD2068C0680028F4D121684AF680
:10AA2000AA200860002070BD00684AF6AA210160D3
:10AA300000207047024881680278114481607047A5
:10AA4000D4000020074810B5016841F010010160F2
:10AA5000032000F095F8002000F006F800F03EF822
:10AA6000002010BD0020024000B5014687B0002242
:10AA70001E2000F065F81E2000F054F81348C1694C
:10AA800041F00401C161C06905A900F0040006900D
:10AA9000684600F0EBFD00F009FE0D494000B0FBF8
:10AAA000F1F10D480B4A491E0260416040F2E73265
:10AAB0000021C0E90321816001F0F0FA10B101200A
:10AAC00007B000BD044801F065FBF9E70010024043
:10AAD00040420F0000080040281600200F4808B52B
:10AAE000816941F001018161816901F001010091F9
:10AAF000C16941F08051C161C069002200F08050FD
:10AB000000900F21901E00F01BF80549486820F0C6
:10AB1000E06040F00070486008BD00000010024096
:10AB200000000140002809DB00F01F0201219140D4
:10AB30004009800000F1E020C0F8001170470000DB
:10AB4000F0B40E4B1B68C3F30223C3F10704042CBB
:10AB500000D904241D1D072D01D2002300E0DB1EB7
:10AB6000012606FA04F56D1E0D409D409E40761E9E
:10AB7000164045EA0601F0BC05F0E0BB0CED00E034
:10AB8000064A00F0070110684FF6FF03184040EA3C
:10AB90000120034908431060704700000CED00E0FD
:10ABA0000000FA05BFF34F8F05480168054A01F41C
:10ABB000E06111430160BFF34F8F00BFFDE700006C
:10ABC0000CED00E00400FA0510B50C0607D501F005
:10ABD000070101EB810100EBC100283005E001EB2A
:10ABE000810100EBC10000F5B47099B232B10122CD
:10ABF00002730181190C4181002010BD00220273F3
:10AC0000C180F9E7704701EB810200EBC202D0F886
:10AC1000E802D26B04F023BB01EB810200EBC2021D
:10AC2000D0F8E802D2F87C2104F07CBB70B5044671
:10AC30000B0601F0070000EB800104EBC1014FF0AF
:10AC400001024FF0000503D581F82920283103E0E7
:10AC500081F8695101F5B471087094F8A8020128CF
:10AC600008D084F8A822206804F0A1FF84F8A85234
:10AC7000002070BD022070BD70B5044601F00F00C9
:10AC80006268904201D9012070BD0B0601F00700F7
:10AC900000EB800104EBC1014FF001024FF0000511
:10ACA00003D581F82920283103E081F8695101F5A5
:10ACB000B4718D70087094F8A802012808D084F847
:10ACC000A822206805F011F884F8A852002070BD71
:10ACD000022070BD2DE9F05F046857040B788D6980
:10ACE000B4F850704FF000064BF68F7948F2800AA6
:10ACF00048F68F7B48F2C00E4FF480682AD54FF09B
:10AD0000020C0CEBC30C674408EB4707E45BC4F38D
:10AD10000904A54203D32D1B8D6101D00BE08E6188
:10AD2000056835F8236006EA090686F4005646EA07
:10AD30000A0625F82360520609D50A78036833F815
:10AD4000225005EA0B0545EA0E0523F8225084B38C
:10AD50000A8929E04FF0060C0CEBC30C674408EBA2
:10AD60004707E45BC4F30904A54203D32D1B8D619F
:10AD700001D00BE08E61056835F8236006EA09060C
:10AD800086F4005646EA0A0625F82360520609D4DE
:10AD90000B78026832F8235005EA0B0545EA0E05E8
:10ADA00022F823502CB14A8949690068234605F0EE
:10ADB0008EFA2046BDE8F09F2DE9F05F0546006859
:10ADC0000C465FEA426C8B6916460978B0F850C0B1
:10ADD0004FF0000248F68F774CF280094FF6FF7B68
:10ADE0004FF4004E4FF4806A6CD54FF0020808EB28
:10ADF000C108E0440AEB480C30F80C00C0F309002D
:10AE0000834211D91B1AA3610FD0730407D52B6895
:10AE100033F821603E4046EA090623F8216094F8A1
:10AE20002410012907D0C5E0A2612846FFF7EBFEF8
:10AE300070046CD4BEE0616901446161E169014460
:10AE4000E1612369216A994203D31846091A2162F4
:10AE500004E084F8242009B108462262617811B127
:10AE6000012923D02BE02968B1F850201144227821
:10AE700001EB021101F2044148B13E280FD842080B
:10AE8000C30700D0521C0BEA82220A8017E00A880E
:10AE900022F4F8420A800A8842F40042F5E74209A7
:10AEA000C30600D1521E4EEA8222EEE72968B1F8AD
:10AEB00050201144227801EB0211A1F8040483B25E
:10AEC000228973E04FF0060808EBC108E0440AEB62
:10AED000480C30F80C00C0F30900834211D31B1A50
:10AEE000A3610FD0730407D42B6833F821603E4070
:10AEF00046EA090623F8216094F82410012910D0AD
:10AF000058E0A2612846FFF77EFE700452D42178F3
:10AF1000286830F821203A4042EA090220F821202E
:10AF200048E0616901446161E1690144E1612369CB
:10AF3000216A994203D31846091A216204E009B133
:10AF40000846226284F824206278296812B1012A16
:10AF500022D029E0B1F850201144227801EB0211EF
:10AF600001F20C4148B13E280FD84208C30700D077
:10AF7000521C0BEA82220A8016E00A8822F4F84268
:10AF80000A800A8842F40042F5E74209C30600D16C
:10AF9000521E4EEA8222EEE7B1F850201144227888
:10AFA00001EB0211A1F80C04628983B2616928687F
:10AFB00005F0AAF92178286830F8212048F6BF73F7
:10AFC0001A4082F0300248F280031A4320F8212010
:10AFD0000020BDE8F09F01F0070101EB810100EBCB
:10AFE000C100D0F8840170472DE9F04104460F06F6
:10AFF00001F0070000EB800104EBC1014FF00106F6
:10B000004FF0000503D581F82960283103E081F86D
:10B01000695101F5B47108700A61CB704A7802B1C8
:10B02000C881022B00D10D7194F8A802012809D023
:10B0300084F8A862206804F07FFC284684F8A852AF
:10B04000BDE8F0810220FBE770B50D4601F0070472
:10B0500004EB840100EBC101C1E95F230022C1F8C8
:10B06000842181F8692181F8684101F5B4716A078A
:10B07000006804F08DFE002070BD70B504460D46DA
:10B0800001F007006168884201D9012070BD2906DE
:10B090004FF000064FF0010207D500EB800104EBF2
:10B0A000C10181F82920283107E005EB850104EB77
:10B0B000C10181F8696101F5B4718A70087094F872
:10B0C000A802012807D084F8A822206804F047FECF
:10B0D000680702D006E0022070BD04F52C712068DC
:10B0E00004F001FE84F8A862002070BD70B50D4622
:10B0F00001F0070404EB840100EBC101C1E90F2357
:10B10000012281F84C208B6400234B6481F82920B4
:10B1100001F8284F6A07006804F03AFE002070BD6D
:10B120001FB50446006805F0CFF8000402D520469C
:10B1300002F078FA206805F0C7F840050CD52068C1
:10B1400030F8441F21F480610180204600F01CF992
:10B150000021204600F033F9206805F0B5F84004DE
:10B1600005D5206830F8441F21F480410180206813
:10B1700005F0AAF8800405D5206830F8441F21F4B2
:10B1800000510180206805F09FF8C00414D52068A4
:10B1900030F8401F21F004010180206830F8401F82
:10B1A00021F008010180204600F001F9206830F804
:10B1B000441F21F480510180206805F085F80005C6
:10B1C0003ED5216800206A4631F8203022F8103040
:10B1D000401CC0B20828F7D331F8400F40F00100FE
:10B1E0000880206830F8401F21F0010101802068AC
:10B1F000B0F844104905FBD530F8441F21F48061B4
:10B2000001800020236832F8101023F82010401C21
:10B21000C0B20828F6D3206830F8401F41F008017A
:10B220000180206830F8441F21F40061018020680B
:10B2300030F8401F41F004010180204600F0F4F88E
:10B24000206805F041F8800508D5206830F8441FD3
:10B2500021F400710180204600F0ADF8206805F06F
:10B2600033F8C00505D5206830F8441F21F48071FB
:10B2700001801FBD2DE9F04186B0040004D094F890
:10B28000A902002520B108E0012006B0BDE8F08148
:10B2900084F8A852204600F059F8032084F8A90247
:10B2A000206804F019FD04F1100114228846684654
:10B2B000FCF7A6FF94E80F0004F077FC0227C8BB58
:10B2C0000021206805F018F8002101260EE001EBAE
:10B2D000810004EBC00080F8296000F8281FC181BC
:10B2E000C57005614561491CC9B2856160688842C5
:10B2F000EDD8002111E001EB810004EBC00080F8E3
:10B30000695180F8681180F86B51C0F87851C0F825
:10B310007C51491CC9B2C0F8805160688842EAD8A3
:10B32000142241466846FCF76BFF94E80F0004F0D6
:10B33000CAFC10B184F8A972A6E784F8245084F8F6
:10B34000A962206804F0BDFC00209EE708B50068F3
:10B350000B49884212D10B48C16941F40001C16117
:10B36000C069002200F40000009005211420FFF7BE
:10B37000E7FBBDE808401420FFF7D4BB08BD000080
:10B38000005C00400010024070B504468068012552
:10B39000022801D0FDF7C6FF2946D4F8E80204F0E0
:10B3A000A2F8D4F8E802BDE8704004F05EB8D0F826
:10B3B000E80204F082B8D0F8E80204F088B810B5CA
:10B3C000044690F8A80201280BD0012084F8A802B6
:10B3D00084F82410206804F091FF002084F8A8026B
:10B3E00010BD022010BDD0F8E82200F52C711046E7
:10B3F00004F085B810B5044690F8A802012810D0D2
:10B40000012084F8A802206804F027FF01212046CB
:10B41000FFF7F8FB206804F052FC002084F8A80233
:10B4200010BD022010BD000010B50446D0F8E8029F
:10B4300004F0A4F8A069002804D00348016841F092
:10B440000601016010BD000010ED00E02DE9F84399
:10B4500004460078344FC00752D0F8690025C00078
:10B4600008D4F86940F08050F861F869012500F0CF
:10B47000805000902D480168C90511D401688046AC
:10B4800041F480710160FFF7A1FA064604E0FFF77E
:10B490009DFA801B642822D8D8F80000C005F6D594
:10B4A000386A10F4407020D0A18801F440718142C4
:10B4B0001BD0386A1E49012220F440700A60002225
:10B4C0000A603862C00710D0FFF780FA064641F2E2
:10B4D000883807E0FFF77AFA811B414502D903203B
:10B4E000BDE8F883386A8007F4D5386A616820F4CB
:10B4F0004070084338621DB1F86920F08050F8614F
:10B500002078800705D57868A16820F4404008437A
:10B5100078602078C00605D57868E16820F480005E
:10B52000084378600020DBE7001002400070004014
:10B53000400442422DE9F0470D46040067D0DFF891
:10B540001881D8F8000000F00700A8420CD2D8F803
:10B55000001021F007012943C8F80010D8F80000B6
:10B5600000F00700A84252D120683C4E810712D556
:10B57000400703D5706840F4E060706020780007F1
:10B5800003D5706840F4605070607068A16820F066
:10B59000F000084370602078C00727D06068012859
:10B5A00010D03168022810D0890700292FDA71687D
:10B5B00021F0030101437160FFF708FA074641F2E9
:10B5C00088390CE031688903EFE78901EDE7FFF77F
:10B5D000FDF9C11B494502D90320BDE8F087706819
:10B5E000616800F00C00B0EB810FF0D1D8F80010CA
:10B5F000404601F00701A9420BD9016821F007017B
:10B6000029430160006800F00700A84201D0012032
:10B61000E3E72078400705D57068E16820F4E06032
:10B62000084370602078000706D57068216920F40F
:10B63000605040EAC100706000F058F87168084A34
:10B64000C1F30311515CC840064908600648006810
:10B65000FFF70AFA0020C0E7002002400010024075
:10B66000942B0108E0000020D80000200F22026087
:10B670000C4A536803F003034360536803F0F0037C
:10B680008360536803F4E063C36052684FF4E0637F
:10B6900003EAD20202610448006800F00700086073
:10B6A0007047000000100240002002400448054995
:10B6B00000684968044AC1F30221515CC8407047E0
:10B6C000E000002000100240A42B010804480549B6
:10B6D00000684968044AC1F3C221515CC840704700
:10B6E000E000002000100240A42B010812A085B049
:10B6F0000FC88DE80F0014A0144B0068049059681F
:10B70000134801F00C02042A10D0082A0ED1C1F30C
:10B710008342C9031DF802000AD5596804AAC1F37F
:10B720004041515C0A4A5043B0FBF1F005B070470C
:10B7300008494843FAE70000020304050607080920
:10B740000A0B0C0D0E0F1010010200000010024039
:10B7500000127A0000093D002DE9F84F04006FD077
:10B760002078BE4DC00747D06868C0F3810001282B
:10B7700007D06868C0F38100022809D16868C00357
:10B7800006D52868800337D560680028E7D033E005
:10B790006068B0F5803F0BD010B1B0F5A02F11D08C
:10B7A000286820F480302860286820F4802002E097
:10B7B000286840F480302860606888B1FFF706F997
:10B7C000064609E0286840F480202860F0E7FFF78B
:10B7D000FDF8801B642873D828688003F7D50BE038
:10B7E000FFF7F4F8064604E0FFF7F0F8801B642842
:10B7F000F1D828688003F7D42078DFF864828007C6
:10B800004FF0010A4FF0000939D5686810F00C0FAD
:10B8100007D06868C0F38100022809D16868C003B6
:10B8200006D42868800714D52069012808D110E0C3
:10B830002069B0B1C8F800A0FFF7C8F8064605E0D7
:10B8400007E1FFF7C3F8801B0228C4D828688007E7
:10B85000F7D52868616920F0F80040EAC100286047
:10B860000DE0C8F80090FFF7B1F8064604E0FFF7D6
:10B87000ADF8801B022823D828688007F7D42078E9
:10B8800000072CD57748A169D9B1C0F800A0FFF70F
:10B890009DF8064604E0FFF799F8801B02280FD8B0
:10B8A000686A8007F7D570484FF4FA510068B0FB1A
:10B8B000F1F0009000BF0098411E0091FAD20EE016
:10B8C0007CE0C0F80090FFF781F8064604E0FFF73F
:10B8D0007DF8801B022871D8686A8007F7D4207829
:10B8E00040075BD5E8690027C00008D4E86940F04C
:10B8F0008050E861E869012700F0805000905B48C3
:10B900000168C90511D40168834641F48071016062
:10B91000FFF75CF8064604E0FFF758F8801B642840
:10B920004CD8DBF80000C005F6D5E06801280AD045
:10B9300008B1052813D0286A20F001002862286A7F
:10B9400020F0040002E0286A40F001002862E0686C
:10B9500041F2883B88B1FFF739F8064609E0286ACA
:10B9600040F004002862EEE7FFF730F8811B5945EC
:10B970005BD8286A8007F7D50BE0FFF727F8064663
:10B9800004E0FFF723F8811B59454ED8286A800749
:10B99000F7D41FB1E86920F08050E861E069A8B3EE
:10B9A0006968C1F38101022946D00228484606D0C1
:10B9B000C8F86000FFF70AF8044639E035E047466A
:10B9C000C8F86000FFF702F8064604E0FEF7FEFF45
:10B9D000801B022829D828688001F7D4206AB0F596
:10B9E000803F05D16868A16820F400300843686092
:10B9F000D4E908010843696821F4741108436860B8
:10BA0000C7F860A0FEF7E2FF044605E023E0FEF77A
:10BA1000DDFF001B022808D828688001F7D51AE04E
:10BA2000FEF7D4FF001B022802D90320BDE8F88FDF
:10BA300028688001F4D40EE00128F7D06868226AF3
:10BA400000F48031914204D1616A00F470108842A0
:10BA500001D00120EAE70020E8E7000000100240E2
:10BA60000000424280044242E0000020007000409A
:10BA700070B5040009D0606A002540B12561656198
:10BA8000A56294F8510040B10CE0012070BD6068DF
:10BA9000B0F5827FF4D0E561F2E784F8505020469B
:10BAA00000F040F8022084F851002068016821F07D
:10BAB00040010160A088218900F4827001F40441F2
:10BAC0000843A18901F400610843217C01F00201CF
:10BAD0000843217D01F001010843218B01F400712D
:10BAE0000843217F01F03801084394F8201001F049
:10BAF00080010843218D01F400510843216808604A
:10BB0000A069042101EA1040216848602068C169E9
:10BB100021F40061C1616565012084F851000020B5
:10BB200070BD000030B585B00024009401940294EB
:10BB3000039400681549884225D11548C16941F42C
:10BB40008041C161C16901F480410491816941F082
:10BB50000801816180690F4D00F0080004904FF4E6
:10BB6000204000900220019003200390694628465F
:10BB7000FEF73CFE4FF48040CDE9000469462846BC
:10BB80000294FEF733FE05B030BD000000380040DF
:10BB900000100240000C01402DE9F84F04464068B7
:10BBA00000261D46904689464FF0040BB0F5827F73
:10BBB00001D1A06888B194F85000012817D0012065
:10BBC00084F85000FEF702FF074694F851004FF04A
:10BBD000000A01280DD002267EE084F851B00093BF
:10BBE00013460A46204600F036F9BDE8F88F0220D9
:10BBF000FBE7B9F1000F6ED0B8F1000F6BD084F8FD
:10BC000051B0C4F854A0C4F83890A4F83C80A4F80B
:10BC10003E80C4F830A0A4F834A0A4F836A0C4F83C
:10BC200040A0C4F844A0A068B0F5004F09D1206836
:10BC3000016821F0400101602068016821F4804121
:10BC4000016020680168490603D4016841F04001A1
:10BC50000160E068B8B131E020688168C90709D0A7
:10BC6000007BA16B0870A06B401CA063E08F401E9E
:10BC7000E08708E0FEF7AAFEC01BA84202D3681CBA
:10BC800001D031E07DB3E08F0028E5D119E02068D4
:10BC90008168C90709D0C068A16B0880A06B801CAF
:10BCA000A063E08F401EE08708E0FEF78FFEC01B18
:10BCB000A84202D3681C01D016E0A5B1E08F00288D
:10BCC000E5D13A462946204602F0BAF908B12020CB
:10BCD0006065606D00B10126012084F8510084F890
:10BCE00050A0304681E7FFE70326F5E72DE9F84F3E
:10BCF000044690F8500000261D46904689460128CB
:10BD00000ED04FF0010B84F850B0FEF75FFE0746EF
:10BD100094F851004146B246012804D0022694E02E
:10BD20000220BDE8F88FB9F1000F74D0B8F1000F10
:10BD300071D0032084F85100C4F854A0C4F83090A6
:10BD4000A4F83480A4F83680C4F838A0A4F83CA045
:10BD5000A4F83EA0C4F844A0C4F840A0A068B0F580
:10BD6000004F09D12068026822F04002026020687A
:10BD7000026842F48042026020680268520603D4DE
:10BD8000026842F040020260E068B0F5006F60684F
:10BD900003D028B3012923D03FE008B101291BD1EA
:10BDA000206B21680088C86006E0206881688907E8
:10BDB00009D5216B0988C160206B801C2063E08E4F
:10BDC000401EE08608E0FEF701FEC01BA84202D339
:10BDD000681C01D030E075B3E08E0028E5D11FE08B
:10BDE000206B21680078087306E020688168890765
:10BDF00009D5216B09780173206B401C2063E08E0C
:10BE0000401EE08609E0FEF7E1FDC01BA84203D317
:10BE1000681C02D010E017E06DB1E08E0028E4D17C
:10BE20003A462946204602F039F908B120206065DB
:10BE3000A06818B106E0FFE7032606E02068C168A5
:10BE400080680090606D00B1012684F851B084F8DC
:10BE500050A0304665E72DE9F84F044690F85000B1
:10BE600001250A9E1F4692468B464FF00008012886
:10BE70000ED0012084F85000FEF7A8FD814694F80A
:10BE80005100616801280CD0B1F5827F07D102E032
:10BE90000220BDE8F88FA16809B9042801D002206A
:10BEA000B6E0BBF1000F27D0BAF1000F24D01FB3CA
:10BEB00094F85100042802D0052084F85100002095
:10BEC0006065C4F838A0E787A787C4F830B0E78674
:10BED000A7862064606420680168490603D401686D
:10BEE00041F040010160E068B0F5006F606805D086
:10BEF000E8B3012F43D079E0012089E008B1012F98
:10BF000034D1206B21680088C860206B801C2063BE
:10BF1000E08E401EE08629E02068816889070DD503
:10BF2000E18E59B1012D09D1216B0988C160206BC7
:10BF3000801C2063E08E401EE0860025206881681A
:10BF4000C9070BD0E18F49B1C068A16B0880A06B15
:10BF5000801CA063E08F401EE0870125FEF736FDC0
:10BF6000A0EB0900B04201D3701C50D100E006E004
:10BF7000E08E0028D0D1E08F0028CDD13CE0206BAE
:10BF8000216800780873206B401C2063E08E401EFF
:10BF9000E0862BE02068816889070DD5E18E59B1D4
:10BFA000012D09D1216B09780173206B401C20639E
:10BFB000E08E401EE086002520688168C9070BD00E
:10BFC000E18F49B1C068A16B0870A06B401CA063F1
:10BFD000E08F401EE0870125FEF7F8FCA0EB09008A
:10BFE000B04202D3701C01D011E086B1E08E00286F
:10BFF000D0D1E08F0028CDD14A463146204602F00C
:10C000004DF838B120204FF00108606508E00320AA
:10C01000804605E0A06818B92068C1688068009073
:10C02000012084F85100002084F85000404630E799
:10C030007047704770B590F83C20012A26D0012542
:10C0400080F83C50022280F83D20026853689468D2
:10C0500023F070060B68334353600D4B02689A421D
:10C0600008D0B2F1804F05D00A4B9A4202D00A4B59
:10C070009A4204D1496824F080031943916080F802
:10C080003D50002180F83C10084670BD022070BD74
:10C09000002C0140000400400008004010B50400DE
:10C0A00003D094F83D0010B107E0012010BD00203E
:10C0B00084F83C00204600F01FF8022084F83D0080
:10C0C000211D206802F05AFB012084F8460084F804
:10C0D0003E0084F83F0084F8400084F8410084F872
:10C0E000420084F8430084F8440084F8450084F852
:10C0F0003D00002010BD000038B504460068214A0C
:10C10000214990420ED1886940F4006088618869B5
:10C11000002200F40060009011461920FEF710FD87
:10C12000192029E0B0F1804F2AD1C86940F0010000
:10C13000C861C869164D00F00100009013482860DE
:10C140001020686000208021C5E9020149002961B2
:10C150008900C5E905108800E8612846FEF7F0F976
:10C1600008B1FDF7DFF8A5622563002211461C2007
:10C170006C62FEF7E5FC1C20BDE83840FEF7D2BC3F
:10C1800038BD0000002C0140001002408000024039
:10C19000940C002090F83D10012901D00120704737
:10C1A000022180F83D100168CA6842F00102CA60AD
:10C1B00000680B49884208D0B0F1804F05D009498A
:10C1C000884202D00849884204D1816801F0070101
:10C1D000062903D0016841F0010101600020704789
:10C1E000002C014000040040000800400168CA68BB
:10C1F00022F00102CA6001680A6A41F211131A4270
:10C2000007D10A6A9B101A4203D10A6822F0010280
:10C210000A60012180F83D100020704770B5044687
:10C2200090F83C00012817D0012584F83C500220EA
:10C2300084F83D002068826822F0770222F47F4271
:10C2400082600868502830D00DDC20284DD005DCF5
:10C2500098B310283BD148E0022070BD302844D06C
:10C26000402834D139E0602828D0702806D0B0F5B5
:10C27000805F2CD0B0F5005F29D10AE0CB68D1E90E
:10C280000121206802F032FB2068816841F07701CB
:10C2900009E0CB68D1E90121206802F027FB206882
:10C2A000816841F48041816011E0CA684968206872
:10C2B00002F0D6FB5021206807E016E0CA68496802
:10C2C000206802F0DEFB6021206802F019FB84F890
:10C2D0003D50002084F83C0070BDCA684968206861
:10C2E00002F0BEFB40212068EFE7226801461046BD
:10C2F000EBE77047704770B50446006801694FF07E
:10C300000005C943890715D4C168C943890711D4F9
:10C31000E91E01610120207720688069800720469E
:10C3200002D0FFF7E7FF04E000F0E0F8204600F05D
:10C33000DFF9257720680169C943490717D4C16827
:10C34000C943490713D46FF004010161022020772B
:10C350002068806910F4407F204602D0FFF7CAFFB2
:10C3600004E000F0C3F8204600F0C2F92577206809
:10C370000169C943090716D4C168C943090712D422
:10C380006FF008010161042020772068C0698007F0
:10C39000204602D0FFF7AEFF04E000F0A7F82046E9
:10C3A00000F0A6F9257720680169C943C90617D4AA
:10C3B000C168C943C90613D46FF010010161082098
:10C3C00020772068C06910F4407F204602D0FFF734
:10C3D00091FF04E000F08AF8204600F089F9257703
:10C3E00020680169C943C90708D1C168C943C907A1
:10C3F00004D1891E0161204600F0D6FA2068016947
:10C40000C943090609D4C168C943090605D46FF0B8
:10C41000800101612046FFF70BFE20680169C943D6
:10C42000490609D4C168C943490605D46FF04001E3
:10C430000161204600F0CAFA20680169C9438906F3
:10C440000BD4C168C943890607D46FF0200101618C
:10C450002046BDE87040FFF7ECBD70BD00B585B06B
:10C460000021009101910291039100681A49022272
:10C47000B0F1804F14D0194B98420FD1886940F029
:10C48000040088618869694600F004000490402037
:10C49000CDE9000212480392FEF7A8F905B000BDED
:10C4A000886940F0080088618869694600F00800E2
:10C4B00004904FF40060CDE900020A480392FEF7B1
:10C4C00095F90949486820F4407040F0E06040F474
:10C4D00000704860E2E700000010024000040040E5
:10C4E00000080140000C01400000014070470000BE
:10C4F00070B5044600680D0006D0042D0AD0082D42
:10C500003AD00C2D0DD13DE0C16821F40071C1601D
:10C51000606A04E0C16821F48061C160A06AFDF72F
:10C5200017FF00222946206802F05EF91D4941F2FA
:10C53000111220689310884209D1016A114206D174
:10C54000016A194203D1416C21F400414164206821
:10C55000016A114206D1016A194203D1016821F032
:10C560000101016001209DB1042D14D0082D15D0CA
:10C5700084F84100002070BDC16821F40061C160F1
:10C58000E06ACCE7C16821F48051C160206BC6E746
:10C5900084F83E00EEE784F83F00EBE784F84000C3
:10C5A000E8E70000002C014070B5044690F83C001C
:10C5B0000D4601280AD0012084F83C0042B1042A2B
:10C5C00018D0082A2AD00C2A4DD139E0022070BD9B
:10C5D000206802F09DF92068816941F008018161BD
:10C5E0002068816921F004018161206881692A69DC
:10C5F000114311E0206802F0B7F92068816941F425
:10C60000006181612068816921F480618161206815
:10C6100081692A6941EA0221816124E0206802F0EF
:10C62000D1F92068C16941F00801C1612068C16980
:10C6300021F00401C1612068C1692A69114311E038
:10C64000206802F0EBF92068C16941F40061C16122
:10C650002068C16921F48061C1612068C1692A69CB
:10C6600041EA0221C161002084F83C0070BD10B590
:10C67000040003D094F83D0010B107E0012010BD84
:10C68000002084F83C00204600F01EF8022084F8C8
:10C690003D00211D206802F071F8012084F8460059
:10C6A00084F83E0084F83F0084F8400084F841009C
:10C6B00084F8420084F8430084F8440084F845007C
:10C6C00084F83D00002010BD08B500680649884286
:10C6D00008D10648C16941F00201C161C06900F09A
:10C6E0000200009008BD000000040040001002405D
:10C6F0000349884203D10C210148FFF7F9BE704776
:10C70000040C00207047000010B5044649B104290C
:10C710000AD008290BD094F8410001280AD0012042
:10C7200010BD94F83E00F8E794F83F00F5E794F860
:10C730004000F2E7022041B3042929D008292AD079
:10C7400084F841000122206802F04EF81349206865
:10C75000884203D1426C42F400424264206888421D
:10C7600008D0B0F1804F05D00D49884202D00D4964
:10C77000884204D1816801F00701062903D00168CD
:10C7800041F001010160002010BD84F83E00D9E7AE
:10C7900084F83F00D6E784F84000D3E7002C01403E
:10C7A00000040040000800402DE9F04116460D004D
:10C7B000044611D0042D12D0082D13D094F8410056
:10C7C00002287DD08DB1042D12D0082D13D094F8FD
:10C7D0004100012812D09BE094F83E00F0E794F865
:10C7E0003F00EDE794F84000EAE794F83E00F0E7F8
:10C7F00094F83F00EDE794F84000EAE70EB9002B0B
:10C800005FD1022085B1042D11D0082D12D084F8FB
:10C81000410043484349444A7DB1042D1FD0082DAF
:10C8200057D00C2D2DD166E084F83E00F1E784F856
:10C830003F00EEE784F84000EBE7676AB862606AA1
:10C84000C162606A314602632268606A3432FDF771
:10C85000A5FEB0BB2068C16841F4007110E0A76A72
:10C86000B862A06AC162A06A314602632268A06A07
:10C870003832FDF793FE20BB2068C16841F4806127
:10C88000C16001222946206801F0AEFF27492068D7
:10C89000884203D1426C42F40042426420688842DC
:10C8A00008D0B0F1804F05D02149884202D02149FB
:10C8B000884204D1816801F00701062906D001E011
:10C8C00005E025E0016841F0010101600020BDE8BC
:10C8D000F081E76AB862E06AC162E06A31460263E9
:10C8E0002268E06A3C32FDF759FE88B92068C168C9
:10C8F00041F40061C4E7276BB862206BC162206B12
:10C90000314602632268206B4032FDF747FE08B1D2
:10C910000120DCE72068C16841F48051B0E70000E5
:10C9200003E8000861E8000899E80008002C0140CD
:10C93000000400400008004030B504460D46006881
:10C94000002201F051FF174A41F2111120688B10AB
:10C95000904209D1026A0A4206D1026A1A4203D100
:10C96000426C22F4004242642068026A0A4206D104
:10C97000016A194203D1016821F00101016001201F
:10C980003DB1042D08D0082D09D084F841000020C5
:10C9900030BD84F83E00FAE784F83F00F7E784F8FA
:10C9A0004000F4E7002C014000680349884201D1AF
:10C9B000FEF740B8704700000008004002490A68CE
:10C9C000D062C860704700004C0C00207047704770
:10C9D00070B5026804461068D168536910F00F0FF3
:10C9E00052D003F0010501F490762E435FD0C207C8
:10C9F00005D0CA0503D5E26B42F00102E2634207AB
:10CA000005D5DA0703D0E26B42F00202E263820747
:10CA100005D5DA0703D0E26B42F00402E2630207B5
:10CA200007D501F020022A4303D0E26B42F008024E
:10CA3000E263E26B002A33D0800604D5880602D573
:10CA4000204602F0B3F820684069E16BC0F3801023
:10CA5000090700D428B3204602F091F82068416904
:10CA600049061AD5416921F040014161606BA0B1CE
:10CA70002D494163606BFDF76BFC002810D0606BA3
:10CA8000416BBDE870400847830610D58B060ED574
:10CA90002046BDE8704002F089B82046FFF797FFB6
:10CAA00070BD2046FFF793FF0020E06370BD0306D2
:10CAB0002BD50B0629D594F839002128F6D1A0688A
:10CAC000B0F5805F01D12069B0B1206A411C2162BC
:10CAD000216800784860E08C401E0004000CE0846F
:10CAE000E4D12068C16821F08001C1602068C1687C
:10CAF00041F04001C16070BD206A0088C0F30800A9
:10CB00005060206A801C2062E5E74006F3D54806A5
:10CB1000F1D5D168204621F04001D160202184F870
:10CB2000391000F035F970BDA7EA000870B50400AF
:10CB300004D094F83900002510B106E0012070BD42
:10CB400084F83850204600F023F8242084F8390077
:10CB50002068C16821F40051C160204602F06CF8E1
:10CB60002068016921F4904101612068416921F048
:10CB70002A0141612068C16841F40051C160E56348
:10CB8000202084F8390084F83A00002070BD0000AD
:10CB90002DE9F04186B000250446009501950295E7
:10CBA000039500682E49884256D12E48816941F488
:10CBB00080418161816901F480410491816941F082
:10CBC000040181618069284E00F0040004904FF454
:10CBD00000700090022001900320039069463046C7
:10CBE000FDF704FE3015CDE9000569463046029593
:10CBF000FDF7FCFD1E4E1D484FF0800801C61020B9
:10CC0000A6E82101070246F8105919487561C6E9DE
:10CC10000657FDF795FC08B1FCF784FB26637462A8
:10CC2000134E124844361430C6E90005C6E90258CE
:10CC300035617561C6E906573046FDF781FC08B1DC
:10CC4000FCF770FB66630022052125207462FDF766
:10CC500077FF2520FDF766FF06B0BDE8F0810000F4
:10CC6000003801400010024000080140440002402A
:10CC7000180D002037B5044690F83A0082B01346EC
:10CC800020283AD1039AAAB3A3B394F83800012814
:10CC900033D0012084F83800A262A3850025E56323
:10CCA000222084F83A00616B15488862616B154850
:10CCB000C862616B14480863606B45632168606BF0
:10CCC000091DFDF76BFC206801684168009184F83C
:10CCD0003850C16841F48071C1602068416941F0F9
:10CCE000010141612068416941F04001416100203A
:10CCF00005B030BDFFE70120FAE70220F8E70000A9
:10CD000001EB00083DEB0008B7EA000870477047E8
:10CD1000F7B5044690F83900202831D1019969B35C
:10CD200062B394F8380001282AD0012084F8380032
:10CD30002162A284E2840025E563212084F8390081
:10CD4000236B10489862236B0F48D862236B0F48FF
:10CD50001863206B134645632668206B321DFDF770
:10CD60001DFC21686FF04000086084F8385020688E
:10CD7000416941F0800141610020FEBD0120FEBDFE
:10CD80000220FEBD47EB000875EB0008B7EA00087B
:10CD90002DE9F041FCF7CAFF04283DD1524C534D18
:10CDA000E07A40B12878FF2805D06878FF2802D0C3
:10CDB000A878FF2830D14E4E4E494F483278FFF7C1
:10CDC00059FF4C490878EA2826D1307802230627F3
:10CDD00040280ED020281FD14879012867D002288A
:10CDE0006DD0062877D0422816D1487B32280DD145
:10CDF00058E048792022012810D002282BD006289C
:10CE000033D0422808D1487B322848D0392803D172
:10CE1000C87B302800D1E372BDE8F081E07A0628B3
:10CE200004D00228F8D1887968B106E0887920B961
:10CE3000887B2928F0D1087C09E0012801D002284C
:10CE4000EAD13270E8E7487B2928E5D1C87B6073D6
:10CE500020746870E0E788790028EED191F83800F6
:10CE60003228D9D191F83A0030E0E07A06280CD087
:10CE70000228D1D188790028DFD1487F3028CBD152
:10CE8000C87F2073E0732870C6E788790028D4D162
:10CE900091F826003028BFD191F82800F1E7887B6F
:10CEA000342802D0C87B3428B6D1E772B4E7887939
:10CEB0000028B1D1887D2928AED1087EC7E78879BE
:10CEC0000028A9D1087A3228A6D1887AA073607484
:10CED000A870A1E7FFE7887900289DD1887B3028DA
:10CEE0009AD1087CCDE70000B2450020AA040020BA
:10CEF000A9040020E8150020D80C00207047FEE7A8
:10CF0000F0B500230A24302537261F4610E0B4EB85
:10CF1000107F02D905EB107C01E006EB107C01F8D4
:10CF200013C001EB430C00015B1C8CF80170DBB2F9
:10CF30009342ECD3F0BD0000FEB5002425480094D8
:10CF400001942349029401608915816001250573CC
:10CF50000475052606614FF460214460C161FDF748
:10CF60009BF808B1FCF7DEF9CDE9004569461948A0
:10CF70000294FDF70FF808B1FCF7D4F90224CDE9CB
:10CF8000005469461348FDF705F808B1FCF7CAF9E3
:10CF90000094032469460F480194FCF7FBFF08B195
:10CFA000FCF7C0F90094042469460A480194FCF790
:10CFB000F1FF08B1FCF7B6F9CDE90046694605482E
:10CFC000FCF7E8FF002801D0FCF7ACF9FEBD00003B
:10CFD00000240140E40A0020154808B5416941F0E9
:10CFE000010141614069002200F00100009005212B
:10CFF0000B20FDF7A5FD0B20FDF794FD0022052178
:10D000000E20FDF79DFD0E20FDF78CFD0022114640
:10D010000F20FDF795FD0F20FDF784FD002205216F
:10D020001120FDF78DFDBDE808401120FDF77ABD08
:10D030000010024000B589B01C220A4902A8FBF783
:10D04000DFF8002102A803F0B7FF0749002364229C
:10D0500048600220CDE9000104A1074805F0D2FB99
:10D0600009B000BD782B0108000000205354415244
:10D07000545F5441534B00009D1701082DE9F047C0
:10D0800086B0002551480095019502950395816968
:10D0900041F010018161816901F010010491816901
:10D0A00041F020018161816901F0200104918169D1
:10D0B00041F004018161816901F0040104918169F9
:10D0C00041F0080181618069DFF8048100F0080007
:10D0D000049000224FF420414046FDF772FCDFF837
:10D0E000F49048F22007002239464846FDF769FCD3
:10D0F000012280214846FDF764FCDFF8DCA0002215
:10D1000041F208015046FDF75CFC4FF40050012449
:10D1100002268DE8710069464046FDF767FBA003D3
:10D12000CDE90005694602944046FDF75FFBE00348
:10D130008DE85100694640460396FDF757FB01AA6A
:10D14000009782E8700069464846FDF74FFB802053
:10D15000CDE90004CDE9024669464846FDF746FBA5
:10D1600040F2F730CDE90005694602945046FDF7DC
:10D170003DFBA00200901948CDE9010669465046E2
:10D18000FDF734FB20038DE831000320039069464E
:10D190005046FDF72BFB2002CDE9000569460294BD
:10D1A0004846FDF723FB08208DE87100694650468C
:10D1B000FDF71CFB002205212820FDF7C1FC2820DB
:10D1C000FDF7B0FC06B0BDE8F0870000001002409B
:10D1D0000010014000080140000C01400000111047
:10D1E000094810B5074901600221416040F6FF710E
:10D1F0008160FDF7F1FB002803D0BDE81040FCF78B
:10D2000091B810BD00300040580B0020104810B5F8
:10D210000E4901604FF48271416000218160C1605C
:10D220004FF400720161C0E905121022C0E9072124
:10D23000416281620A21C162FEF71AFC002803D014
:10D24000BDE81040FCF76EB810BD0000003800408B
:10D25000640B002010B586B0002418480094019497
:10D260000294039404941449059401604721C0E991
:10D27000011444F62061C0E903148021C0E905418E
:10D28000FEF70CFF08B1FCF74DF84FF4805000900A
:10D2900069460A48FEF7C2FF08B1FCF743F8049458
:10D2A00004A906480594FEF7C5FE002801D0FCF746
:10D2B00039F806B010BD0000002C0140BC0B002066
:10D2C00010B58EB000240794089409940A940B9426
:10D2D0001C2168460C94FAF7ACFF1D484FF08041C2
:10D2E000C0E900145921C0E9024104618461FEF7DC
:10D2F000D5FE08B1FCF716F84FF48050079007A947
:10D300001348FEF78BFF08B1FCF70CF81048FFF745
:10D31000AEF908B1FCF706F80B940BA90C480C9475
:10D32000FEF788FE08B1FBF7FDFF6020CDE90004A1
:10D3300002940C22694606480494FFF735F908B1B7
:10D34000FBF7F0FF0248FFF789F80EB010BD0000B0
:10D35000040C002010B58AB0002407941C216846F4
:10D360000894FAF766FF1548134901606321C0E984
:10D370000114C46004618461FFF779F908B1FBF717
:10D38000D1FF079407A90D480894FEF753FE08B192
:10D39000FBF7C8FF6020CDE9000402940022694633
:10D3A00006480494FFF700F908B1FBF7BBFF0348F8
:10D3B000FFF754F80AB010BD000400404C0C0020E8
:10D3C0000C4810B50A4901600B4941600021816099
:10D3D0000C22C160C0E904128161C161FFF7A6FBA4
:10D3E000002803D0BDE81040FBF79CBF10BD000033
:10D3F00000380140D80C0020801A060010B5002229
:10D400000F49104801F004FF08B1FBF78BFF0E49EC
:10D410000C4802F0D9F808B1FBF784FF0B49094822
:10D4200001F0F4FC08B1FBF77DFF064802F022F999
:10D43000002803D0BDE81040FBF774BF10BD00000A
:10D4400008000020A00D002048010020C40000209A
:10D45000FEE7000070B504461B48042200EBC40040
:10D4600006461A4900F086FE184D2888082808D874
:10D470006888012805D8A888642802D8E888C828C0
:10D4800011D92C80002068806420A880E880304674
:10D4900004220E4900F07AFE0D48042200EBC4007D
:10D4A0000A4900F073FE094904EB440030392A7838
:10D4B00001F8102001EB4000AA78427029798170B0
:10D4C000A979C17070BD000000700008B03F002055
:10D4D0000071000810B504460B48042200EBC4009C
:10D4E0000A4900F047FE094904EB4400A1F130026B
:10D4F0000B7802F8103002EB40008B7843700A7909
:10D5000082708979C17010BD00710008B03F0020A1
:10D5100030B587B00C460546FBF7F4F84FF0000233
:10D520000E4BCDE90222CDE90423642D134609D226
:10D530000B4BCDE90023134603F0B8FB2044A0F5C4
:10D54000FA7007E0074BCDE900230022044B03F0FB
:10D55000ADFB204407B080B230BD000000407F40EA
:10D56000000059400000694010B540F2DC546423CB
:10D57000A1F2DC52A14205D9424392FBF3F000F242
:10D58000DC5006E05142414391FBF3F0A0F2DC5045
:10D59000404280B210BD10B502EB4103A2EB410244
:10D5A00040F2DC54A3F5805348B1A14202D9B3F84C
:10D5B00048040DE0B2F8B80B05E080B210BDA142FE
:10D5C00004D9B3F8480400F2DC50F6E7B2F8B80B1F
:10D5D000A0F2DC504042F0E710B50024E0B2FFF7C3
:10D5E00039FF641C082CF9DB10BD28B1A1F6B83056
:10D5F000404240F2DC5281B20846704710B5002428
:10D60000E0B2FFF767FF641C082CF9DB10BD40F2A5
:10D61000DC71884203D84FF47771884200D2084603
:10D62000704770472DE9F05F04464FF0060A4FF04F
:10D63000020B4FF4806966E1B0F8441011F00F0658
:10D6400039D030F826805FEA08417DD530F82610C1
:10D6500040F68F72114041F0800120F8261006EB51
:10D66000860004EBC00595F8740105F5B475002833
:10D670006BD0E878022869D02978206830F821201A
:10D6800048F68F731A4048F2C0031A4320F821204D
:10D690002978206830F82120B0F8503052047DD528
:10D6A0000BEBC1015A1809EB4201415A8F05BF0D1E
:10D6B00075D02A89CFE0C9062ED4018848F60F72AA
:10D6C000114041F400410180206804F12805B0F8C0
:10D6D00050202B780BEBC3010A4409EB4201405A5E
:10D6E000C0F309006064E16B0844E0630021204658
:10D6F000FDF789FA94F8240000289CD0A869002836
:10D7000099D194F82400216840F08000A1F84C00E1
:10D71000002084F82400F6E0018804F5B4750A05B9
:10D7200021D5B0F850202B780AEBC3010A4409EB4D
:10D730004201405A04F52C71C0F30903EB61EA88F9
:10D74000206802F0C4FD02E09DE064E072E0206821
:10D75000018840F68F72114041F08001018020461F
:10D76000FDF741FECFE00904D5D5018840F68F7260
:10D77000114041F0800101802068B0F850202B78E2
:10D780000AEBC3010A4409EB4201405A83059B0D91
:10D79000EB6110D0696971B1EA8801E051E04FE0B6
:10D7A000206802F094FDE969686908446861002115
:10D7B0002046FDF731FA2068B0F850100844296976
:10D7C00000F20C4051B13E2910D84A08C90700D0D8
:10D7D000521C4FF6FF7101EA82210FE0018821F40B
:10D7E000F8410180018841F4004107E04A09C90677
:10D7F00000D1521E4FF4004141EA8221018020688D
:10D8000001884BF68F72114081F4405148F280023A
:10D810001143018077E02068B0F850202B780AEBA4
:10D82000C3010A4409EB4201415A8F05BF0D16D0CE
:10D83000EA8810E0424629462046FDF74BFA0746A3
:10D840000DE00AEBC1015A1809EB4201415A8F055C
:10D85000BF0D04D06A893B46696902F038FDE8696A
:10D860003844E861686938446861A86910B128697A
:10D87000B84204D929782046FDF7CEF903E02946BD
:10D88000206802F085FA5FEA08603CD506EB860066
:10D8900004EBC001206830F8262048F60F731A40C8
:10D8A00042F4004220F8262091F82B00283102286B
:10D8B00002D15FEAC85022D42068B0F850300D7809
:10D8C0000BEBC502134409EB4302805A8A69C0F38B
:10D8D000090082420CD9121A8A610BD04A690244AB
:10D8E0004A61CA691044C861206802F051FA0AE02E
:10D8F00000208861E9B22046FDF785F903E0424641
:10D900002046FDF759FA2068B0F8441009043FF5A5
:10D9100093AE0020BDE8F09F10B50024FF21002049
:10D9200000F086F8C82003F03BFBFF21042000F044
:10D930007FF8C82003F034FB641CE4B2082CEDD35C
:10D9400001490020087010BD0804002070B5114C7A
:10D950000546A07948B9618911B1491E618101E08C
:10D960000120A0710A2003F01BFBA07901280AD135
:10D970006189FF2902D2491C618101E00020A07168
:10D98000052003F00DFBA17A2846BDE8704000F0A9
:10D990004FB800000804002070B5094C0546FF2070
:10D9A000608181B2491E6181C9B2284600F040F809
:10D9B0000A2003F0F5FA60890028F2D170BD00005A
:10D9C0000804002070B5094C05460020608181B232
:10D9D000491C6181C9B2284600F02AF80A2003F0E8
:10D9E000DFFA6089FF28F2D370BD00000804002030
:10D9F00010B5FF21002000F01BF8C82003F0D0FA7A
:10DA0000FF21042000F014F8C82003F0C9FAFF2118
:10DA1000002000F00DF8C82003F0C2FAFF21042016
:10DA200000F006F8BDE81040C82003F0B9BA0000C5
:10DA300010B5FBF703FC1B4B1B4C002019780A06A2
:10DA400001D53C2200E01E2224F810204900401C91
:10DA5000C0B219700828F1D3082059780A0601D5F8
:10DA60003C2200E01E2224F810204900401CC0B2D5
:10DA700059701028F1D3102099780A0601D53C225C
:10DA800000E01E2224F810204900401CC0B299700A
:10DA90001828F1D31923BDE81040034A0C2103488C
:10DAA000FEF782BE14040020F2430020040C002084
:10DAB0002DE9F041FCF78AFF364D00244FF00106B6
:10DAC000C5E90604A978EA782B790A431A4356D0A7
:10DAD00099B1D5E90823871A64EB03010022D7F135
:10DAE00096008A4109D2AC70EE70FF210420FFF746
:10DAF0009FFFFCF76BFFC5E90A04E87818B3D5E986
:10DB00000610D5E90A238A1A60EB03009623002148
:10DB10009A1A814117D2EC70687801280CDAAE703D
:10DB2000FF210020FFF784FFFCF750FFC5E9080440
:10DB30006878401C687006E06C7027462E71FCF710
:10DB400045FFC5E90C072879002816D0D5E90C1245
:10DB5000D5E906305B1A60EB02004FF4FA7200213F
:10DB6000D21A814109D22C71AE70FF210020FFF73B
:10DB70005FFFFCF72BFFC5E90804BDE8F081AE703C
:10DB8000FCF724FFC5E90804FF210020FFF750FF40
:10DB90006C70F2E70804002070B50D4606460428B4
:10DBA0004FF0000410D912E0FF210020FFF740FFE2
:10DBB0002846FCF72BFDFF210420FFF739FF2846FC
:10DBC000FCF724FD641CE4B2B442EDD370BDFF2128
:10DBD0000620FFF72DFF2846FCF718FDFF21042043
:10DBE000FFF726FF2846FCF711FD641CE4B2032C66
:10DBF000EDD370BD10B501222849294800F0BAFACA
:10DC0000264927480122891C801C00F0B3FA2349C9
:10DC100023480122091D001D00F0ACFA1F492048CD
:10DC20000122891D801D00F0A5FA1C491C48012213
:10DC30000831083000F09EFA1849194801220A31CB
:10DC40000A3000F097FA154C15480C3C0122A11D32
:10DC50000C3000F08FFA1248012204F108010E3056
:10DC600000F088FA0E48012204F10A01103000F099
:10DC700081FA0B4801222146123000F07BFA084855
:10DC80000122A11C143000F075FA211D0448012264
:10DC9000BDE81040163000F06DBA0000C802002048
:10DCA0000078000870B52A4C0546607910B102284A
:10DCB00027D129E02089274DB0F5167F18D2401CC6
:10DCC00020812F20FBF700FC2878FBF7E3F83A20AF
:10DCD000FBF708F9FBF756FD1320FBF70DFB362089
:10DCE000FBF700F91C480178491CFBF715F908E01F
:10DCF00000202070208120712878FBF7CBF80220CB
:10DD0000607142F2283070BD207961782F22014481
:10DD1000B1FBF2F002FB101020713620FBF7E2F8A5
:10DD20000D4821793238415C2520FBF705F90A4876
:10DD300021796438415C0A20FBF7FEF82846FBF79E
:10DD4000DBFB3620FBF7CEF821210348CDE70000AE
:10DD500040040020290300208844002070B5254C91
:10DD6000064642F27E25A07920B102282DD042F24B
:10DD7000283070BD2089B0F5167F18D22F20FBF710
:10DD80005BFC6079FBF786F83A20FBF7ABF8FBF712
:10DD900065FD3620FBF7A6F83B20FBF7A3F8122120
:10DDA0001548FBF7B9F82089401C20810BE00020C2
:10DDB0002070208160706079FBF76CF82078FBF7A9
:10DDC00023FC0220A071284670BD6178BC20491C4C
:10DDD000B1FBF0F200FB12106070FBF793FC3046D1
:10DDE000FBF742FC3620FBF77DF812210248FBF7D7
:10DDF00093F8E8E76C040020144500202DE9F04773
:10DE0000314C00250226A178304F4FF4FA6840F2D9
:10DE1000E479052955D2DFE801F003091C223A0014
:10DE2000657000F0F7F80120A0700FE02520FAF7E8
:10DE3000F7FF61787854491CC8B26070322802D26A
:10DE400000F0E8F802E06570A580A6704046BDE8E5
:10DE5000F08700F043F800F0D7F8032014E000F05A
:10DE60003DF800F0D1F8607821780844801CC0B2F9
:10DE700060701D2807D91F2802D20844801C6070DA
:10DE8000C0B21F3860700420A0704846DFE7A6705B
:10DE90003620FBF727F86078102100EB400001EBFB
:10DEA0004000C1B20A20FBF747F86078395C2520B2
:10DEB000FBF742F806480078FAF7ECFF40F6C62078
:10DEC000C5E70020C3E700008804002026450020A5
:10DED000290300200120FCF799BB0000F0B5344D68
:10DEE000A978022901D0012100E00021AA880A4472
:10DEF000C2F30902AA8041F00201D20701D041F029
:10DF00000801042202EA51042A4A8388284E138019
:10DF1000C3885380438893800388D3800389138107
:10DF20004389538183899381C089D0810020224F06
:10DF300012362318FB5C32F8133026F81030401CE0
:10DF4000C0B20428F5D31B48812228380270184A31
:10DF50000C3213784370527882700022C2700271C2
:10DF600032886C78C2F3422343EAC40343715308F6
:10DF700083717388C3F3461444EAC212C271B28833
:10DF8000C2F3422444EAC303037253084372F38882
:10DF9000C3F3461444EAC21282722A78C2F382049E
:10DFA00044EAC303C37241EA82110173F0BD000069
:10DFB0008804002080450020CE30010830B5114C87
:10DFC00000210120A26890430A46A368054618462E
:10DFD0005B0865F35F00A360830702D0C3439B0720
:10DFE00005D1491CC9B2062902D980F001000021DF
:10DFF000521CD2B2102AE8D30249020A0C310A702C
:10E00000487030BD880400200D210148FAF784BF14
:10E010005845002010B53620FAF764FF0748102154
:10E02000407800EB400001EB4000C1B20A20FAF753
:10E0300083FFBDE810403320FAF754BF8804002066
:10E04000F8B5044640684FF48273984217D1A0682F
:10E050004FF48065B0F5004F01D0A8420FD1206881
:10E06000066826F0400606606068984207D1A068FE
:10E07000A84204D100920B460022012103E0009245
:10E080000B4600228021204600F018F8002804D01A
:10E09000606D40F0200060650320F8BD38B50B4688
:10E0A000009204460022802100F008F8002804D0E5
:10E0B000606D40F020006065032038BD2DE9F84315
:10E0C0001E46914688460446089DFCF77FFC401B8F
:10E0D000351AFCF77BFC074625480068C0F3CB30B7
:10E0E000684338E0701C37D0FCF770FCC01BA842B6
:10E0F00003D215B1009860B32CE02068416821F08C
:10E10000E00141606068B0F5827F0BD1A068B0F596
:10E11000004F02D0B0F5806F04D12068016821F073
:10E1200040010160A06AB0F5005F09D12068016874
:10E1300021F4005101602068016841F40051016040
:10E14000012084F85100002084F850000320BDE82D
:10E15000F8830025401E00902068816838EA01009D
:10E1600004D000204845BDD10020F0E70120F9E7A8
:10E17000E000002010B5002305E030F8024B21F844
:10E1800013405B1C9BB29342F7D310BD2DE9F05FA7
:10E19000A0F10064154688468246B4F5803F5ED201
:10E1A000FCF792FAA70AC4F34806C6F50074A54224
:10E1B00000D82C46DFF8ACB04FF0006000EB8720B1
:10E1C00081464FF400722749FFF7D4FF00204FF635
:10E1D000FF7206E033183BF81310914203D1401C44
:10E1E00080B2A042F6D3A0422DD24846FBF79CF85D
:10E1F0004CF25030FBF7E6F81B48016921F00201B0
:10E2000001610020594606E038F810208319401CAF
:10E2100021F8132080B2A042F6D348464FF4007292
:10E22000104900F023F8A54215D0281B08EB44083C
:10E230000AEB440A002685B24FF400747F1CA54205
:10E24000BAD82C46B8E74CF25030FBF7BBF8224660
:10E2500041465046E5E7BDE8F05FFCF7E9B9BDE8A7
:10E26000F09F0000803B0020002002402DE9F0419B
:10E2700016460F460546002409E037F8142000230F
:10E2800029460120FCF7DEF9641CA4B2AD1CB4429F
:10E29000F3D3BDE8F081000010B5354C012204F144
:10E2A0000C01208819382080A0881930A080E088CF
:10E2B0002838E080608928306081A0891938A081E1
:10E2C000208A19302082608A28386082E08A2830CB
:10E2D000E0822848FFF75AFF2648012204F10E0188
:10E2E000801CFFF753FF2348012204F11001001D99
:10E2F000FFF74CFF1F48012204F11201801DFFF7B8
:10E3000045FF1C48012204F114010830FFF73EFFCD
:10E310001848012204F116010A30FFF737FF1548AB
:10E320000122A11D0C30FFF731FF1248012204F138
:10E3300008010E30FFF72AFF0E48012204F10A01FE
:10E340001030FFF723FF0B48012221461230FFF760
:10E350001DFF08480122A11C1430FFF717FF211DE3
:10E3600004480122BDE810401630FFF70FBF00003F
:10E37000BC02002000780008F0B595B0544B002096
:10E3800010AC195C24F81010401C0828F9DB504828
:10E390001A78012641780025072A47D017DC4D4816
:10E3A000012A26D0052A10D120226946FFF7E2FE75
:10E3B000202269464848FFF7E9FE47480322A11C8E
:10E3C0006030FFF7E3FEFCF7EDFB15B0F0BD082A67
:10E3D00017D0112AF9D14148414A00290170987893
:10E3E0001070F2D101286FD00328EED13D4806709D
:10E3F000EBE700EBC1000422211DFFF7C7FE3A48FE
:10E40000F5E7012902D002290AD00FE0012237489E
:10E41000211DFFF7BBFE3649BDF84400088005E02A
:10E4200032480122801E211DFFF7B0FEBDF84210C8
:10E43000304801291CD0F1B10229C6D14671BDF87E
:10E440004C10012919D0BDF84E10012917D0BDF884
:10E450004410BDF84830CAB2BDF846108373C37A81
:10E4600003270224C9B2022B12D0062B19D10FE0C8
:10E47000C6710671A9E7C571A7E70672A5E74672DE
:10E48000A3E7012908D0022908D0032909D107E010
:10E490000029F6D1477304E0447302E0467300E0BC
:10E4A0004573022B03D0062B8FD102738DE7032A0D
:10E4B00005D0042A05D0052A87D1047385E70573A2
:10E4C00083E7067381E7FFE70B4805807DE70000DF
:10E4D000A81500200071000800700008A0020020AC
:10E4E000A10200206D020020280200201672000800
:10E4F000E4020020B24500201E02002010B50C4CA2
:10E50000EE220623227063702D23A370E270EA22AC
:10E5100022716071A171A01C052101F09DFFE071C5
:10E520002146BDE8104008220248FEF7F1BB00007A
:10E53000B4040020D80C002004480021018141715E
:10E54000034890F82F00FAF7BFBF000040040020F6
:10E5500024440020FEF752FF0A2002F021FDFBE7D1
:10E560002DE9F041264F012224493846FFF702FEEB
:10E57000224C02250A3C6089042805D965810122C4
:10E580001E493846FFF702FE1E4E4FF4807130469A
:10E59000FCF712FA60B96089401C80B260810428DF
:10E5A00001D900206081012214493846FFF7EEFDB1
:10E5B0004FF480411448FCF7FFF928B9A07AB42140
:10E5C000401CC0B2FFF7E8FA608901F0B1FE618932
:10E5D0000E48052910D2DFE801F00303030307000A
:10E5E00001220821256103E00122D1033046256183
:10E5F000BDE8F041FCF7E5B9BDE8F081720200200A
:10E60000607000080008014000100140000C01404B
:10E610002DE9F041204CDFF88480214DE078214E37
:10E620004FF40047012818D16089042804D1012241
:10E6300039464046FCF7C5F9022020706078012871
:10E6400002D1286803F0BAFC6078032805D130684D
:10E6500003F028FD286803F0B1FCE078C0B96089B8
:10E66000042804D1002239464046FCF7AAF90320C9
:10E6700020706078012802D1306803F09FFC607838
:10E68000022805D1286803F00DFD306803F096FCE0
:10E6900020786070BDE8F081680200200008014029
:10E6A000380200202402002010B5502080F3118889
:10E6B000BFF34F8FBFF36F8F04F012F918B1044905
:10E6C0004FF080500860002080F3118810BD0000DA
:10E6D00004ED00E030B593B028216846F9F7A9FDB4
:10E6E00014210AA8F9F7A5FD002401210F94109424
:10E6F0000804CDE9001011941294029402250491AB
:10E70000CDE907504FF4E01009906846FDF724F872
:10E710000F20CDE90A056802CDE90C4002210AA8C4
:10E720000E94FCF707FF12200F90A803CDE9110407
:10E730000FA8FCF78BFE13B030BD704710B505482D
:10E74000FDF7D9FD05490448096888470449086070
:10E7500010BD0000BC0B0020C2430020540200206A
:10E760002C2C01400148FDF7C6BD0000040C002020
:10E770000148FDF7C0BD000028160020F0B5026872
:10E78000164C174D174E4FF08047A04205D0B842A7
:10E7900003D0A84201D0B04203D122F070034A68EE
:10E7A0001A43A04205D0B84203D0A84201D0B042DB
:10E7B00003D122F44073CA681A434B6922F08002E5
:10E7C0001A4302608A68C2620A688262A04201D16A
:10E7D0000969016301214161F0BD0000002C014085
:10E7E000000400400008004010B501F01F010123A3
:10E7F000046A8B409C430462036A8A4013430362A9
:10E8000010BD10B5446A0121626A824205D12177A8
:10E810008069F8B984F83E101CE0A26A824206D1F1
:10E82000022222778069A8B984F83F1012E0E26AD8
:10E83000824206D104222277806958B984F84010B8
:10E8400008E0226B824205D108222277806908B94C
:10E8500084F841102046FDF74BFF0020207710BDC3
:10E8600010B5446A616A814201D101200DE0A16ABC
:10E87000814201D1022008E0E16A814201D10420F5
:10E8800003E0216B814201D1082020772046FDF76B
:10E8900039FF0020207710BD10B5446A0121626A5B
:10E8A000824203D1217784F83E1019E0A26A8242A5
:10E8B00004D10220207784F83F1011E0E26A8242FE
:10E8C00004D10420207784F8401009E0226B8242B2
:10E8D00004D10820207784F8411001E084F83D102D
:10E8E0002046FDF706FD0020207710BD10B5846896
:10E8F00042EA032224F47F440A432243826010BD8B
:10E90000826822F070020A4342F00701816070477A
:10E9100030B5026A22F001020262036A4268846929
:10E9200024F073050C682C4323F002058B682B43FD
:10E930000C4DA84206D123F00805CB6843EA050335
:10E9400023F0040307D14D6922F4407245EA020521
:10E950008A6942EA05024260846149684163036250
:10E9600030BD0000002C014030B5026A22F01002D8
:10E970000262026A436884690D6824F4E64444EA4A
:10E9800005248D6822F0200242EA05120C4DA842AF
:10E9900006D1CD6822F0800242EA051222F0400240
:10E9A00007D14D6923F4406343EA85038D6943EA47
:10E9B00085034360846149688163026230BD000061
:10E9C000002C014030B5026A22F480720262036AB0
:10E9D0004268C46923F4007324F073050C682C4367
:10E9E0008D6843EA05230C4DA84206D1CD6823F477
:10E9F000006343EA052323F4806307D14D6922F4C1
:10EA0000405242EA05128D6942EA05124260C46131
:10EA10004968C163036230BD002C014030B5026A11
:10EA200022F480520262036A4268C4690D6824F4C9
:10EA3000E64444EA05248D6823F4005343EA053391
:10EA4000064DA84204D14D6922F4804242EA851263
:10EA50004260C46149680164036230BD002C01401A
:10EA600010B5046A036A23F001030362836923F08B
:10EA7000F00343EA021324F00A020A4383610262AC
:10EA800010BD10B5036A23F0100303628469036AA2
:10EA900024F4704444EA023223F0A00343EA011153
:10EAA0008261016210BD10B5406A0021C185C18438
:10EAB000FDF78DFF10BD70B5446A2068406994F879
:10EAC0003910C0F3C0100025212904D118B1E58404
:10EAD000204600F062F82068406994F83A10C0F3CC
:10EAE0008010222904D118B1E585204600F047F8AE
:10EAF000E06B40F01000E0632046FDF768FF70BD5A
:10EB000010B50146406A09680968890613D40021D6
:10EB1000C1850168CA6822F48072CA6001684A69C6
:10EB200022F001024A6101684A6922F040024A610A
:10EB3000202180F83A10FEF7E9F810BD10B5406AC0
:10EB4000FEF7E5F810BD10B50146406A096809688E
:10EB500089060CD40021C18401684A6922F0800230
:10EB60004A610068C16841F04001C16010BDFEF714
:10EB70000FF910BD10B5406AFEF7C0F910BD01686D
:10EB8000CA6822F49072CA6001684A6922F00102E0
:10EB90004A61202180F83A1070470168CA6822F063
:10EBA000C002CA60202180F83910704710B590F873
:10EBB0003A10222901D0022010BD81684FF4805301
:10EBC000994201D1026922B1826A99421BD049B1AE
:10EBD0000AE00268816A5268C2F308020A80816A08
:10EBE000891C08E0016971B10168496801F07F0181
:10EBF0001170816A491C8162C18D491E0904090C8A
:10EC0000C18503D016E001684968F1E70168CA6868
:10EC100022F02002CA600168CA6822F48072CA60C9
:10EC200001684A6922F001024A61202180F83A1005
:10EC3000FEF76CF8002010BD70B50446006801694D
:10EC4000E26821F4405111430161A1682069014348
:10EC5000606901432068C26841F20C639A430A4329
:10EC6000C26020684169A26921F440711143416189
:10EC70001E492068884202D1FCF728FD01E0FCF71C
:10EC800015FD00EBC00101EB0011606864228000FB
:10EC9000B1FBF0F3B3FBF2F36FF018067343B1FB73
:10ECA000F0F5B1FBF0F605EB8305322303EB051518
:10ECB000B5FBF2F5B6FBF2F605F0F00505EB06152F
:10ECC000B1FBF0F6B1FBF0F0B0FBF2F06FF0180121
:10ECD000484306EB800003EB0010B0FBF2F0216824
:10ECE00000F00F002844886070BD0000003801402B
:10ECF0000148FDF76DBE0000D80C0020D0F8B80226
:10ED0000002180F850100846704770B50546D0F8CD
:10ED1000B842D5F8BC226178D26820789047402369
:10ED200022460121284600F097FB002070BD70B5F7
:10ED30000446812100F08AFA002501212046E5627F
:10ED400000F084FAC4F86C51D4F8B80248B1D4F891
:10ED5000BC0204F52E7480688047206800F0E7FD4F
:10ED60002560002070BD10B5D0F8B842E16C0129D3
:10ED700008D1D0F8BC0223786178C2681846904761
:10ED80000020E064002010BD0A2101800048704787
:10ED900010020020292101800048704780010020D6
:10EDA0002921018000487047AC0100202921018001
:10EDB00000487047D801002070B5044600260223A1
:10EDC0000322812100F03CFB012502230322294676
:10EDD0002046E56200F034FB5420C4F86C5100F08A
:10EDE000A7FDC4F8B80278B10546002085F85000A8
:10EDF000D4F8BC024068804740232A4601212046BF
:10EE000000F02AFB304670BD0126FBE702460220D7
:10EE1000002902D00020C2F8BC12704710B513467A
:10EE200090F89C42D0F8B822032C0BD192F85040B5
:10EE30000CB1012010BD012482F850400A46812106
:10EE400000F0A5FB002010BDF8B50022D0F8B832C4
:10EE5000ADF800200D781646144615F0600522D056
:10EE6000202D56D14A78921E0A2A52D2DFE802F0AB
:10EE700010085151515151140C05887818644BE019
:10EE8000012203F1400135E04888000A586443E05C
:10EE9000012203F144012DE00122DA64CA881946F7
:10EEA00000F064F838E04D7835B1062D0BD00A2D0E
:10EEB00023D00B2D2DD128E090F89C22032A28D1B5
:10EEC0000222694616E04B882225B5EB132F07D1A5
:10EED000CA886C2A00D96C22D0F8BC120E6808E0EF
:10EEE0002125B5EB132F04D1CA880E4E092A00D96B
:10EEF0000922314600F054F80EE090F89C22032AD3
:10EF000007D1012203F14801F4E790F89C22032A7B
:10EF100004D000F020F802242046F8BD88789864D8
:10EF2000FAE700000402002010B5D0F8B4225268BD
:10EF30009047002010BD134610B50A46002100F08E
:10EF40008BFA002010BD134610B50A46002100F0D0
:10EF50001EFB002010BD10B50446802100F0FCFA15
:10EF60002046BDE81040002100F0F6BA10B503239A
:10EF7000C0F85C21C0F89432C0F8602113460A46FC
:10EF8000002100F069FA002010BD10B50521002312
:10EF9000C0F894121A46194600F05EFA002010BD1F
:10EFA00010B50223C261C0F89432026213460A46C9
:10EFB000002100F0ECFA002010BD10B50421002360
:10EFC000C0F894121A46194600F0E1FA002010BD6C
:10EFD00010B50A46024903A000F0EAF8004810BD47
:10EFE000A8130020437573746F6D20484944204373
:10EFF0006F6E666967000000122008800048704745
:10F000002800002010B50A46024903A000F0D0F8FD
:10F01000004810BDA8130020437573746F6D20481D
:10F02000494420496E7465726661636500000000A2
:10F0300004200880004870472400002010B50A46CC
:10F04000024903A000F0B4F8004810BDA813002046
:10F0500053544D6963726F656C656374726F6E694A
:10F060006373000010B50A46024903A000F0A0F83F
:10F07000004810BDA8130020424554414650562078
:10F080004A6F79737469636B0000000010B51A2031
:10F0900008800A480168001D0468001D00680818FF
:10F0A00009D008220649FDF72BFF0549042210313B
:10F0B0002046FDF725FF0248801E10BDE8F7FF1F20
:10F0C0003E000020F8B504460020ADF80000488856
:10F0D0000D46010A082948D2DFE801F04704091764
:10F0E00047473D45D4F8B012207C0A6819E0207CDF
:10F0F00002260028D4F8B40205D0C16A68468847C1
:10F10000014646703EE0816AF8E7C0B206282CD27C
:10F11000DFE800F0030B1115191DD4F8B0024268A6
:10F1200006E06946904701462CE0D4F8B0028268B8
:10F13000DAB1207CF5E7D4F8B002C268F8E7D4F879
:10F14000B0020269F4E7D4F8B0024269F0E7D4F8FB
:10F15000B0028269ECE7207C38B9D4F8B402416B84
:10F1600068468847DFE7207C20B129462046FFF724
:10F17000F2FEF8BDD4F8B402016B68468847014638
:10F1800007204870BDF8000048B1EA8852B18242B9
:10F1900000D90246ADF800202046FFF701FFE888BD
:10F1A0000028E6D12046FFF708FFF8BD00F0FBB8C5
:10F1B00070B5002300281ED00446002502E06D1C17
:10F1C000EDB2641C2678002EF9D1022404EB45042C
:10F1D00014801278CA545B1C0322CA5400245B1C9E
:10F1E00006E0CA545B1CDAB28C54521CD3B2401CE9
:10F1F0000278002AF5D170BD01004FF0000004D064
:10F20000012901D0022901D0022070470120704756
:10F2100010B580B1D0F8B43213B10023C0F8B432C5
:10F2200009B1C0F8B012012180F89C12027000F000
:10F23000BFF8002010BD022010BD10B5D0F8C002EC
:10F24000FBF71AFDBDE81040FFF7D6BF10B5D0F8A8
:10F25000C002FBF7EBFCBDE81040FFF7CDBF2DE986
:10F26000F0411746044651B1D4F8B40242691AB1CC
:10F2700094F89C02032851D00220BDE8F081D4F814
:10F280009432002504F11400022B03D0042B3AD051
:10F29000C3B33CE0D0E903639E4207D9F11AC160D1
:10F2A0008AB239462046FFF74EFE12E08068B0FB76
:10F2B000F3F103FB110199B9984211D3D4F89812D4
:10F2C00088420DD2002211462046FFF73CFEC4F8CA
:10F2D000985200231A461946204600F0BDF816E061
:10F2E000D4F8B402C16829B194F89C02032801D172
:10F2F000204688478021204600F02EF92046FFF75F
:10F3000044FE04E0FFE78021204600F025F994F850
:10F31000A002012804D184F8A05201E020469047C1
:10F320000020AAE770B51546044649B1D4F8B402E6
:10F3300082691AB194F89C02032830D0022070BD73
:10F34000D4F8941204F5AA70032902D005291ED01E
:10F3500027E0D0E903318B420BD95B1AC360084622
:10F36000834200D303469AB229462046FFF7E3FDC5
:10F3700017E0D4F8B402016929B194F89C0203287B
:10F3800001D1204688472046FFF717FE09E00020FC
:10F390000146C4F89402204600F0DEF801E0204661
:10F3A0009047002070BDD0F8C002FBF714BE0000EB
:10F3B00010B5044618481949C0F8E842C4F8C0021C
:10F3C0000160082141600221816000218161C161E9
:10F3D0000162FBF74FFF08B1F9F7A4FF0022D4F850
:10F3E000C0021823114604F53074FBF7EDFB5823D7
:10F3F000002280212068FBF7E7FB9823002281216F
:10F400002068FBF7E1FBD823002201212068FBF7ED
:10F41000DBFB002010BD0000BC100020005C0040A1
:10F420000A0601F07F01D0F8C00201EB810100EB78
:10F43000C10002D590F82A00704790F86A01704721
:10F4400010B51C461346D0F8C0022246FBF7CCFD8F
:10F45000BDE81040FFF7D0BE10B5D0F8C002FBF7F2
:10F46000F3FDBDE81040FFF7C7BE70B500220446AB
:10F4700040231146FFF7E4FF40260125C4F86461EC
:10F480003346002280212046C4F85851FFF7D8FFA8
:10F490006662A56184F89C520020C4F89402606002
:10F4A000C4F8A402D4F8B80228B1D4F8B4020021F8
:10F4B000426820469047002070BD90F89C120429B5
:10F4C00003D190F89D1280F89C120020704710B56F
:10F4D00090F89C12032904D1D0F8B412C96901B183
:10F4E0008847002010BD01740020704710B5D0F887
:10F4F000C002FBF764FFBDE81040FFF77DBE70B5AA
:10F50000044600F52A70054600F04AF80120C4F8C8
:10F510009402B4F8AE02C4F8980294F8A82212F04B
:10F520001F000AD001280DD0022810D002F080015F
:10F53000204600F011F8002070BD2946204600F05A
:10F540009EF8F8E72946204600F0CAF9F3E7294675
:10F55000204600F01DF9EEE710B5D0F8C002FBF729
:10F560008CFDBDE81040FFF747BE10B5D0F8C002D3
:10F57000FBF740FFBDE81040FFF73EBE90F89C123D
:10F5800080F89D12042180F89C120020704710B56D
:10F59000D0F8C002FBF7AAFDBDE81040FFF72CBE73
:10F5A0000A7802704A7842708A78CB7802EB03229C
:10F5B00042800A794B7902EB032282808A79C979E9
:10F5C00002EB0121C18070470246002011B1C2F850
:10F5D000B41270470220704710B5D0F8B42202244C
:10F5E0001AB11268904700B90024204610BD0000EF
:10F5F00070B50E461E4D897804462970012931D810
:10F6000094F89C0202280BD003280FD031462046E4
:10F61000FFF7A1FC29782046BDE87040FFF784BCC5
:10F62000D9B10320616084F89C0209E071B160687F
:10F63000884212D0C1B22046FFF776FC297861607B
:10F640002046FFF7C9FF02280CD006E0022084F80C
:10F650009C0220466160FFF767FC2046BDE87040D1
:10F66000FFF7ABBC31462046BDE87040FFF773BCE6
:10F670004401002010B5FFF778FF002010BD2DE9F0
:10F68000F0410A78002712F0600208D0202A01D049
:10F69000402A70D1D0F8B422926890476DE04A7841
:10F6A000002301260A2A66D2DFE802F0405D655792
:10F6B000650805652C29FFF705FD5EE0044688888E
:10F6C000D8B9C888C8B94888802816D200F07F0504
:10F6D00094F89C02032810D084F89E5229462046B4
:10F6E000FFF704FF2046FFF768FC1DB1022084F8F5
:10F6F0009C0242E084F89C623FE020463BE0FFF73A
:10F7000077FF3AE0CA88012A35D190F89C22012A75
:10F7100004D0022A02D0032A2DD104E0012200F1F4
:10F720000801836016E00122011D13E090F89C227D
:10F73000012A03D0022A01D0032A1CD1CA88022A36
:10F7400019D1C660D0F8A41209B10321C160022208
:10F7500000F10C01FFF724FC0FE0498801290CD1CE
:10F76000C0F8A46211E090F89C22012A08D0022A75
:10F7700006D0032A04D0FFF7EEFB3846BDE8F0813F
:10F7800049880129F9D1C0F8A432FFF716FCF4E743
:10F790002DE9F0410A46044613780027097913F051
:10F7A00060000AD0202801D0402850D1D4F8B402FB
:10F7B00011468368204698478FE0C3F34110012823
:10F7C00006D05078D0B301282AD003283FD107E0D3
:10F7D000D4F8B402114683682046BDE8F0411847CA
:10F7E00094F89C02022802D0032872D10AE071B377
:10F7F00080296ED02046FFF7AFFE80212046FFF71C
:10F80000ABFE6AE0508838B931B1802904D0D08885
:10F8100010B92046FFF7A0FE2046FFF7CEFB5CE0C4
:10F8200094F89C020228E2D0032852D1508898BB59
:10F830004806F1D02046FFF700FDEDE7FFE794F81A
:10F840009C020026022803D0032842D112E040E0A7
:10F8500009B180293DD1080601F07F0000EB80004E
:10F8600004EB800101D5143101E001F5AA710222F7
:10F870000E602AE0080601F00F0000EB800004EBA8
:10F8800080000AD5806920B301F07F0000EB800082
:10F8900004EB800514350BE01FE0D0F85801C0B12F
:10F8A00001F07F0000EB800004EB800505F5AA75F0
:10F8B00041B1802906D02046FFF7B2FD10B10120EA
:10F8C000286000E02E60022229462046FFF768FBF0
:10F8D00003E011462046FFF73EFB3846BDE8F081C5
:10F8E00070B5054608780C4610F0600203D0202A57
:10F8F00001D0402A16D195F89C22012A03D0022A71
:10F9000001D0032A0ED1207901280BD8D5F8B402F2
:10F91000826828469047E188014306D12846FFF7D0
:10F920004CFB02E02846FFF716FB002070BD704735
:10F9300000487047641000202DE9F0470D7800263C
:10F9400030F8252048F68F131A40CB78002B79D059
:10F95000012B7DD0022B02D0032B76D0012648F25A
:10F960008004224320F825200A7830F8223048F617
:10F970008F773B401343234320F822300B7B48F220
:10F98000C00548F6BF724CF2800C4BF68F79E3B39A
:10F990000B789A4630F8238048F2801308EA07086B
:10F9A00048EA030820F82A80B0F8503091F8008027
:10F9B000034403EB0813B1F8088028F00108A3F80A
:10F9C0000084B0F8503091F80080034403EB081332
:10F9D000B1F80A8028F00108A3F808844B78002BBE
:10F9E0000B7830F823804FEA48487DD0B8F1000FFB
:10F9F00007DA30F8238008EA070848EA0C0820F8FC
:10FA000023800B7830F823C000E024E05FEA4C6CE0
:10FA100007D530F823C00CEA070C4CEA050C20F897
:10FA200023C0CB78012B0B7830F8235005EA020570
:10FA30007ED085F02002224320F82320AAE001E0B6
:10FA400006E002E042F4007289E742F4C06286E711
:10FA500042F4806283E74B7863B3B0F8503091F89A
:10FA600000C0034403EB0C13B1F806C02CF0010CEA
:10FA7000A3F800C40B7830F823C05FEA4C6C07D5BC
:10FA800030F823C00CEA070C4CEA050C20F823C020
:10FA9000CB78012B06D0097830F82130134083F061
:10FAA00020027CE0097830F821301340234320F80D
:10FAB000213077E0B0F850200B78024402EB0312BB
:10FAC000CB8823F00103A2F80834B0F850200B785B
:10FAD000024402EB03120B6902F20C4263B13E2BAB
:10FAE00012D85D08DB0700E02DE000D06D1C4FF65A
:10FAF000FF7303EA85230FE0138823F4F843138090
:10FB0000138843F4004307E05D09DB0600D16D1E56
:10FB10004FF4004343EA852313800A7830F82230FB
:10FB20005B0408D530F822303B4043EA0C0300E088
:10FB30002DE020F82230097830F8212002EA09026D
:10FB400082F440522BE0B8F1000F07DA30F823803E
:10FB500008EA070848EA0C0820F823800B7830F8F8
:10FB600023C05FEA4C6C07D530F823C00CEA070CC1
:10FB70004CEA050C20F823C00B7830F8235005EA36
:10FB8000090585F44055254320F823508AE725438D
:10FB900020F82350097830F8212002EA0902224394
:10FBA00020F821203046BDE8F087002070472DE97D
:10FBB000F04391F80C804C780A7848F6BF774BF602
:10FBC0008F7948F2800548F2C0064CF2800C48F666
:10FBD0008F73B8F1000F29D0002C30F822404FEA83
:10FBE000444448D0002C06DA30F822401C4044EA55
:10FBF0000C0420F822400A7830F82240640605D52B
:10FC000030F822401C40344320F822400A7830F873
:10FC100022401C4044EA0C0420F822400A7830F8C4
:10FC200022303B402B4320F8223019E0002C30F8E2
:10FC300022400CD0640605D530F822401C403443E5
:10FC400020F82240097830F821203A400DE0640481
:10FC500006D530F822401C4044EA0C0420F822402B
:10FC6000097830F8212002EA09022A4320F82120ED
:10FC70000020BDE8F083002C06DA30F822401C405A
:10FC800044EA0C0420F822400A7830F82240640646
:10FC900005D530F822401C40344320F822400A7831
:10FCA00030F822401C40344320F822400A7830F8D3
:10FCB000223003EA09032B4320F82230C2E7002058
:10FCC000704700207047012120F8401F002101806B
:10FCD000818001820846704730F8401F21F43F417F
:10FCE0000180002070470020704730B50A7BA2BB1E
:10FCF0004A7848F68F75002A0A7848F2800430F86E
:10FD0000223015D05B0607D530F822302B4048F260
:10FD1000C0052B4320F82230CA78012A1DD009786B
:10FD200030F8212048F6BF731A4082F0200211E01B
:10FD30005B0407D530F822302B404CF280052B4372
:10FD400020F82230097830F821204BF68F731A40C2
:10FD500082F44052224320F82120002030BD10B50B
:10FD60004A780978002A48F2800330F8212005D02B
:10FD700048F6BF74224082F0100204E04BF68F7404
:10FD8000224082F480521A4320F82120002010BD26
:10FD90002DE9F04F0C464A78097B05464FF00009E3
:10FDA00048F68F7A48F2800B4FF6FF774FF4004801
:10FDB000012A09D000297DD0E07802287BD00128D3
:10FDC0007AD00120BDE8F08FA6692069864200D96B
:10FDD000064681B1E17802291CD0207835F8201040
:10FDE0004906B5F85010294401EB001070D5A0F871
:10FDF0000C64628927E1B3B2E2882846616900F0A9
:10FE000083FAB5F850002178284400EB0110A0F8DF
:10FE1000046434E1216A8142207875D935F82010D4
:10FE200048F2801201EA0A01114325F82010206AE5
:10FE3000801B2062207835F820104906617876D53D
:10FE400011B1012921D027E0B5F85010294401EB68
:10FE5000001000F20C404EB13E2E0FD87108F20790
:10FE600000D0491C07EA8121018015E0018821F4B6
:10FE7000F8410180018841F40041F5E77109F2067B
:10FE800000D1491E48EA8121EEE7B5F8502051190A
:10FE900001EB0010A0F80C646289B3B228466169D6
:10FEA00000F032FA6069304460612169206A88425A
:10FEB00006D902E0ECE00BE176E1801B206202E073
:10FEC0000646C4F82090607818B1012824D02BE0B1
:10FED000B6E0B5F850002178284400EB011000F29C
:10FEE00004404EB13E2E10D87108F20700D0491CD4
:10FEF00007EA8121018017E0018821F4F84101809F
:10FF0000018841F40041F5E786E07109F20600D16D
:10FF1000491E48EA8121EDE7B5F8500021782844D0
:10FF200000EB0110A0F8046422896FE0FFE711B133
:10FF3000012921D027E0B5F85010294401EB001029
:10FF400000F204404EB13E2E0FD87108F20700D0E7
:10FF5000491C07EA8121018015E0018821F4F8415C
:10FF60000180018841F40041F5E77109F20600D1F2
:10FF7000491E48EA8121EEE7B5F85010294401EB0B
:10FF80000010A0F804642289B3B22846616900F029
:10FF9000BBF96069304460612169206A884202D9F6
:10FFA000801B206202E00646C4F82090607810B101
:10FFB000012822D029E0B5F850002178284400EB30
:10FFC000011000F20C404EB13E2E0FD87108F2071E
:10FFD00000D0491C07EA8121018016E0018821F444
:10FFE000F8410180018841F40041F5E77109F2060A
:10FFF00000D1491E48EA8121EEE7B5F850104819B2
:020000040801F1
:10000000217800EB0110A0F80C646289B3B2284695
:10001000616900F079F932E035F8202048F68F6305
:100020001A4042EA0B0225F82020B5F85000227849
:10003000284400EB02108BB2A0F804342289E6E7D2
:10004000A0F804642289B3B22846616900F05CF923
:10005000607810B1012808D011E0207835F8201020
:1000600048F2C00201EA0A0106E0207835F82010C3
:100070004CF2800201EA0A01114325F82010207891
:1000800035F8201048F6BF72114081F03001DEE0F3
:10009000A1692069814202D9091AA161B5E0084627
:1000A000C4F81890B1E0088820F4F8400880088867
:1000B00040F400400AE03E2875D84208C00700D04E
:1000C000521C07EA822001E048EA82200880B6E05C
:1000D00092B9B5F850002178284400EB011021694D
:1000E00000F2044069B13E2913D84A08C90700D07C
:1000F000521C07EA82210180607888B1012832D041
:100100003AE0018821F4F8410180018841F400417E
:10011000F1E74A09C90600D1521E48EA8221EAE7FE
:10012000B5F850002178284400EB0110216900F255
:100130000C4049B13E290FD84A08C90700D0521CCB
:1001400007EA8221018017E0018821F4F84101804B
:10015000018841F40041F5E74A09C90600D1521E61
:1001600048EA8221EEE7B5F850104819217800EBF3
:100170000110218AA0F80C14E069B0B3217835F899
:100180002100420401D5420603D444F24002104249
:1001900055D135F8210048F2C00200EA0A001043A8
:1001A00025F821004BE03CE0A1692069814202D999
:1001B000091AA16102E00846C4F818908AB9B5F896
:1001C00050102278294401EB021101F2044168B178
:1001D0003E2813D84208C30700D0521C07EA8222E7
:1001E0000A80617889B1012921D028E00A8822F4A7
:1001F000F8420A800A8842F40042F1E74209C30645
:1002000000D1521E48EA8222EAE7B5F8501022785F
:10021000294401EB021101F20C4100287FF44BAF9D
:1002200041E74209C0067FF44FAF521E4CE7B5F8D4
:1002300050205119227801EB0211A1F80C0420780A
:1002400035F820104BF68F72114081F4405141EA8D
:100250000B0125F820100020B4E50021A0F844107F
:100260004FF43F41A0F840100020704710B51448EB
:10027000FAF756FF1248006800F026F8C0051DD5B1
:100280001048018821F4E8510180018841F00801FB
:100290000180018841F004010180001D018821F4E2
:1002A00080610180018821F400610180018821F4CE
:1002B00080510180018821F48071018010BD00000F
:1002C000BC100020405C0040B0F84400704710B5FE
:1002D00000EB42005C0800F5806008D030F8042B89
:1002E00001F8012B120A01F8012B641EF6D1DA077E
:1002F00001D00088087010BD0020704711B980211E
:10030000A0F84C100020704710B55B1C00EB4200B9
:100310005B0800F5806009D011F8012B11F8014B42
:1003200042EA042220F8042B5B1EF5D110BDFEE743
:100330000149087070470000400200200907090EBB
:10034000002804DB00F1E02080F80014704700F082
:100350000F0000F1E02080F8141D704702E008C88B
:10036000121F08C1002AFAD170477047002001E02F
:1003700001C1121F002AFBD17047000008B50025FB
:100380002E4601222A492B48FDF7F4FE284FA846A5
:100390003F1F052001F012FDCDF80080002301224F
:1003A000FE21B86801F066FF0446B8880F283DD0EA
:1003B000E00601D5F8F71DFCA00601D5F8F777FB9C
:1003C000A00704D50125012E01D002203870600756
:1003D00000D50225200700D50325600602D50DB9FA
:1003E000F8F722FC200601D5F8F778FCF5B1012DCD
:1003F00004D0022D04D0032D18D106E0022100E024
:1004000003210120F8F76EFB10E0F8F78BFCC82001
:1004100000F0C6FD87F8018087F8028087F8038026
:100420004FF416710120F8F7D5FB00252E46B0E7F2
:10043000E402002016720008064931F8100040F26C
:100440000A51A0F5577000EB4000C00301EB1040CB
:1004500080B270477804002030B503460020024681
:10046000044D04E013F8014B4440521C285D8A42BD
:10047000F8D330BDAE2F0108F0B504460020034686
:100480000B4E12E014F8012B82EA102202F00F0545
:10049000120936F8155002EBC21707EB02326A4018
:1004A00082EA00205B1C80B2DBB28B42EAD3F0BD53
:1004B000AE30010808B5F9F733FC1F4D00220821C2
:1004C000E860142001F0AEFF002605F1100468601A
:1004D000E86801F073FC0020F9F792FB208001200E
:1004E000F9F78EFBA0F6B830404260800320F9F7A0
:1004F00087FBE0800220F9F783FBA0F6B83040428A
:10050000A0800122009600231146A86801F0B2FEE7
:10051000C00702D06878401C68706878401E0228C6
:1005200001D8F9F795FC044900231A461031686890
:1005300001F0E0FFCCE70000A40200202DE9F0412B
:100540000446F9F733FA264D6881F8F729FE4FF093
:10055000E0208069F7F74CFEF7F740FE2E2190FB74
:10056000F1F201FB1200401CC2B2AA7003E0491C68
:1005700001F00300E870E978501A8007F7D1C8B29B
:10058000101A800828712046F8F7ECFB012825D0C6
:10059000144E002406F132073620F8F7A3FC315D33
:1005A0000A20F8F7C9FC3320F8F79CFC0120FAF781
:1005B0002DF82520F8F734FC3855641CE4B2302CB3
:1005C000EAD32878F9F720F86879F8F763FC022075
:1005D000A8713078BDE8F041F9F72EB8BDE8F08198
:1005E0006C040020B04400202DE9F0410446F9F7E6
:1005F000DDF91F4DA860FDF7E1FC4FF0E0208069B8
:10060000F7F7F6FDF7F7EAFD1C2190FBF1F201FB8D
:1006100012002870F8F72AFC0120F9F7F7FF2046AE
:10062000F8F7A0FB134E01281AD03620F8F75AFC31
:10063000114F00242046395DF8F77EFC641CE4B2BB
:10064000272CF7D34FF4FA70F8F756FE0A210C2046
:10065000F8F772FC0120F8F729FC3078F8F71AFC5B
:100660003078F8F717FC0020A870BDE8F081000092
:100670008804002029030020DE30010892B0F9F739
:100680004FFBFE4CDFF8F883DFF8F8A3DFF8F893B0
:10069000DFF8F8B306AD00266060606801F08EFBFD
:1006A000FB4800220AA9006801F0D6FF9BF8000071
:1006B00001287DD002287CD003287BD004287AD062
:1006C000BDF82800F8F71EF80022F24BCDE902220F
:1006D000CDE90423F04BF14FCDE900233B4600F078
:1006E000E5FAADF81800BDF82A00F8F70BF800227B
:1006F000E84BCDE90222CDE90423E74BCDE9002305
:100700003B4600F0D3FAADF81A00BDF82C00F7F71D
:10071000F9FF0022DF4BCDE90222CDE90423DE4BB5
:10072000CDE900233B4600F0C1FAADF81C00BDF84E
:100730002E00F7F7E7FF0022D64BCDE90222CDE9E4
:100740000423D54BCDE900233B4600F0AFFAADF8CA
:100750001E00BDF83000F7F7D5FF0022CD4BCDE9E4
:100760000222CDE90423CC4BCDE900233B4600F027
:100770009DFAADF82000BDF83200F7F7C3FF002264
:10078000C44BCDE90222CDE90423C34BCDE90023BC
:100790003B4600F08BFAADF82200BDF83400F7F7C5
:1007A000B1FF0022BB4BCDE90222CDE9042303E0D7
:1007B0001BE040E0C7E041E1B74BCDE900233B46F9
:1007C00000F074FAADF82400BDF83600F7F79AFF90
:1007D0000022B04BCDE90222CDE90423AE4BCDE996
:1007E00000233B4600F062FA1DE098F800006FF02D
:1007F000FE0101EB0021ADF8181000EB4001A84804
:1008000000EB410030F8061DADF81A104088ADF835
:100810001C000020228815F81010401C1144218073
:100820000728F7DB88B2ADF82600102206A99D48FC
:10083000FEF7F4FA42E198F8000020B1012820D038
:1008400002282BD03AE103220EA99748FDF792FC2B
:100850000520ADF81800BDF83800BDF83A1040EAA0
:100860000120ADF81A00BDF83C00ADF81C000020D6
:10087000228815F81010401C114421800728F7DB4E
:10088000D0E78A490120C8710020228815F810108D
:10089000401C114421800728F7DBC3E760885746D6
:1008A000401C80B260809AF80B305BB199F8002050
:1008B0004946FF2A06D04A78FF2A03D099F8021049
:1008C000FF2903D142F210718842B3D340F20710DE
:1008D000ADF8180000200146022B01D0062B0BD1E9
:1008E0007A7B22B1012A04D0022A05D103E0032039
:1008F00002E0022000E00120022B02D0062B0ED1E4
:100900000CE03A7B22B1012A04D0022A07D103E08D
:10091000032104E0042102E0052100E0397B41EAE3
:100920000020ADF81A009AF80E0040EA0320ADF856
:100930001C000020228815F81010401C1144218052
:100940000728F7DB6EE766808AF80B60FF2189F8DD
:10095000001089F8011089F8021014216846F7F791
:1009600068FC012269465248FDF704FC50486F4676
:100970000122801CB91CFDF7FDFB4D480122391DE9
:10098000001DFDF7F7FB4A480122B91D801DFDF748
:10099000F1FB474801220E3002A9FDF7EBFB44486A
:1009A000012210300DF10A01FDF7E4FB0220ADF841
:1009B0000C00ADF810003E48ADF80E600122801E1C
:1009C0000DF11201FDF7D6FB5A20ADF81800BDF865
:1009D0000200C1B2BDF8000061F31F20ADF81A009B
:1009E000BDF80600C1B2BDF8040061F31F20ADF8E8
:1009F0001C00BDF80A00C1B2BDF8080061F31F2059
:100A0000ADF81E00BDF80E00C1B2BDF80C0061F3D8
:100A10001F20ADF82000BDF81000C0B2ADF82200D4
:100A2000BDF81200ADF824000020228815F810103F
:100A3000401C114421800728F7DBF3E601226946B8
:100A40001C48FDF797FB1B48012201A9801CFDF7FC
:100A500091FB0820ADF81800BDF80400C1B2BDF844
:100A6000000061F31F20ADF81A000020228815F85D
:100A70001010401C1144218007281DE01C0200209A
:100A8000A1020020B2450020AA040020A0020020FC
:100A90002C02002000FC9F4000709F4000E08E4030
:100AA000803F0020A00D002060700008A0450020BD
:100AB000027A000814720008D8DBB3E62680ECE561
:100AC000DFF870B101245C4E4FF4807A4FF4FA776E
:100AD00000250A2001F072F9307840B95146584695
:100AE000F9F76AFF18B9347001F0F4FEF06070781D
:100AF00040B902215148F9F75FFF18B9747001F04D
:100B0000E9FE3061B07848B94FF480414C48F9F7BC
:100B100053FF18B9B47001F0DDFE7061307800B396
:100B2000F078F0B9D0465146D9465846F9F744FF17
:100B3000012800D1357001F0CDFEF168401AB842AD
:100B400005D90221B06801F04FFBF47009E041467D
:100B50004846F9F731FF012803D10121B06801F0BF
:100B600043FB51465846F9F727FF012803D1F5709A
:100B700001F0B0FEF060707800B33079F0B9DFF8C2
:100B8000BC8002214046F9F717FF012800D175709B
:100B900001F0A0FE3169401AB84205D90821B068B9
:100BA00001F022FB347109E002214046F9F704FF0D
:100BB000012803D10421B06801F016FB02211F486F
:100BC000F9F7FAFE012803D1357101F083FE306197
:100BD000B07810B3707900BBDFF864904FF48048B0
:100BE00041464846F9F7E8FE012800D1B57001F00A
:100BF00071FE7169401AB84205D92021B06801F030
:100C0000F3FA747109E041464846F9F7D5FE012828
:100C100003D11021B06801F0E7FA4FF48041084891
:100C2000F9F7CAFE01287FF454AF757101F052FE46
:100C300070614EE70008014010030020000C0140E5
:100C40000010014014491348086062B6F9F7FAFE33
:100C5000FDF740FDFCF712FAFCF7BEF9FCF76CF962
:100C6000FCF778FBFCF7D2FAFCF72AFBFCF7A8FBB1
:100C7000FCF7F0FA0948FBF7B9FAFCF7B1FAF8F714
:100C800057F8F9F77FF9FDF76BFCFCF7D3F900F0A3
:100C90008EF9FEE70080000808ED00E0BC0B0020A4
:100CA00001460020842900D0C81C70472DE9F05F60
:100CB0001446DDE90C89DDE90AAB1D46F7F72DFC8A
:100CC00006460F4622462B4650465946F7F725FC66
:100CD00004460D46DDE90E0142464B46F7F71DFC82
:100CE00022462B46F7F791FC3B463246F7F71BFCB2
:100CF00042464B46F7F770FBF7F725FD80B2BDE89B
:100D0000F09F0000ADF5856D9C4D0024ADF81C44AE
:100D100001220DF21C412846FDF72CFABDF81C14E7
:100D2000491E0A2908D30420ADF81C0401220DF243
:100D30001C412846FDF72AFA0020914B64254FF408
:100D40000072A146BDF81C1401EB8104844202DD4F
:100D500023F810900AE000FB01F494FBF5F44942FB
:100D600001EB81010144214423F81010401C904202
:100D7000E8DD4FF4FF7023F81020401C9042FADDAC
:100D800040F204427F496846F7F73AFAF8F7C8FF9D
:100D90007D4C7E4D0122A060A11C2846FDF7EAF99A
:100DA0006088012806D9A4F802900122A11C2846D7
:100DB000FDF7ECF900221021142001F033FB6060F4
:100DC000FCF70AFC6E4EDFF8C8A1DFF8C8B1403E60
:100DD000A0464446D8F8080000F0F0FF207801282B
:100DE00003D1FCF70BFC84F800906B4800220DF255
:100DF0001441006801F030FC684800220DF5846160
:100E0000006801F029FC6088A0460128BDF81A049A
:100E1000ADF80A042AD0BDF81804ADF80804BDF8EE
:100E20001404ADF80404BDF81604ADF80604BDF8CA
:100E30002004ADF80C04BDF82204ADF80E04BDF892
:100E40002404ADF81004BDF82604ADF81204002502
:100E500005EB450416F81400042832D268B10128C5
:100E60000ED0022863D003280FD168E0BDF8140427
:100E7000ADF80804BDF81804D3E7BDF80A0401E092
:100E8000BDF8080406EB4401888006EB44073C4AA1
:100E9000B9887878FCF77FFBB88006EB4407B988FF
:100EA000F878FCF735FBB880BA7801461046FCF7B5
:100EB0005BFBB880FCF7ABFBB88016F81400042885
:100EC0000BD3C0B20DF2044106EB440331F810100D
:100ED00099805878FCF789FB98806D1CEDB2082D3D
:100EE000B6D3B088ADF804047089ADF80604308A32
:100EF000ADF80804F08AADF80A04B08BADF80C0424
:100F0000708CADF80E04308DADF81004F08DADF896
:100F1000120400231A460DF204414446D8F8040096
:100F200001F0E8FA9AF8061001290BD015E006EB5B
:100F30004407BDF80414B98078786A46AAE7BDF87A
:100F400006049FE79AF80700012806D100231A46F5
:100F50000DF20441606801F0CDFA9BF806100129FA
:100F60007FF437AF9BF807000128F9D100231A4618
:100F70000DF20441606801F0BDFA2AE7147200081E
:100F8000C03F0020AC2B010828020020627000083E
:100F9000B2450020A0450020A8020020D402002075
:100FA00010B500B9012000F009FF002010BD10B5F8
:100FB00001F042F8002010BD7FB50D46044641699E
:100FC000B0F9080081B1A16971B1FFF769FED4E9F8
:100FD00005128DE80700D4E900102B46226901F0C4
:100FE0003EFC039004B070BDFFF75AFE03A9CDE9A3
:100FF0000001208A2B4682B2D4E9001001F002FCE5
:10100000012801D00020EDE70398EBE72DE9F0413E
:10101000184E0F46044675693068001D00F0FEFD4D
:1010200038B9306890F82C1001208840B1698143AC
:10103000B161601C07D137B13168BDE8F0410E489D
:10104000091D00F03BBE30682C44AC42446031685E
:1010500005D2B068BDE8F041091D00F017BE706808
:10106000091D00F013FE306B844200D23463BDE8EA
:10107000F0810000E40000206C1700202DE9F04111
:10108000054600F027FE2E4E3069401C3061306866
:101090002C4F10B1F06940B32DE035603069012864
:1010A00029D1002404EB840007EB800000F0E0FD70
:1010B000641C072CF6D323488C3000F0D9FD21485E
:1010C000A03000F0D5FD1F48B43000F0D1FD1D4820
:1010D000C83000F0CDFD1B48DC3000F0C9FD1948D8
:1010E0008C3070601430B06005E03068E96AC06A26
:1010F000884200D83560F06A0121401CF062E86A3D
:10110000B26981401143B16100EB800007EB8000C0
:10111000291D00F0D3FD00F0FDFDF06900280CD082
:101120003068E96AC06A884207D207494FF08050A8
:101130000860BFF34F8FBFF36F8FBDE8F0810000F1
:10114000E40000209016002004ED00E030B4026CB2
:101150000B46002A0BD0C1681144C1604468A1420B
:1011600001D30168C16030BC1846F7F749B830BCFC
:1011700070472DE9F041856B174604460026026C46
:1011800082B1C7B1E068F7F73BF8E168206C091A53
:10119000E1602268914202D26168081AE060022F81
:1011A00016D017E02068A8B9606801F0FDFB06467C
:1011B000002060600EE0A068F7F722F8216CA068BC
:1011C0000844A0606168884204D32068A06001E000
:1011D00005B16D1E6D1CA5633046BDE8F08110B5EC
:1011E000044690F8510058B101280CD002280FD0C5
:1011F000502080F31188BFF34F8FBFF36F8FFEE74E
:10120000206B00F09BFD2046BDE8104000F096BD2D
:1012100010BD000010484FF41051420706D0C01D09
:101220000D4920F00700411AC1F510510B4A002367
:101230000144C2E900030839103A21F007011160A6
:101240004B600B600B1AC0E9001393604FF0004035
:101250005360D060704700008017002030010020EC
:10126000134E144DA6F1C8074FF08058DFF8489090
:1012700011E000F02FFDF068C468201D00F0CEFCE6
:101280002869401E2861E868401EE86000F042FDC1
:101290002046FFF7A4FFE8680028EAD13868012853
:1012A000F9D9C9F80080BFF34F8FBFF36F8FF2E712
:1012B00058170020E400002004ED00E003460098E9
:1012C00029B10260C0E90F31012101F0CFB80060FF
:1012D000F8E72DE9F0470E46DDE909841746824616
:1012E00091009946089DA522206BF6F79BFF6FF0B1
:1012F0000301206B01EB8701084420F00707780702
:1013000007D0502080F31188BFF34F8FBFF36F8F4A
:10131000FEE72218315C82F83410315C11B1401CB8
:101320001028F6D3002684F84360072D00D3062545
:10133000E562C4E91156201D00F0A5FC04F1180077
:1013400000F0A1FC2461C5F107006462A061E664BD
:1013500084F850604A465146384600F027F920602C
:10136000B8F1000F01D0C8F80040BDE8F0870000D8
:1013700030B5114900E011460A688242FBD34B6840
:101380005C18844203D140681844486008464368AA
:101390001C18944209D1084C103C2468A24209D080
:1013A00052681A4442600A6812680260814200D0A2
:1013B000086030BD0460F9E73001002010B5044634
:1013C00000F088FCA06B20B1002400F0A3FC2046B4
:1013D00010BD0124F9E7000006484168096829B1F9
:1013E0004168C968C9684968016370474FF0FF31B7
:1013F000FAE70000E400002008484068401C4FF075
:10140000500080F3118804D0BFF34F8FBFF36F8F6C
:10141000FEE7BFF34F8FBFF36F8FFEE73801002069
:10142000002150B10A4B42699A420FD1806AA3F160
:10143000280290420AD040B108E0502080F3118881
:10144000BFF34F8FBFF36F8FFEE701210846704750
:101450006C1700200346002012B1994302D0704758
:101460000B42FCD0012070472DE9F041044600F00A
:1014700031FC94F9455004F1240609E0606A48B152
:10148000304601F0DDFA08B100F01CFD6D1E6DB2B2
:10149000002DF3DC4FF0FF3684F8456000F03AFC95
:1014A00000F018FC94F9445004F1100709E0206999
:1014B00048B1384601F0C4FA08B100F003FD6D1ED2
:1014C0006DB2002DF3DC84F84460BDE8F04100F01B
:1014D00021BC00002DE9F0410546002600F040FE49
:1014E000314F386808B9FFF795FEF86805424BD1CF
:1014F000C5B3083568070ED005F00700C0F1080035
:101500000544680707D0502080F31188BFF34F8F40
:10151000BFF36F8FFEE72DB37868854234D8224938
:1015200010310846046801E0214604466068A8427C
:1015300002D220680028F7D13868844224D00E688F
:101540002068086060680836411B10290FD96019AF
:10155000420708D0502080F31188BFF34F8FBFF3AC
:101560006F8FFEE710E041606560FFF701FF616883
:101570007868401A7860BA68904200D2B860F8681B
:1015800001430020C4E9000101F094FA700707D07C
:10159000502080F31188BFF34F8FBFF36F8FFEE7AA
:1015A0003046BDE8F08100002001002010B5031F87
:1015B0004FF080741C601B1F21F001011960191F7E
:1015C000024B0B60143940380A6010BDF913010852
:1015D00008B5F8F7A5FB254C254D264EA0602078D0
:1015E0002549264F264B42F2283205281FD2DFE834
:1015F00000F0030308101800C4E90571C4E903569C
:1016000005E0204DE560A1611F4D204906E01A600C
:101610000DE01F4DE560A1611E4D1F49C4E9045155
:10162000F5E71E49E1601E49A1611E492161E1689B
:1016300088471D4E0025A06800F0C0FB00221B4912
:10164000306801F009F80122009500231146606816
:1016500000F010FEC00701D020698047A16913483F
:101660008847F9F7B3F9C4E90805E4E74002002028
:101670001994000839E50008F58D0008A5DC00087C
:101680002C2C01403D050108819200085DDD000819
:10169000E9050108D5DE0008FDDD0008C58F00085A
:1016A000CD8F0008199100082C020020E243002091
:1016B000364D08B50127EF710026012000F07EFBB2
:1016C000009600230122FF21286900F0D3FD044683
:1016D000400604D50020FCF775F924F0200420060C
:1016E00004D50220FCF758F924F00804A00701D51E
:1016F000FCF77EF9E00702D02F70FCF70DF96007C8
:1017000001D5FCF7D5F920071CD52878D0B9E879A0
:1017100050B1F7F779FDE871FF210020FCF788F957
:101720001B48FAF763FD0DE0FF210220FCF780F96A
:10173000F8F702FB032805D8687918B96F711448C7
:10174000FAF728FDE00603D5FF210320FCF770F926
:10175000A006B2D50F48007820B1FF210620FCF783
:1017600067F9AAE701210C48F9F726F950B1288951
:10177000401C80B22881B0F5FA7F9ED90120FCF789
:10178000E5F89AE72E810020F9E700000804002020
:10179000BC0B00206D020020000C01401CB5002590
:1017A000DFF8F880DFF8F890DFF8F8A0DFF8F8B09D
:1017B00003243E4E3E4F00F009FDC8F8000000F043
:1017C00005FDC9F8000000F001FDCAF8000000F0B6
:1017D000FDFCCBF8000000F0F9FC3649086000F091
:1017E00079FA0023502234A13548CDE9004501F0B3
:1017F00009F8CDE9004600234FF4807231A1354845
:1018000001F000F80023642233A13548CDE90045FA
:1018100000F0F8FF0023802232A13348CDE90045D3
:1018200000F0F0FF0120CDE90005002340222FA1A8
:10183000304800F0E7FFCDE90047002380222EA1C9
:10184000304800F0DFFF0220CDE9000500236422CC
:101850002DA1304800F0D6FF2F480023CDE90040ED
:101860004FF416722DA12F4800F0CCFF0023502218
:101870002DA13048CDE9004500F0C4FF386800F0E4
:1018800011FC306800F00EFC2B48006800F0BCFA38
:1018900000F040FA0120FFF783FB8CE718030020DB
:1018A000E802002018040020440200203802002032
:1018B00024020020AC020020535441545553000030
:1018C0003D190108444154415F50524F4345535321
:1018D00000000000D115010847494D42414C00006D
:1018E000B504010852474200B116010842555A5A40
:1018F000455200007D0301084A4F59535449434B58
:10190000000000007D0601085357495443484553E1
:1019100000000000D11B0108340200204D49584549
:1019200053000000050D0108425554544F4E5F53BB
:1019300043414E00C10A01080000002008B5DFF84D
:1019400060A2DFF860B2984DDFF8609201264FF098
:101950000008012000F032FA0320F8F751F8944C07
:1019600040F2DC57B842E0814FF004000AD9F8F7A2
:1019700047F8E1896E22A1F2DC51514391FBF7F166
:10198000401A0AE0F8F73CF8E1896FF06D02A1F225
:10199000DC51514391FBF7F10844A081E38822898F
:1019A000217980B2F7F7F2FB2071E17801291CD18F
:1019B000D8B9F9F70BF8C4E90A08D4E90C23821A5C
:1019C00068EB030144F6206300209A1A88410CD288
:1019D0004021DAF8000000F007FC0221286800F03E
:1019E00003FCD4E90A01C4E90C01607810B10128B4
:1019F00006D007E040F6B830FFF7D2FA667001E093
:101A0000FCF706FE607998B1F8F7E0FFC4E9060834
:101A1000D4E90823871A68EB03024FF47A7C002389
:101A2000BCEB07074146934100D26171C4E908014C
:101A30006048CDF80080002301222521006800F0D5
:101A400019FC0746800624D5E07880B184F803802D
:101A50002021DAF8000000F0C7FB8021286800F0A0
:101A6000C3FB4FF49660FFF79BFA00220AE0E67092
:101A70001021DAF8000000F0B7FB4021286800F0E0
:101A8000B3FB01224FF400414B48F8F79AFFFCF7F3
:101A9000BFFDF80709D02078032806D04748012168
:101AA000006800F0A1FB0220A07078070BD5207819
:101AB000032808D00121DBF8000000F095FB207816
:101AC000022800D1A6700123CDF8008047461A46AF
:101AD0000221DBF8000000F0CDFB800700D5A770E5
:101AE000207801283FF435AF022812D003287FF474
:101AF00030AF4FF480413048F8F75EFF18B1202135
:101B0000286800F071FB2E4CA079A8B101281FD0E5
:101B100028E0A07848B1012809D00228E7D10121A6
:101B2000286800F061FBA77013E7082100E004219A
:101B3000286800F059FB0CE7E079012812D1D9F8A8
:101B4000000000F03BFA1F48FAF724FBA67109E0F9
:101B5000E07938B9D9F8000000F0A4FA1948FAF78A
:101B600045FBA771184CA07980B10128DCD1E07940
:101B70000028D9D1D9F8000000F094FAA77100220A
:101B80004FF400411148F8F71CFFE2E6E079012824
:101B9000CAD1D9F8000000F011FAA6710122EFE7CE
:101BA000E8020020AC0200201804002038020020C7
:101BB00068020020180300200010014044020020A9
:101BC000A0450020BC0B0020B245002000080140C9
:101BD00000220821142000F025FC0F4D2C1D286048
:101BE0000A2000F0EBF80020F8F7ACF82080012084
:101BF000F8F7A8F860800220F8F7A4F8A080032086
:101C0000F8F7A0F80449E08000231A46091D286867
:101C100000F070FCE4E70000D4020020D0E90132BB
:101C200001699A60D0E901235A604A68824201D171
:101C300082684A60002202610868401E08600868E5
:101C400070470000044908680A688069D26A096818
:101C5000C2F107028A617047E4000020034B036071
:101C600003F1540008608020106070476407002072
:101C700000F108014FF0FF32C0E90112C1600161BB
:101C800000210160704700210161704730B50C6888
:101C9000621C02D000F1080202E0026904E01A4668
:101CA00053681D68A542FAD953684B6099608A60F1
:101CB000516008610168491C016030BD42684A609A
:101CC00093688B6093685960916008610168491C52
:101CD00001607047502080F31188BFF34F8FBFF32E
:101CE0006F8F0A494868401C486001280CD1084899
:101CF000006810F0FF0F07D0502080F31188BFF369
:101D00004F8FBFF36F8FFEE7704700003801002050
:101D100004ED00E00849486828B1401E486001D140
:101D200080F311887047502080F31188BFF34F8FE4
:101D3000BFF36F8FFEE700003801002070B5002868
:101D400027D0144DA0F108046068E968084207D163
:101D5000502080F31188BFF34F8FBFF36F8FFEE7E2
:101D600022683AB1502080F31188BFF34F8FBFF340
:101D70006F8FFEE78843606000F0F2F96068696881
:101D8000084468602046FFF7F3FABDE8704000F0B1
:101D900091BE70BD200100204FF0E02000210161C4
:101DA000816105494FF47A720968B1FBF2F1491E6D
:101DB0004161072101617047E000002010B5020079
:101DC00014D00F48806B38B1502080F31188BFF3D6
:101DD0004F8FBFF36F8FFEE700F0C2F9002110466E
:101DE000FFF714F900F066FE002807D105494FF00F
:101DF00080500860BFF34F8FBFF36F8F10BD00009E
:101E0000E400002004ED00E070B50446FFF762FF37
:101E1000254D04B92C68201DFFF700FF58B9E06A72
:101E2000224A00EB800152F8211021B901218140A2
:101E3000A8698843A861A06A18B104F11800FFF7E7
:101E4000EDFEE86A401CE8622868844208D1174821
:101E5000211DC830FFF732FFE868401CE86007E04A
:101E60002869401E28612046FFF7B9F9FFF7B4FA48
:101E7000FFF750FFE869002814D02868844211D188
:101E8000A86B38B1502080F31188BFF34F8FBFF398
:101E90006F8FFEE706494FF080500860BFF34F8F09
:101EA000BFF36F8F70BD0000E4000020901600208B
:101EB00004ED00E002498A6A0260496941607047A6
:101EC000E40000200149012048627047E40000203E
:101ED00010B50C4650B1094909681831FFF7D6FE14
:101EE0002046BDE810400121FFF790B8502080F354
:101EF0001188BFF34F8FBFF36F8FFEE7E400002020
:101F000010B5144680B1104B9A6BAAB11A6841F013
:101F10000041916119681831FFF7D0FE2046BDE8F5
:101F200010400121FFF772B8502080F31188BFF3F1
:101F30004F8FBFF36F8FFEE7502080F31188BFF300
:101F40004F8FBFF36F8FFEE7E400002070B5194D8F
:101F5000AA6BFAB141F000410160C46814B3FFF705
:101F60005DFE201DFFF75AFEE06A0126AA6906FA07
:101F700000F11143A961104900EB800001EB8000E2
:101F8000211DFFF79BFEE06A2968C96A884200D9D3
:101F90006E6270BD502080F31188BFF34F8FBFF386
:101FA0006F8FFEE7502080F31188BFF34F8FBFF390
:101FB0006F8FFEE7E40000209016002070B504004B
:101FC0002BD01A4D286884422FD0FFF783FE20467D
:101FD000FFF726FAE8B1201DFFF720FEE06A012195
:101FE000AA6981401143A961114900EB800001EB0E
:101FF0008000211DFFF762FEE06A2968C96A8842F5
:1020000007D30C494FF080500860BFF34F8FBFF3E8
:102010006F8FBDE87040FFF77DBE502080F31188C0
:10202000BFF34F8FBFF36F8FFEE770BDE40000205A
:102030009016002004ED00E010B586B00024039453
:1020400005AA04A903A80494FFF708FEDDE903012B
:102050000094CDE9011000230EA11048059A00F06C
:10206000FEFB0F490028486311D0502080F31188EF
:10207000BFF34F8FBFF36F8F4FF0FF300863012026
:10208000C8614C6106B0BDE8104000F077B906B0F9
:1020900010BD000049444C450000000061120108D9
:1020A000E400002070B50446FFF714FE294D04B982
:1020B0002C68201DFFF7B2FD58B9E06A264A00EBF4
:1020C000800152F8211021B901218140A86988437B
:1020D000A861A06A18B104F11800FFF79FFD1E481F
:1020E000211DDC30FFF7EAFD94F85000002601289E
:1020F00001D184F85060FFF70DFEE86928B1FFF7C1
:10210000E9FDFFF769F9FFF705FE2868844213D15E
:10211000E86990B1A86B38B1502080F31188BFF303
:102120004F8FBFF36F8FFEE70C494FF08050086070
:10213000BFF34F8FBFF36F8F70BD0748DC3000686F
:102140002969884201D12E6070BDBDE8704000F061
:102150000FB80000E40000209016002004ED00E01D
:102160000248816B491C816370470000E400002035
:10217000144A906B10B101205062704700205062E9
:1021800090691149B0FA80F0C0F11F0000EB8000A7
:1021900051F820306BB101EB800000F10803416879
:1021A00049684160994201D149684160C86810603E
:1021B0007047502080F31188BFF34F8FBFF36F8FAC
:1021C000FEE70000E40000209016002070B51C20FF
:1021D000FFF780F9040005D00025201D2560FFF7DA
:1021E00047FD2576204670BD2DE9F0410025884643
:1021F00004000AD05FEA18600FD0502080F31188E5
:10220000BFF34F8FBFF36F8FFEE7502080F311882D
:10221000BFF34F8FBFF36F8FFEE7261D04F10C074E
:10222000FFF79EFF2168F06841EA0801216017E08E
:10223000D0E9001601F07F425301236821F07F416D
:1022400002D40B4203D10AE031EA030307D1D201E1
:1022500000D50D43216841F00071FFF777FE30464D
:10226000B842E5D12068A843206000F023FC206834
:10227000BDE8F0812DE9F0479A46089F91460D464A
:1022800004004FF0000609D0280E0FD0502080F334
:102290001188BFF34F8FBFF36F8FFEE7502080F39D
:1022A0001188BFF34F8FBFF36F8FFEE71DB100F0B2
:1022B00003FB40B110E0502080F31188BFF34F8F33
:1022C000BFF36F8FFEE73FB1502080F31188BFF35B
:1022D0004F8FBFF36F8FFEE7FFF742FFD4F8008008
:1022E000524629464046FFF7B5F840B1002746461A
:1022F000B9F1000F15D02068A843206011E0AFB1FC
:10230000B9F1000F01D04FF08076BAF1000F01D083
:1023100046F0806645EA06013A46201DFFF7F0FDCB
:10232000002600F0C7FB1FB310B109E04646F8E7EE
:1023300011494FF080500860BFF34F8FBFF36F8F8C
:10234000FFF780FC0646800110D4FFF7C3FC266827
:10235000524629463046FFF77DF828B1B9F1000F03
:1023600002D02068A8432060FFF7D4FC26F07F4607
:102370003046BDE8F087000004ED00E01CB52649BA
:1023800008780190FF20087008788DF800009DF80B
:1023900000009DF8002000F0F000904207D050208F
:1023A00080F31188BFF34F8FBFF36F8FFEE79DF867
:1023B00000001A4B00F0500018700720986006E0EB
:1023C000401E98609DF8000040008DF800009DF8C8
:1023D000000000069868F3D4032807D0502080F34B
:1023E0001188BFF34F8FBFF36F8FFEE74FF440703C
:1023F0009860019808700A48016841F47001016012
:10240000016841F070410160FFF7C6FC0020586090
:10241000F5F788FE00201CBD00E400E03801002034
:1024200020ED00E0F8B517460E46050014D0DEB1E9
:1024300005FB06F04830FFF74DF804000AD00020F5
:1024400084F8460004F148023B4631462846009491
:10245000FEF734FF2046F8BD502080F31188BFF30B
:102460004F8FBFF36F8FFEE70020E3E770B50D4697
:10247000040025D0FFF72EFCD4E90F20216802FBD1
:10248000001161600021A1632168A1600A46D4E9BE
:102490000F01401E00FB0121E16021464FF0FF309B
:1024A00001F8440F487004F110008DB1FFF7E0FB14
:1024B00004F12400FFF7DCFBFFF72CFC012070BDCA
:1024C000502080F31188BFF34F8FBFF36F8FFEE76B
:1024D00021690029F0D000F0B3FA0028ECD00449BB
:1024E0004FF080500860BFF34F8FBFF36F8FE3E76B
:1024F00004ED00E02DE9FF4F83B01F468B4604003A
:102500004FF0000603D0BBF1000F08D011E05020BF
:1025100080F31188BFF34F8FBFF36F8FFEE7206CFE
:1025200038B1502080F31188BFF34F8FBFF36F8F06
:10253000FEE7022F0AD1E06B012807D0502080F37C
:102540001188BFF34F8FBFF36F8FFEE700F0B4F930
:10255000DFF800914FF0000A4FF0805848B9059815
:1025600038B1502080F31188BFF34F8FBFF36F8FC6
:10257000FEE7FFF7AFFBA06BE16B884205D3022FAC
:1025800003D00598C8B1DEB11EE03A465946204650
:10259000FEF7EFFD616A19B104F1240000F050FA72
:1025A00028B1C9F80080BFF34F8FBFF36F8FFFF7DB
:1025B000B1FB012007B0BDE8F08FFFF7ABFB21E0D6
:1025C0006846FFF777FC0126FFF7A4FBFFF7C8FD7D
:1025D000FFF780FB94F94400401C01D184F844A02B
:1025E00094F94500401C01D184F845A0FFF792FB07
:1025F00005A9684600F0CCF830B12046FEF734FF5C
:1026000000F058FA0020D5E7FFF764FBA06BE16B00
:10261000884201D1012500E00025FFF77BFB95B141
:1026200004F110000599FFF753FC2046FEF71CFF4C
:1026300000F040FA00289CD1C9F80080BFF34F8F0A
:10264000BFF36F8F95E72046FEF70EFF00F032FADA
:102650008FE7000004ED00E02DE9F74783B08A46DC
:1026600004004FF0000603D0BAF1000F08D011E0CB
:10267000502080F31188BFF34F8FBFF36F8FFEE7B9
:10268000206C38B1502080F31188BFF34F8FBFF317
:102690006F8FFEE700F010F9DFF8F09000274FF0A1
:1026A000805848B9059838B1502080F31188BFF39D
:1026B0004F8FBFF36F8FFEE7FFF70CFBA56BC5B124
:1026C00051462046FEF742FD6D1EA563206950B1BC
:1026D00004F1100000F0B4F928B1C9F80080BFF38C
:1026E0004F8FBFF36F8FFFF715FB012006B0BDE8DA
:1026F000F087059808B11EB106E0FFF70BFB27E055
:102700006846FFF7D7FB0126FFF704FBFFF728FD1C
:10271000FFF7E0FA94F94400401C01D184F84470BA
:1027200094F94500401C01D184F84570FFF7F2FA96
:1027300005A9684600F02CF8002820460AD0FEF7CC
:1027400093FE00F0B7F92046FEF738FE0028B3D01C
:102750000020CBE7FEF732FE90B104F1240005998A
:10276000FFF7B6FB2046FEF77FFE00F0A3F9002836
:10277000A2D1C9F80080BFF34F8FBFF36F8F9BE7E3
:102780002046FEF771FE00F095F995E704ED00E0B4
:102790002DE9F0410C46050011D0C4B1FFF79AFABB
:1027A000174E71696B682268C81A571C17D02F68BA
:1027B000B66AB74219D08B4217D8012410E05020D6
:1027C00080F31188BFF34F8FBFF36F8FFEE7502068
:1027D00080F31188BFF34F8FBFF36F8FFEE70024A4
:1027E000FFF798FA2046BDE8F081824205D9101A19
:1027F00020602846FFF75EFBF1E700202060DCE761
:10280000E40000202DE9FF5F8346DDE90E8799464D
:1028100016468A469000FEF75DFE05001CD0542047
:10282000FEF758FE040014D00020256384F8510000
:10283000CDE90240CDE900874B4632465146584625
:10284000FEF747FD2046FEF719FC012004B0BDE865
:10285000F09F2846FFF772FA4FF0FF30F6E7F0B529
:1028600085B00546DDE90B040A9EA8B1E4B1542702
:1028700000972063022084F851000020CDE9024037
:1028800004AF2846CDE90067FEF723FD2046FEF79A
:10289000F5FB049805B0F0BD502080F31188BFF31C
:1028A0004F8FBFF36F8FFEE7502080F31188BFF387
:1028B0004F8FBFF36F8FFEE70548C16919B1806B79
:1028C00018B10020704701207047022070470000B7
:1028D000E40000200148406970470000E400002047
:1028E0002DE9F0412E4F0026B86B40B1386A401CEC
:1028F0003862786A00B101263046BDE8F0817D6912
:102900006D1C7D6113D17868006838B1502080F368
:102910001188BFF34F8FBFF36F8FFEE77868B968F8
:102920007960B860B86A401CB862FEF755FD386B34
:10293000DFF87080854209D37868006880B17868D4
:10294000C068C468606885420DD238633868C06A60
:1029500000EB800158F821000128CAD90126C8E7F8
:102960004FF0FF30F1E7201DFFF758F9A06A18B1CA
:1029700004F11800FFF752F9E06A0121BA698140B9
:102980001143B96100EB800108EB8100211DFFF7C5
:1029900095F9E06A3968C96A8842CDD30126CBE748
:1029A000E40000209016002070B504004FF00000F5
:1029B00041D0214D29688C4207D0502080F31188E6
:1029C000BFF34F8FBFF36F8FFEE7A16C71B1491E4C
:1029D000A164636CE26A9A422DD000292BD1201D9C
:1029E000FFF71CF91549012240B112E0502080F395
:1029F0001188BFF34F8FBFF36F8FFEE7E06A00EBE4
:102A0000800351F8233023B9AB6902FA00F0834305
:102A1000AB61606CE062C0F10700A061E06AAB6985
:102A200082401A43AA6100EB800001EB8000211D67
:102A3000FFF744F9012070BDE4000020901600204B
:102A40002DE9F041C068C468ACB104F11800074634
:102A5000FFF7E4F8154DA86B0126A0B139461448DC
:102A6000FFF72CF9E06A2968C96A88421CD901205D
:102A70006E62BDE8F081502080F31188BFF34F8F64
:102A8000BFF36F8FFEE7201DFFF7C8F8E06AAA6961
:102A900006FA00F11143A961054900EB8000B43941
:102AA00001EB8000211DDBE70020E2E7E4000020CD
:102AB000441700202DE9F0472C4D00242746A86B31
:102AC00038B1FFF707F9A86B401EA863A86B40B1A7
:102AD00046E0502080F31188BFF34F8FBFF36F8F14
:102AE000FEE7286922490126D0B3A1F1B40988463E
:102AF000D8F80010E9B1D8F80C00C46804F1180047
:102B0000FFF78CF8201DFFF789F8E06AAA6906FA3A
:102B100000F11143A96100EB800109EB8100211D47
:102B2000FFF7CCF8E06A2968C96A8842E0D36E6290
:102B3000DEE70CB1FEF750FC2C6A3CB1FFF7D0FE8B
:102B400000B16E62641EF9D100202862686A38B153
:102B50000849012738070860BFF34F8FBFF36F8F15
:102B6000FFF7D8F83846BDE8F0870000E400002001
:102B70004417002004ED00E00831010855E5000885
:102B80000000000000000000800000001005002090
:102B900010070020000000000000000001020304F4
:102BA00006070809000000000102030400000000FD
:102BB0000000000000000000010003000500070005
:102BC00009000B000D000F00110013001500170085
:102BD00019001B001D001F002100230025002700F5
:102BE00029002B002D002F00310033003500370065
:102BF00039003B003D003E003F00400041004200E4
:102C000043004400450046004700480049004A0090
:102C10004B004C004D004E004F0050005100520040
:102C200053005400550056005700580059005A00F0
:102C30005B005C005D005E005F00600061006200A0
:102C400063006400650066006700680069006A0050
:102C50006B006C006D006E006F0070007100720000
:102C600073007400750076007700780079007A00B0
:102C70007B007C007D007E007F0080008100820060
:102C800083008400850086008700880089008A0010
:102C90008B008C008D008E008F00900091009200C0
:102CA00093009400950096009700980099009A0070
:102CB0009B009C009D009E009F00A000A100A20020
:102CC000A300A400A500A600A700A800A900AA00D0
:102CD000AB00AC00AD00AE00AF00B000B100B20080
:102CE000B300B400B500B600B700B800B900BA0030
:102CF000BB00BC00BD00BE00BF00C000C100C200E0
:102D0000C300C400C500C600C700C800C900CA008F
:102D1000CB00CC00CD00CE00CF00D000D100D2003F
:102D2000D300D400D500D600D700D800D900DA00EF
:102D3000DB00DC00DD00DE00DF00E000E100E2009F
:102D4000E300E400E500E600E700E800E900EA004F
:102D5000EB00EC00ED00EE00EF00F000F100F200FF
:102D6000F300F400F500F600F700F800F900FA00AF
:102D7000FB00FC00FD00FE00FF000001010102015C
:102D800003010401050106010701080109010A0107
:102D90000B010C010D010E010F01100111011201B7
:102DA00013011401150116011701180119011A0167
:102DB0001B011C011D011E011F0120012101220117
:102DC00023012401250126012701280129012A01C7
:102DD0002B012C012D012E012F0130013101320177
:102DE00033013401350136013701380139013A0127
:102DF0003B013C013D013E013F01400141014201D7
:102E000043014401450146014701480149014A0186
:102E10004B014C014D014E014F0150015101520136
:102E200053015401550156015701580159015A01E6
:102E30005B015C015D015E015F0160016101620196
:102E400063016401650166016701680169016A0146
:102E50006B016C016D016E016F01700171017201F6
:102E600073017401750176017701780179017A01A6
:102E70007B017C017D017E017F0180018101820156
:102E800083018401850186018701880189018A0106
:102E90008B018C018D018E018F01900191019201B6
:102EA00093019401950196019701980199019A0166
:102EB0009B019C019D019E019F01A001A101A20116
:102EC000A301A401A501A601A701A801A901AA01C6
:102ED000AB01AC01AD01AE01AF01B001B101B20176
:102EE000B301B401B501B601B701B801B901BA0126
:102EF000BB01BC01BD01BE01BF01C001C101C201D6
:102F0000C301C401C501C601C701C801C901CA0185
:102F1000CB01CC01CD01CE01CF01D001D101D20135
:102F2000D301D401D501D601D701D801D901DA01E5
:102F3000DB01DC01DD01DE01DF01E001E101E20195
:102F4000E301E401E501E601E701E801E901EA0145
:102F5000EB01EC01ED01EE01EF01F001F101F201F5
:102F6000F301F401F501F601F701F801F901FA01A5
:102F7000FB01FC01FD01FE01FF0100020002000255
:102F80000002000200020002000200020002000231
:102F90000002000200020002000200020002000221
:102FA000000200020002000200020002000200D53E
:102FB0007FAAFE2B815429FC5683D702A87D528715
:102FC0002DF8AC79D3067BAE04D18550FA2FA471CD
:102FD000DB0E5A8F25F08D58F22773A60CD9F623F5
:102FE000895C08DD77A2DF0AA07521F45E8B9D481D
:102FF000E23763B61CC9B461CB1E4A9F35E0CF1AD5
:10300000B06531E44E9BE633994C18CD67B239EC8C
:103010004693C712B86D10C56FBAEE3B91446BBEB4
:1030200014C19540EA3F42973DE8BC69C316EF3AA8
:10303000904511C46EBBC613B96C38ED4792BD689C
:10304000C21743963CE99441EB3E6ABF15C04B9EC4
:1030500034E1B560CA1F62B71DC89C49E33619CC7C
:1030600066B3E732984D30E54F9ACE1BB16472A734
:103070000DD88C59F3265B8E24F1A570DA0F20F55C
:103080005F8ADE0BA17409DC76A3F722885DD60384
:10309000A97C28FD5782FF2A805501D47EAB84513C
:1030A000FB2E7AAF05D0AD78D20753862CF90000FD
:1030B000891112239B322446AD573665BF74488C64
:1030C000C19D5AAFD3BE6CCAE5DB7EE9F7F80302B7
:1030D00000010405060708090A0B0C0D0E0F2F2E20
:1030E0002F07D3910D040C291006005C4EC47C43BD
:1030F00083233B44070C081D1C434091576BF8B6D3
:1031000010EA0A111100000064656661756C745460
:1031100061736B00343101080000002010050000CD
:1031200008890008EC32010810050020B8420000B0
:103130006C0301088113F9EF140831F01B083D04FA
:103140001A65041A8D041AD1141A05081704030904
:103150000412013202164083045057260201020372
:1031600001031A1A031F05010904A101061301A195
:103170001008093309340935151226580908751045
:1031800095038102C0183E3009310932184D95036C
:103190007510181A36186A362C0A1501141B090105
:1031A0000E12FF2009954075089102C05814202383
:1031B000911B081F041A2904199B1182100359241A
:1031C000F41AAA018113B9ED1B082F041349EE422A
:1031D000081A670C13FDEC1B080B08C11AA1101A82
:1031E00095041AAD041A8904140902291301012552
:1031F000C032090433020315092111011401226CA4
:103200001607058103022D0207050107291A091E69
:103210002C4A052C0A22052CA958691A313B0A06AA
:1032200013034F4001198C111201054AE40CE40C00
:103230000D12FE0FFF070601541250130206101163
:1032400006170C18180619070508053EFF0B080C91
:1032500010260D5C0E760F2710AA113912111323B8
:10326000147A15421B0319161A6C1C401D91215625
:10327000221023A9240A25480E261129592C882D0D
:10328000312E0B030709481A0E487E230704080154
:103290004813800F3F107B11F81203482A53460B46
:1032A0001F1B434829905A1E487A0A903E7B1161A1
:1032B0001213480A205148014362020B1CDC05022C
:1032C000514AFF2D09131C011C052340FFFFFF126B
:1032D0000F100B341FA809086A5003108013042034
:0C32E0001501080738290B09249E110075
:04000005080080ED82
:00000001FF
